:020000040800F2
:100000000000012045DC00082FDC000831DC00087E
:1000100033DC000835DC000837DC00080000000095
:1000200000000000000000000000000039DC0008B3
:100030003BDC0008000000003DDC00083FDC00085D
:1000400095DC000895DC000895DC000895DC0008CC
:1000500095DC000895DC000895DC000895DC0008BC
:1000600095DC000895DC000895DC000895DC0008AC
:1000700095DC000895DC000895DC000895DC00089C
:1000800095DC000895DC000895DC000895DC00088C
:100090000000000095DC000895DC000895DC0008F5
:1000A00095DC000895DC000895DC000895DC00086C
:1000B00095DC000895DC000895DC000895DC00085C
:1000C00095DC000895DC000895DC000895DC00084C
:1000D0003D3800086D3500083965000895DC0008DA
:1000E00095DC000895DC000895DC000895DC00082C
:1000F00095DC0008000000000000000095DC00080E
:1001000095DC000895DC000861C6000895DC000855
:1001100095DC000895DC000895DC000895DC0008FB
:1001200095DC000895DC000895DC000895DC0008EB
:0801300095DC000895DC0008D5
:1001380010B5054C237833B9044B13B10448AFF319
:1001480000800123237010BDA802002000000000D9
:100158000C10010808B5034B1BB103490348AFF362
:10016800008008BD00000000AC0200200C1001084F
:1001780010F8012B11F8013B012A28BF9A42F7D049
:10018800D01A7047034613F8012B002AFBD1181A1E
:100198000138704781F0004102E000BF83F000435E
:1001A80030B54FEA41044FEA430594EA050F08BF0A
:1001B80090EA020F1FBF54EA000C55EA020C7FEACE
:1001C800645C7FEA655C00F0E2804FEA5454D4EB4B
:1001D8005555B8BF6D420CDD2C4480EA020281EA15
:1001E800030382EA000083EA010180EA020281EA4D
:1001F8000303362D88BF30BD11F0004F4FEA01319F
:100208004FF4801C4CEA113102D0404261EB4101AD
:1002180013F0004F4FEA03334CEA133302D0524233
:1002280063EB430394EA050F00F0A780A4F10104EF
:10023800D5F1200E0DDB02FA0EFC22FA05F2801829
:1002480041F1000103FA0EF2801843FA05F359410F
:100258000EE0A5F120050EF1200E012A03FA0EFC8E
:1002680028BF4CF0020C43FA05F3C01851EBE371B8
:1002780001F0004507D54FF0000EDCF1000C7EEBD5
:1002880000006EEB0101B1F5801F1BD3B1F5001F13
:100298000CD349085FEA30004FEA3C0C04F1010432
:1002A8004FEA445212F5800F80F09A80BCF1004F5B
:1002B80008BF5FEA500C50F1000041EB045141EADD
:1002C800050130BD5FEA4C0C404141EB0101013CA6
:1002D80028BFB1F5801FE9D291F0000F04BF014695
:1002E8000020B1FA81F308BF2033A3F10B03B3F167
:1002F80020020CDA0C3208DD02F1140CC2F10C02F7
:1003080001FA0CF021FA02F10CE002F11402D8BF54
:10031800C2F1200C01FA02F120FA0CFCDCBF41EA20
:100328000C019040E41AA2BF01EB0451294330BDEF
:100338006FEA04041F3C1CDA0C340EDC04F11404CC
:10034800C4F1200220FA04F001FA02F340EA0300A3
:1003580021FA04F345EA030130BDC4F10C04C4F1E9
:10036800200220FA02F001FA04F340EA03002946C9
:1003780030BD21FA04F0294630BD94F0000F83F413
:10038800801306BF81F480110134013D4EE77FEAF6
:10039800645C18BF7FEA655C29D094EA050F08BF42
:1003A80090EA020F05D054EA000C04BF1946104623
:1003B80030BD91EA030F1EBF0021002030BD5FEA67
:1003C800545C05D14000494128BF41F0004130BD8F
:1003D80014F580043CBF01F5801130BD01F00045E3
:1003E80045F0FE4141F470014FF0000030BD7FEA56
:1003F800645C1ABF194610467FEA655C1CBF0B4651
:10040800024650EA013406BF52EA033591EA030F67
:1004180041F4002130BD00BF90F0000F04BF00215F
:10042800704730B54FF4806404F132044FF0000592
:100438004FF0000150E700BF90F0000F04BF00210B
:10044800704730B54FF4806404F1320410F0004571
:1004580048BF40424FF000013EE700BF42004FEA6C
:10046800E2014FEA31014FEA02701FBF12F07F43E9
:1004780093F07F4F81F06051704732F07F4208BFA0
:10048800704793F07F4F04BF41F40021704730B5A7
:100498004FF4607401F0004521F000411CE700BFF3
:1004A80050EA010208BF704730B54FF000050AE076
:1004B80050EA010208BF704730B511F0004502D577
:1004C800404261EB41014FF4806404F132045FEA79
:1004D800915C3FF4D8AE4FF003025FEADC0C18BF22
:1004E80003325FEADC0C18BF033202EBDC02C2F114
:1004F800200300FA03FC20FA02F001FA03FE40EAA6
:100508000E0021FA02F11444BDE600BF70B54FF0A9
:10051800FF0C4CF4E06C1CEA11541DBF1CEA135587
:1005280094EA0C0F95EA0C0F00F0DEF82C4481EAEF
:10053800030621EA4C5123EA4C5350EA013518BF0F
:1005480052EA033541F4801143F4801338D0A0FBFC
:1005580002CE4FF00005E1FB02E506F00042E0FBA9
:1005680003E54FF00006E1FB03569CF0000F18BFAF
:100578004EF0010EA4F1FF04B6F5007F64F5407457
:1005880004D25FEA4E0E6D4146EB060642EAC621EA
:1005980041EA55514FEAC52040EA5E504FEACE2E57
:1005A800B4F1FD0C88BFBCF5E06F1ED8BEF1004F5A
:1005B80008BF5FEA500E50F1000041EB045170BDD6
:1005C80006F0004646EA010140EA020081EA03011A
:1005D800B4EB5C04C2BFD4EB0C0541EA045170BD16
:1005E80041F480114FF0000E013C00F3AB8014F190
:1005F800360FDEBF002001F0004170BDC4F10004D9
:10060800203C35DA0C341BDC04F11404C4F1200559
:1006180000FA05F320FA04F001FA05F240EA0200B4
:1006280001F0004221F0004110EBD37021FA04F6EA
:1006380042EB06015EEA430E08BF20EAD37070BDA4
:10064800C4F10C04C4F1200500FA04F320FA05F003
:1006580001FA04F240EA020001F0004110EBD37005
:1006680041F100015EEA430E08BF20EAD37070BD75
:10067800C4F1200500FA05F24EEA020E20FA04F34E
:1006880001FA05F243EA020321FA04F001F00041FD
:1006980021FA04F220EA020000EBD3705EEA430E6E
:1006A80008BF20EAD37070BD94F0000F0FD101F09D
:1006B8000046400041EB010111F4801F08BF013CD6
:1006C800F7D041EA060195F0000F18BF704703F014
:1006D8000046520043EB030313F4801F08BF013D9B
:1006E800F7D043EA0603704794EA0C0F0CEA135557
:1006F80018BF95EA0C0F0CD050EA410618BF52EA11
:100708004306D1D181EA030101F000414FF0000016
:1007180070BD50EA410606BF1046194652EA430624
:1007280019D094EA0C0F02D150EA013613D195EA98
:100738000C0F05D152EA03361CBF104619460AD1E0
:1007480081EA030101F0004141F0FE4141F47001EA
:100758004FF0000070BD41F0FE4141F4780170BDDA
:1007680070B54FF0FF0C4CF4E06C1CEA11541DBF3F
:100778001CEA135594EA0C0F95EA0C0F00F0A7F841
:10078800A4EB050481EA030E52EA03354FEA01316E
:1007980000F088804FEA03334FF0805545EA131381
:1007A80043EA12634FEA022245EA111545EA106549
:1007B8004FEA00260EF000419D4208BF964244F1E0
:1007C800FD0404F5407402D25B084FEA3202B61AFF
:1007D80065EB03055B084FEA32024FF480104FF4D3
:1007E800002CB6EB020E75EB030E22BFB61A754647
:1007F80040EA0C005B084FEA3202B6EB020E75EBDA
:10080800030E22BFB61A754640EA5C005B084FEA41
:100818003202B6EB020E75EB030E22BFB61A75460E
:1008280040EA9C005B084FEA3202B6EB020E75EB19
:10083800030E22BFB61A754640EADC0055EA060EDA
:1008480018D04FEA051545EA16754FEA06164FEA1D
:10085800C30343EA52734FEAC2025FEA1C1CC0D1C9
:1008680011F4801F0BD141EA00014FF000004FF056
:10087800004CB6E711F4801F04BF01430020B4F117
:10088800FD0C88BFBCF5E06F3FF6AFAEB5EB030CCF
:1008980004BFB6EB020C5FEA500C50F1000041EBCC
:1008A800045170BD0EF0004E4EEA113114EB5C0499
:1008B800C2BFD4EB0C0541EA045170BD41F480116C
:1008C8004FF0000E013C90E645EA060E8DE60CEA74
:1008D800135594EA0C0F08BF95EA0C0F3FF43BAF91
:1008E80094EA0C0F0AD150EA01347FF434AF95EA48
:1008F8000C0F7FF425AF104619462CE795EA0C0F2C
:1009080006D152EA03353FF4FDAE1046194622E7F8
:1009180050EA410618BF52EA43067FF4C5AE50EAD2
:1009280041047FF40DAF52EA43057FF4EBAE12E7C2
:100938004A0011D212F5001211D20DD56FF4787356
:10094800B3EB62520ED44FEAC12343F0004343EAAB
:10095800505323FA02F070474FF00000704750EAF6
:10096800013002D14FF0FF3070474FF00000704760
:1009780080F0004002E000BF81F0004142001FBF4C
:100988005FEA410392EA030F7FEA226C7FEA236C55
:100998006AD04FEA1262D2EB1363C1BFD21841404A
:1009A80048404140B8BF5B42192B88BF704710F0E0
:1009B800004F40F4000020F07F4018BF404211F083
:1009C800004F41F4000121F07F4118BF494292EAEB
:1009D800030F3FD0A2F1010241FA03FC10EB0C0017
:1009E800C3F1200301FA03F100F0004302D54942A4
:1009F80060EB4000B0F5000F13D3B0F1807F06D351
:100A080040084FEA310102F10102FE2A51D2B1F148
:100A1800004F40EBC25008BF20F0010040EA03003D
:100A28007047490040EB0000013A28BFB0F5000FBD
:100A3800EDD2B0FA80FCACF1080CB2EB0C0200FA73
:100A48000CF0AABF00EBC25052421843BCBFD040C2
:100A58001843704792F0000F81F4000106BF80F43C
:100A680000000132013BB5E74FEA41037FEA226CFF
:100A780018BF7FEA236C21D092EA030F04D092F0CA
:100A8800000F08BF0846704790EA010F1CBF0020FE
:100A9800704712F07F4F04D1400028BF40F000405B
:100AA800704712F100723CBF00F50000704700F07B
:100AB800004343F0FE4040F4000070477FEA2262A2
:100AC80016BF08467FEA23630146420206BF5FEA73
:100AD800412390EA010F40F4800070474FF0000373
:100AE80004E000BF10F0004348BF40425FEA000C3A
:100AF80008BF704743F0964301464FF000001CE0E2
:100B080050EA010208BF70474FF000030AE000BF37
:100B180050EA010208BF704711F0004302D5404275
:100B280061EB41015FEA010C02BF844601460020E7
:100B380043F0B64308BFA3F18053A3F50003BCFA02
:100B48008CF2083AA3EBC25310DB01FA02FC6344AF
:100B580000FA02FCC2F12002BCF1004F20FA02F2B6
:100B680043EB020008BF20F00100704702F12002A9
:100B780001FA02FCC2F1200250EA4C0021FA02F20A
:100B880043EB020008BF20EADC7070474FF0FF0C0F
:100B98001CEAD0521EBF1CEAD15392EA0C0F93EA0A
:100BA8000C0F6FD01A4480EA010C400218BF5FEAAC
:100BB80041211ED04FF0006343EA501043EA51111F
:100BC800A0FB01310CF00040B1F5000F3EBF490019
:100BD80041EAD3715B0040EA010062F17F02FD2A1D
:100BE8001DD8B3F1004F40EBC25008BF20F0010000
:100BF800704790F0000F0CF0004C08BF49024CEA17
:100C0800502040EA51207F3AC2BFD2F1FF0340EAA8
:100C1800C250704740F400004FF00003013A5DDC19
:100C280012F1190FDCBF00F000407047C2F100025A
:100C3800410021FA02F1C2F1200200FA02FC5FEA47
:100C4800310040F1000053EA4C0308BF20EADC7091
:100C5800704792F0000F00F0004C02BF400010F403
:100C6800000F013AF9D040EA0C0093F0000F01F0B0
:100C7800004C02BF490011F4000F013BF9D041EAD2
:100C88000C018FE70CEAD15392EA0C0F18BF93EAD4
:100C98000C0F0AD030F0004C18BF31F0004CD8D1FE
:100CA80080EA010000F00040704790F0000F17BF85
:100CB80090F0004F084691F0000F91F0004F14D0CB
:100CC80092EA0C0F01D142020FD193EA0C0F03D123
:100CD8004B0218BF084608D180EA010000F0004026
:100CE80040F0FE4040F40000704740F0FE4040F401
:100CF800400070474FF0FF0C1CEAD0521EBF1CEAA0
:100D0800D15392EA0C0F93EA0C0F69D0A2EB0302BD
:100D180080EA010C49024FEA402037D04FF0805357
:100D280043EA111143EA10130CF000408B4238BF1C
:100D38005B0042F17D024FF4000C8B4224BF5B1A2A
:100D480040EA0C00B3EB510F24BFA3EB510340EA78
:100D58005C00B3EB910F24BFA3EB910340EA9C0026
:100D6800B3EBD10F24BFA3EBD10340EADC001B0196
:100D780018BF5FEA1C1CE0D1FD2A3FF650AF8B423A
:100D880040EBC25008BF20F0010070470CF0004C47
:100D98004CEA50207F32C2BFD2F1FF0340EAC25072
:100DA800704740F400004FF00003013A37E792F033
:100DB800000F00F0004C02BF400010F4000F013A91
:100DC800F9D040EA0C0093F0000F01F0004C02BF8C
:100DD800490011F4000F013BF9D041EA0C0195E7F5
:100DE8000CEAD15392EA0C0F08D142027FF47DAF8E
:100DF80093EA0C0F7FF470AF084676E793EA0C0F7E
:100E080004D14B023FF44CAF08466EE730F0004C7B
:100E180018BF31F0004CCAD130F000427FF45CAF0B
:100E280031F000437FF43CAF5FE700BF4FF0FF3C79
:100E380006E000BF4FF0010C02E000BF4FF0010CCC
:100E48004DF804CD4FEA40024FEA41037FEA226C95
:100E580018BF7FEA236C11D001B052EA530C18BFB7
:100E680090EA010F58BFB2EB030088BFC81738BF1C
:100E78006FEAE17018BF40F0010070477FEA226C0A
:100E880002D15FEA402C05D17FEA236CE4D15FEA06
:100E9800412CE1D05DF8040B704700BF844608463A
:100EA8006146FFE70FB5FFF7C9FF002848BF10F1FB
:100EB800000F0FBD4DF808EDFFF7F4FF0CBF012040
:100EC80000205DF808FB00BF4DF808EDFFF7EAFFCA
:100ED80034BF012000205DF808FB00BF4DF808ED85
:100EE800FFF7E0FF94BF012000205DF808FB00BF7A
:100EF8004DF808EDFFF7D2FF94BF012000205DF800
:100F080008FB00BF4DF808EDFFF7C8FF34BF01200C
:100F180000205DF808FB00BF4FEA40024FEA41039A
:100F28007FEA226C02D15FEA402C08D17FEA236C69
:100F380002D15FEA412C02D14FF0000070474FF018
:100F4800010070474FEA4002B2F1FE4F0FD34FF055
:100F58009E03B3EB12620DD94FEA002343F000431E
:100F680010F0004F23FA02F018BF404270474FF0CC
:100F78000000704712F1610F01D1420205D110F053
:100F8800004008BF6FF0004070474FF00000704706
:100F980042000ED2B2F1FE4F0BD34FF09E03B3EBDB
:100FA800126209D44FEA002343F0004323FA02F007
:100FB80070474FF00000704712F1610F01D14202F3
:100FC80002D14FF0FF3070474FF00000704700BF6C
:100FD80053B94AB9002908BF00281CBF4FF0FF3198
:100FE8004FF0FF3000F070B9ADF1080C6DE904CE98
:100FF80000F006F8DDF804E0DDE9022304B07047EC
:101008002DE9F047089E0D4604460F46002B4AD1AD
:101018008A42944665D9B2FA82F343B102FA03FCD4
:10102800C3F120029F4020FA02F217439C404FEA86
:101038001C4E1FFA8CF5B7FBFEF1220C0EFB117744
:1010480042EA074201FB05F090420AD91CEB020272
:1010580001F1FF3780F01B81904240F2188102397C
:101068006244121AA4B2B2FBFEF00EFB102244EA4C
:10107800024400FB05F5A5420AD91CEB040400F163
:10108800FF3280F00681A54240F2038164440238B1
:1010980040EA0140641B00211EB1DC400023C6E980
:1010A8000043BDE8F0878B4208D9002E00F0EC80A1
:1010B8000021C6E900050846BDE8F087B3FA83F1C8
:1010C800002949D1AB4202D3824200F2F780841A48
:1010D80065EB030201201746002EE2D0C6E900475F
:1010E800DFE702B9FFDEB2FA82F3002B40F08F800F
:1010F8008A1A4FEA1C471FFA8CFE0121B2FBF7F54A
:1011080007FB1520220C42EA00420EFB05F0904234
:1011180008D91CEB020205F1FF3802D2904200F216
:10112800CA804546121AA4B2B2FBF7F007FB102298
:1011380044EA02440EFB00FEA64508D91CEB040451
:1011480000F1FF3202D2A64500F2BA801046A4EBA5
:101158000E0440EA05409FE7C1F120078B4022FAC0
:1011680007FC4CEA030C05FA01F420FA07F3FD40EA
:10117800234300FA01F94FEA1C401FFA8CFEB5FB25
:10118800F0F81C0C00FB185544EA054408FB0EF562
:10119800A54202FA01F20BD91CEB040408F1FF3A4C
:1011A80080F08780A54240F28480A8F10208644458
:1011B800641B9DB2B4FBF0F300FB134445EA0444FE
:1011C80003FB0EFEA64508D91CEB040403F1FF300F
:1011D8006BD2A64569D9023B644443EA0840A0FBA8
:1011E8000283A4EB0E049C42C6461D4655D352D03A
:1011F80056B1B9EB0E0364EB050404FA07F7CB40CC
:10120800CC401F43C6E900740021BDE8F087C3F154
:10121800200102FA03FC20FA01F225FA01F19D40AF
:101228002A434FEA1C471FFA8CFEB1FBF7F007FB75
:101238001015110C41EA054100FB0EF58D4204FA28
:1012480003F408D91CEB010100F1FF382FD28D42BD
:101258002DD902386144491B92B2B1FBF7F507FB5F
:10126800151142EA014205FB0EF1914208D91CEB27
:10127800020205F1FF3816D2914214D9023D6244A8
:10128800521A45EA004139E73146304609E73946FE
:10129800E7E61046FCE6C145AAD2B8EB020E63EBBE
:1012A8000C050138A4E74546EAE7034695E74046BA
:1012B800D1E7D0467CE7023D624433E708460BE7B6
:1012C8006444023843E700BF704700BF0022427001
:1012D80082700122C270B1FA81F1022249090271B9
:1012E800032201704271704743788B421FD0012955
:1012F80041700AD0022910D0C1B90123C37081708E
:1013080002230371032343717047037843B1012318
:1013180083700223C3700023F3E70378002BF6D011
:10132800022383700023C3700123EAE7FEE77047B6
:1013380082B00B88ADF800304B88ADF802308B884E
:10134800ADF80430CB88ADF806300239431C0530BF
:1013580013F8012F0DF1080C0CEB4202834232F80E
:10136800082C21F8022FF3D102B0704710B50C46B3
:101378001146FFF7B9FF2146BDE81040FFF7D8BF77
:101388000A4B10B54FF07F32C0E923234FF47F4357
:10139800A0F89430FF2380F896300446983000F087
:1013A800E3FC002384F8A43010BD00BFFFFF7F00DA
:1013B80070B51146154604461E4600F04BFC2946FA
:1013C80004F1140000F046FC294604F1280000F05E
:1013D80041FC294604F13C0000F03CFC294604F19C
:1013E800500000F037FC294604F1640000F032FC9C
:1013F800294604F1780000F02DFC4FF4FA733246C8
:101408004FF4FA6104F1980000F094FC2046FFF7CD
:10141800B7FF002384F8A5304FF47F43A4F8A63023
:1014280070BD704700F01DBC143000F01ABC08B540
:10143800503000F020FC292100F114030246B3FBD0
:10144800F1F313F0FF0002D1101E18BF012008BDF0
:1014580008B5643000F00FFC292100F1140302469E
:10146800B3FBF1F313F0FF0002D1101E18BF0120E7
:1014780008BD90F8903013B990F98C00704790F936
:101488008D00704790F8903013B990F98E0070472E
:1014980090F98F00704710B504460BF0FDF938B18C
:1014A80004F13C0000F0E1FB012838BF0120C0B284
:1014B80010BD783000F0E1BB783000F0E6BB10B525
:1014C800044600F0A8FB04F1140000F0A4FB04F1AA
:1014D800280000F0A0FB04F13C0000F09CFB04F1A4
:1014E800500000F0A4FB04F1640000F0A0FB04F13C
:1014F8007800BDE8104000F0A0BB7F2807D0002886
:1015080007DA10F1800F06D04042C0B270470020C1
:101518007047012070477F20704710B1404240B2A9
:1015280070477F2070477F280FD010F1310F0EDAF7
:1015380010F1780F0DDB7830FE2340B2584323308A
:101548004623B0FBF3F0C0B27047FF207047FE207F
:10155800704700207047012805DD40F2FE7398426D
:1015680003DC80B270470120704740F2FF7070477B
:10157800A0F57870C0EBC02040F2AE7390FBF3F09A
:1015880000F58060FFF7E7BFFFF7F2BF032812DD21
:101598000C2812DD0F2812DD122812DD162812DDA4
:1015A800192812DD1C2812DD1F2812DD2128CCBFC6
:1015B800FF20062070470020704701207047022056
:1015C80070470820704703207047072070470420A1
:1015D800704705207047000005289ABF014B185C2A
:1015E800FF2070476810010805289ABF014B185C56
:1015F800FF2070476E1001087F2803D0002803DA07
:10160800C0B2704700207047FF2070477F2811D074
:1016180010F1320F10DA884210DD401A6423C1F14C
:10162800FF21584301F57F01CE31313090FBF1F0B5
:10163800C0B27047FF207047642070470020704791
:10164800014B4840185C70477410010852B110B43F
:10165800054C0A4411F8013B58408A42205CF9D1F4
:1016680010BC7047704700BF74100108392808D8AB
:1016780022280ED9094B2338C0B2C34003F0010019
:1016880070475F2807D0613819288CBF00200120D7
:101698007047002070470120704700BF01EC7F00B1
:1016A800F8B50246451E461D00245F2715F8010FB0
:1016B800FF2804BF0134E4B2FFF7D8FF00B92F7048
:1016C800AE42F3D1062C04D119B10B6813608B8894
:1016D800938000239371F8BD2DE9F843DFF8349027
:1016E800471E441D012500264FF0280817F8011F42
:1016F80008480FF028FC034610B1A0EB0903DBB241
:10170800A3FB05329E19A742A5FB0853EED130462C
:10171800BDE8F8837411010810B54179A1F13000D2
:10172800C3B2092B07D80523B0FBF3F303EB8303FC
:10173800C01AC0B210BD044C20460FF004FC0028AB
:10174800F1D0001BC0B2EEE774110108F0B5094BE7
:10175800094F821D2826B1FBF3F4272C94BF3D5D69
:10176800302502F8015D824203FB1411B3FBF6F346
:10177800F1D1F0BD00801A067411010870B5044655
:10178800FEF700FD82B20023551E98B2A84214FA53
:1017980083F104DA265C302E03F10103F5D0121A26
:1017A80001322046BDE870400FF09CBB2DE9F04F98
:1017B8000D4699B0164600211A461F4680460FF07E
:1017C800ABFB00212A2201A800910FF0A5FBDFF84E
:1017D800CC90DFF8CCA0DFF8CCB005EB4606AE42E3
:1017E80011D16846FEF7CEFC30B100F160030DEB75
:1017F8000300002300F8613C694640460FF0ECFB0B
:1018080019B0BDE8F08F35F9020B47F6FF7398421F
:10181800E7D0002812DC59460CA80FF0DDFB68461B
:10182800FEF7B0FC04460CA8FEF7ACFC0444A74243
:10183800D5D30CA968460FF077FBD0E7B0F57A7FCF
:101848000BDA0CA980B20DF006FD0CA8FFF796FF85
:1018580051460CA80FF068FBE1E764230CA932306D
:10186800B0FBF3F080B20DF0F6FC0CA8FFF786FF92
:101878000CA8FEF787FC00F15F036B4400F16001E0
:101888000DEB010013F8302C00F8302C2E2203F851
:10189800302C002300F82F3C4946DAE76210010893
:1018A8005D10010858100108F0B589B06D46002494
:1018B8002F468E1CE1B28A4204D83946FFF776FFDC
:1018C80009B0F0BD36F8241025F8021B0134F1E701
:1018D80042F210736421B0FBF3F203FB1200B0FB79
:1018E800F1F301FB130000EB023000EB831080B230
:1018F8007047020B00F03F0342F2107101FB023304
:10190800C0F38510642202FB003070472DE9F041D6
:1019180042F2107388B0B1FBF3F603FB16141F49AB
:10192800DFF87C8005460FF057FB6946F0B20DF0F2
:101938006FFC6846FFF722FF694628460FF0F4FA65
:10194800414628460FF0F0FA64276946B4FBF7F6DB
:10195800F0B20DF05DFC6846FFF710FF69462846B7
:101968000FF0E2FA07FB1644414628460FF0DCFA6E
:101978006946E0B20DF04CFC9DF801308DF800305E
:101988009DF802308DF801306946002328468DF80D
:1019980002300FF0C9FA08B0BDE8F0810122010851
:1019A8006610010870B50E460021054614460FF072
:1019B800B3FA00239AB2944200D870BDF25C002AB0
:1019C800FBD0EA540133F5E770B50E461446002102
:1019D800013205460FF0A0FA00239AB2944200D8CB
:1019E80070BDF25C002AFBD0EA540133F5E730B54C
:1019F8000023044698B2904201D3012005E0E55C3B
:101A0800C85C1DB9B0FA80F0400930BD0028FCD090
:101A1800854203F10103EDD00020F6E77D234380E2
:101A280043F2390309B2C360002301808180C38077
:101A38000372704702680449044B01FB023323F028
:101A480000430360180C7047FD430300C39E260043
:101A5800F0B5002597B001608580044656222946D6
:101A680068460FF059FA0126E27DAA4209D80023F8
:101A7800802104F1B800A37517B0BDE8F0400FF05D
:101A88004BBA2046FFF7D6FFE7797B1B002190FB76
:101A9800F3F202FB1300C0B2EC460A46CBB29F42F7
:101AA80023D800230022277B1146D0B2874227D8AB
:101AB8000029D9D1A279033A012A04EB050105D9F5
:101AC80025B191F9172012BB012BCDD90B76A2684D
:101AD80052F82310583305F10E026B44013544F8CF
:101AE800221003F8586CEDB2BEE71CF801EBBEF10A
:101AF800000F03D18242D5D00132D2B20131CDE7F5
:101B08002069805C0132984208BF0121CDE7501E50
:101B18008342DBDB01329342D8DCA5E72DE9F047AD
:101B2800154696B0013D0160027104464371EDB25D
:101B38005622002168460FF0EFF90027022D84BFD6
:101B48004FF0010900253E464FF0010A94F807803E
:101B58009CBF4FF00309B8FBF9F8E27DB24209D8FF
:101B68000023802104F1B800A37516B0BDE8F04742
:101B78000FF0D2B92046FFF75DFFA8EB060300215E
:101B880090FBF3F202FB1300C0B2EC460A46CBB25C
:101B9800434506D21CF801EBBEF1000F2AD1824260
:101BA80026D1434528BF434603FB0951002094F83A
:101BB8000CE001F0FF018446C2B296451CD8BCF186
:101BC800000FCAD116B1FFB9012BC6D9A2191F46F9
:101BD8001176A26852F8211006F10E02013644F877
:101BE800221003F158026A44F6B202F858ACB4E77E
:101BF8000132D2B20131CAE72269125C01308A424D
:101C080008BF4FF0010CD7E77A1E9342DEDB7A1C3F
:101C18009342DBDCA1E7D0E901236421D31AC36036
:101C280082604B43418AB3FBF1F303747047D0E9F8
:101C38000123D31AC0E90223704743682BB1C26855
:101C480064214A43B2FBF3F2D3B203740023C360A6
:101C5800436070470023C0E9023341824360037444
:101C680070474368013343607047007C704743689E
:101C78000B4443607047C068704711B1C3680133B3
:101C8800C3604368013343607047007C704700239A
:101C980003808370037270470346007810B10022F6
:101CA8001A707047587810B100225A7070479878A7
:101CB80010B100229A707047187A08B100221A727F
:101CC800704701707047017070478170704781706C
:101CD8004260704740687047002343600381704743
:101CE8000A2310B50446838001F016FF2368E080BC
:101CF8009B6820469847208110BD038970B504462B
:101D08009BB1858845B1013DADB285806DB9036849
:101D18001B68BDE87040184701F0FEFEE388C01A52
:101D2800238980B2834201D2258170BD2368204671
:101D38005B68EEE72DE9F041044610461D4616465D
:101D48008846FEF7CBFE074606EB0800FEF7C6FE00
:101D580001463846FEF7CEFF656020602846FEF74C
:101D6800C1FEA060BDE8F08110B504464068FEF7EA
:101D7800B9FEA06010BD000010B50229044680EA33
:101D8800E070A0EBE47068D15AB9002CACBF7F2397
:101D98003F239842A8BF1846002C01DA40F04000C3
:101DA80010BD012A1AD1632805DC4000002CF7DA9F
:101DB80040F48070F4E740F2F54398420CDCFEF7FB
:101DC8008DFE5749FEF7E2FE0DF062FFFFF7E0F8DF
:101DD800400040F00100E9E7FF20E7E7022A40F071
:101DE8009C80632805DC8000002CD9DA40F4007060
:101DF800D6E7B0F57A7F0CDAFEF770FE4849FEF7B1
:101E0800C5FE0DF045FFFFF7C3F8800040F0010064
:101E1800EAE742F20F7398420CD8FEF75FFE414999
:101E2800FEF7B4FE0DF034FFFFF7B2F8800040F083
:101E38000200D9E73C4B98420CD8FEF74FFE3B49CD
:101E4800FEF7A4FE0DF024FFFFF7A2F8800040F093
:101E58000300C9E740F2FF10C6E703295DD1012A54
:101E68001BD1B0F57A7F05DA4000002C98DA40F4EF
:101E7800006095E7B0F5205F0CDAFEF72FFE2849E1
:101E8800FEF784FE0DF004FFFFF782F8400040F0F3
:101E98000100EAE740F2FF70E7E7022A3DD1B0F51A
:101EA8007A7F06DA8000002CBFF67AAF40F48050C3
:101EB80076E742F20F7398420CDCFEF70FFE1849E2
:101EC800FEF764FE0DF0E4FEFFF762F8800040F0D4
:101ED8000100E8E7164B98420CD8FEF7FFFD1149C0
:101EE800FEF754FE0DF0D4FEFFF752F8800040F0E4
:101EF8000200D8E7B0F57A2F0CD2FEF7EFFD0B49B8
:101F0800FEF744FE0DF0C4FEFFF742F8800040F0F3
:101F18000300C8E740F6FF70C5E7002040E700BFB0
:101F2800CDCCCC3D0AD7233C17F001006F12833A81
:101F38009F860100002303607047000038B5084BF6
:101F480009291B7828BF09218B4204460D4602D176
:101F58000023036038BD01F0D3FD25712060F9E747
:101F6800C4020020036810B504460BB9002010BD58
:101F780001F0C6FD2368C01A40F2EE239842F5D955
:101F88000023054A2360127823799A42EED0034A47
:101F98000120D377EBE700BFC40200202003002014
:101FA800FF2343710023017183710381837270479A
:101FB80038B5037904460D465BB14179A94208D08A
:101FC80041B101290AD00023A371657155B1012DD2
:101FD8000FD038BD03689B689847F4E70368002171
:101FE800DB68F9E723689B68012120469847A071C0
:101FF800EFE723682946DB68F7E72DE9F04F077C10
:10200800C37B857CC67C90F815E090F8208090F81A
:102018000EC0BF000C4647EA931703F03F01437C0C
:1020280003F0010247EA822705F00F02D20142EAD3
:10203800530206F07F031B0143EA1513057D89B09F
:102048006D0045EAD6150EF00306059345EA4623CA
:10205800867D009306F01F05AD0145EA9E03C57D08
:1020680090F819E00193ED0045EA5613057E0293B6
:102078000EF0070645EA0623857E039305F03F0622
:10208800760146EADE03C67E90F81CE00493B600AB
:1020980046EA95160EF0010546EA8526457F069222
:1020A80005F00F0B4FEACB1B4BEA5E0B90F81EE0D6
:1020B8000EF07F0A4FEA0A1A4AEA151AC57F6D0020
:1020C80045EADE1508F0030E45EA4E2590F821E0B2
:1020D8000EF01F094FEA891949EA9809490190F851
:1020E8002280407B41EADC010CF0070C40EA0C201E
:1020F8004FEAC80848EA5E180791FFF739FA0799C6
:1021080020800846FFF734FA60803846FFF730FA37
:10211800069AA0801046FFF72BFA059BE080184628
:10212800FFF726FA20810098FFF722FA60810198CC
:10213800FFF71EFAA0810298FFF71AFAE0810398C8
:10214800FFF716FA20820498FFF712FA60823046E9
:10215800FFF70EFAA0825846FFF70AFAE0825046C7
:10216800FFF706FA20832846FFF702FA60834846FD
:10217800FFF7FEF9A0834046FFF7FAF94FF48063B2
:10218800E0832384638409B0BDE8F08F2DE9F04132
:1021980004460F4601F0C0FC4FF0010805462368CD
:1021A80020461B689847064650B9A37A012B1FD1D1
:1021B8002389ED1A40F6C4139D42C8BFA07217E0E8
:1021C800236820465B689847A37AA3B90F2814D1DF
:1021D800A4F80A80E37AE2180133DBB2182B1073F3
:1021E800E3720AD939462046FFF707FF0023A37296
:1021F8003046BDE8F081012BECD02581CFE782790C
:1022080022B14379012B01D8FFF7C0BF00207047E6
:10221800704770477047002070477047002070472C
:1022280000207047704700207047002070474FF02B
:10223800B04382B0DA6C0243DA64DB6C034001938A
:10224800019B02B070474FF0B04382B09A6D0243D1
:102258009A659B6D03400193019B02B070474FF054
:10226800B04382B0DA6D0243DA65DB6D0340019357
:10227800019B02B070474FF0B04382B01A6E024320
:102288001A661B6E03400193019B02B0704750E829
:10229800003F43F0200340E80032002AF7D170479E
:1022A80050E8003F43F0800340E80032002AF7D1AD
:1022B800704750E8003F23F0200340E80032002A2E
:1022C800F7D1704750E8003F23F0400340E8003260
:1022D800002AF7D1704750E8003F23F0800340E818
:1022E8000032002AF7D17047704700000288044B7B
:1022F8005140C9B233F8113083EA12230380704782
:10230800043F01089AB110B4B0F800C0084C0A4460
:1023180011F8013B83EA0C03DBB2914234F8133025
:1023280083EA1C2CA0F800C0F2D110BC704770479B
:10233800043F010837B54FF6FF730446ADF8063081
:102348004518AC4203D1BDF8060003B030BD14F8FF
:10235800011B0DF10600FFF7C9FFF2E7044B1888CF
:10236800044B1B8880B29BB2C01A18BF012070476B
:10237800643D0020623D0020044A00231380044A83
:102388001380044A1380044A13807047623D00207A
:10239800643D0020663F0020683F00200120704710
:1023A800044B1888044B1B8880B29BB2C01A18BF14
:1023B800012070476C4100206A41002070470000EE
:1023C8000649074A0B8812880133C3F3080392B2FF
:1023D8009A421EBF034AD0540B8070475C330020DA
:1023E8005A3300205A3100200023A0F87032A0F898
:1023F8006E3270470023A0F85C32A0F85A3270475A
:102408003A4B5A6A037A92B263B18389D31A9BB260
:10241800B3F5FA7F84BF00230372837A4F2B84BFFE
:1024280000230372037A8281082B0FD8DFE803F0B8
:10243800050E0E0E0E0E0F172200EE2901D0C82928
:1024480004D1012383724175062303727047837A8E
:102458005A1C03448272597541720723F5E7827A40
:10246800531C0244DBB283725175427A9A42EDD210
:102478000823EAE7837A5A1C034482725975C37D9C
:10248800162B04D1012380F865300923DDE7436961
:10249800174A03F0FF23934203D1012380F86730E2
:1024A800F3E7144A93421CD1837E102B19D1C37EC3
:1024B800022B08D0052B0DD0012BE6D1027EEE2A87
:1024C80008BF80F86A30037EEE2BDED1012380F846
:1024D8006B30DAE7012380F86830037F80F86930D1
:1024E800D3E7012380F86630CFE700BF00440140FE
:1024F80000C8002800C80032044B1888044B1B8809
:1025080080B29BB2C01A18BF012070475C3300200C
:102518005A3300200278024B51405B5C03707047CD
:10252800842B0108FF230370704700BF7047B0F881
:102538006E32B0F870229B1A98B21B0444BF00F5A3
:10254800006080B2003818BF01207047A0F1140065
:10255800EDE7B0F87022B0F86E12914203461FBF43
:102568008118013291F87402B3F872121ABF0A4046
:10257800A3F8702200207047A0F11400E9E770B5B5
:102588000B7803704B7843700B78FD2B05460C468F
:1025980038D18B788370CB78C3700B7903714B7902
:1025A80043718B7983718B68C3718B68C3F30F2375
:1025B80003728B7A43720A26627804F10C01A81917
:1025C8000EF012FD6378B4F80C213344981CEA54D9
:1025D8005A1CB4F80C1192B2090AA954A278D2076D
:1025E80080B20ED504F58872054404F58E7452F84D
:1025F800041B45F8041BA242F9D112782A700F3344
:1026080098B270BD00238B700B7983704B79C370BF
:102618008B7903718B6843710626CDE738B54A7804
:10262800352A0D46044601F10C010AD80EF0DCFCEF
:1026380068780021C0F136022044BDE838400EF029
:102648006BBC403551F8043B40F8043BA942F9D132
:102658000B88038038BD38B54A781B2A0C460546D6
:1026680001F10C010AD80EF0BFFC60780021C0F11E
:102678001C022844BDE838400EF04EBC283451F8FE
:10268800043B45F8043BA142F9D138BD38B54A7836
:10269800082A0D46044601F10C010AD80EF0A4FCE4
:1026A80068780021C0F109022044BDE838400EF0E6
:1026B80033BCEB6803604B6843600B7A037238BD28
:1026C80038B54A78072A0C46054601F10C010AD8A4
:1026D8000EF08AFC60780021C0F108022844BDE8A9
:1026E80038400EF019BCE36803604B68436038BD9E
:1026F80008B52422034800210EF00EFC024B0022EC
:102708001A7008BDA40C0020740500202DE9F041C2
:102718001378037092F8018080F80180FD2B04463D
:102728000F46154654D193788370D378C3701379C4
:10273800037153794371937983716B7A127A1B040D
:1027480003EB0223EA79134423F07F430A26A268A5
:1027580063F31702A260A919424604F10C000EF0B7
:1027680043FC7A7B904507D208F10C00A2EB0802E3
:10277800002120440EF0D0FB63781E44AB195A7830
:10278800AB5D03EB0223A4F80C31A378DB070ED56D
:10279800023615FA86F304F5887203F10C0153F832
:1027A800040B42F8040B8B42F9D11B781370BB7AE7
:1027B80084F82131FB7A84F822313B7B84F8233179
:1027C8007B7B84F824313B7884F82031BDE8F081A4
:1027D8000023438093780371D3784371137983710D
:1027E80053790626B3E738B54A78132A0C460546C6
:1027F80001F10C010AD80EF0F7FB60780021C0F156
:1028080014022844BDE838400EF086BB203451F845
:10281800043B45F8043BA142F9D138BD2DE9F04FFE
:102828000C465188B1F58C7F054685B04FF0000005
:1028380010D31070D91CC9B2012995BF01210023FA
:10284800518053809CBF237011700020287005B000
:10285800BDE8F08F16780E2E00F2908001A757F889
:1028680026F000BF3D280008A9280008D128000844
:10287800EF2800088529000885290008852900080F
:102888008529000885290008852900088529000868
:1028980085290008852900088529000801290008DC
:1028A800481C508063542178FD299BB206D10C3313
:1028B8000A21D380918002231370C6E708330621CA
:1028C800D38091800E23F7E7481C50806354D807C3
:1028D80042BFD1880D31D1800020012B8CBF034627
:1028E80003231370B2E7481C5080002083426354CE
:1028F80014BF03460E23F4E7481C508063545388E2
:10290800D1888B4232D300235380137002232B705B
:1029180069802378FD2B37D163792B72A3796B7289
:10292800637A227A1B0403EB0223E27913446B6077
:10293800637803F10C026A80A278D10701D51933B4
:102948006B8000266968DFF800816E814FF4BC72E5
:102958000C20B31801335B0800FB03F758F8077025
:10296800B9421AD25A1EB242F3D818E092889A4253
:102978003FF66BAF01232B70002068E71070508082
:102988009080D0802870F7E7E3782B7223796B72F8
:1029980063796B6063780833D2E71E46E3D80C2767
:1029A800774358F80730994227D123782046FD2BE2
:1029B80010F801BF0CBF4FF00A094FF0060909EBE8
:1029C8000B03591E89B247440193FFF7B3FC97F8EC
:1029D80004A0ADF80E0051460DF10E00FFF786FC7D
:1029E800019BE218E35C527803EB0223BDF80E204A
:1029F8009BB29A4209D0052000E0032028700238D3
:102A080001288CBF0020012021E7BB79DA0706D511
:102A1800FA79934582BF04EB09018A5CAA729B0785
:102A280009D50C2303FB068362781B7A9A4282BF7E
:102A38004C44E35CEB720C2303FB068385F80CA083
:102A48005B796B730220DAE7842C01080148436A3A
:102A5800FFF71DBC008000400A4A0B4B12680B4967
:102A6800A3FB02323220920C00FB02F2084B4868AA
:102A780002F5FA72A3FB023292094B681B1A9A42BA
:102A8800FBD870474402002083DE1B43001000E09F
:102A9800D34D621030B587B0034601AC00F1100584
:102AA80018685968224603C20833AB421446F7D166
:102AB8000024094D8DF81440A96801A8FDF758FBBA
:102AC80010B920B207B030BD01342E2C05F10C0529
:102AD800F2D14FF0FF30F5E70800002002780A4BEA
:102AE80090F801C08178D243D2B29A5C82EA0C0293
:102AF80090F803C09A5C4A40995C027981EA0C011B
:102B0800595C4A40985C7047842B0108028810B5CC
:102B18008488531C234044889C421EBF121891711C
:102B2800038010BD411A88B20B0444BF00F5007041
:102B380080B2704770B5104C0025234626782EB118
:102B480066788E4202D1A67896420BD001350C2DBC
:102B580004F10404F2D1002413F824501DB1013407
:102B68000C2CF9D170BD012503F8245003EB840324
:102B7800D87059709A70F5E7790500202DE9F84367
:102B88000B460D795A7A9E7ADF7A204B097A1B5CBC
:102B9800DB07044600D50DB9FFF7CCFF00231C491D
:102BA8001A4898464FF0010E9C4201F8018B25D037
:102BB8002DB90278920702D501F801EC1EE0154AFA
:102BC8004FF0000C92F80090B9F1000F0FD092F876
:102BD800039099450BD1002EEED092F80190B145A3
:102BE80005D1002FE8D092F80290B945E4D00CF155
:102BF800010CBCF10C0F02F10402E3D10133DBB28A
:102C0800042B00F10100CFD1BDE8F883A90500200D
:102C1800750500207905002007B503688DF80710B1
:102C28001B6901220DF10701984703B05DF804FB09
:102C3800F0B50546FD2305F80C3B85B004468DF834
:102C4800043090F8243103F10C020244012B42D8DD
:102C58000026637066808DF805308B7A23718DF8B5
:102C680008308B7AADF8066001338B7263798DF882
:102C78000930A3798DF80A30A368C3F317031A1231
:102C88008DF80B3009211B140DF105008DF80D305E
:102C98008DF80C20FFF74EFB6778ADF802003A4636
:102CA80029460DF10200FFF72DFB94F82311FFF7D9
:102CB8001DFB94F82421BDF80230A4F80C3197428A
:102CC80010D207F10C00D21B3146204405B0BDE8F4
:102CD800F0400EF021B912F8010D0028B8D1013BDF
:102CE800DBB2B3E705B0F0BD7047000008B5FFF7E9
:102CF800B3FE044AD2F8903043F40043C2F890304F
:102D080008BD00BF00040058044AD2F8903023F4EC
:102D18000043C2F89030FFF79FBE00BF0004005880
:102D280070B5044608460D46FDF72CFA236882B2B2
:102D3800294620461B69BDE87040184708B5FFF7CB
:102D4800EFFF08BDB0F1904F02D10120FFF76FBA35
:102D5800084B984205D003F58063984203D10420BC
:102D6800F4E70220F2E7044B984201D18020EDE716
:102D7800704700BF00040048001C00480C4B9842F4
:102D880003D14FF40060FFF776BAB0F1804F05D059
:102D9800084B984205D14FF40030F4E70120FFF7C3
:102DA80052BA054B984202D14FF48020EBE77047A6
:102DB800002C014000440140004801402DE9F04347
:102DC80087B00E46054614460021142201A89DF836
:102DD80038809DF83C901F460EF09EF800960B2C0C
:102DE80007D8DFE804F007070A1214141416161699
:102DF8001A1CFEE70323019301E002230493032F27
:102E080011D8DFE807F0111321110123F6E7012398
:102E1800F1E7012301930393F1E70223EBE7022390
:102E280001930123F7E7FEE702230293B8F1100F9D
:102E38000CD8DFE808F02D2D0C11131517191B1DE0
:102E48001F21232527292B000123EEE7FEE7012375
:102E58000593022301931EE00223F9E70323F7E712
:102E68000423F5E70523F3E70623F1E70723EFE754
:102E78000823EDE70923EBE70A23E9E70B23E7E754
:102E88000C23E5E70D23E3E70E23E1E70F23DFE754
:102E9800B8F1000FDDD1B9F1000F02D02846FFF7D5
:102EA80051FF053C042C05D8DFE804F0030B0403AC
:102EB8000B00AE62694628460BF084FD07B0BDE8FA
:102EC800F083AE61F6E713B54FF0010C0024CDE9AD
:102ED800004CFFF773FF02B010BD000007B50E48A5
:102EE800FFF7E7F9036823F001030360436843F43D
:102EF80000434360036843F0010303600022092391
:102F0800CDE90032054803230A220121FFF756FFC5
:102F180003B05DF804FB00BF0080004000080048D3
:102F280030B587B0002315460446ADF80630FFF7E4
:102F380025FF042D04D8DFE805F02E3204363F00C3
:102F4800FEE71E4B1E4A1B68B3FBF2F39BB200223E
:102F5800CDE90221013B01A92046ADF804300492D5
:102F680005920BF0DFFF236823F080032360A3683A
:102F780023F4A03323F00703A360636823F07003EE
:102F88006360636823F470036360A36823F08003BD
:102F9800A36007B030BD094B0A4A1B68D4E7074B4A
:102FA800094A1B68D0E7054B064A1B68B3FBF2F3D6
:102FB80003EB83035B00C9E70123C8E74402002051
:102FC80080A8120140420F0000127A0010B5044692
:102FD800FFF7A6FF236843F00103236010BD00221A
:102FE8004FF0FF31FFF7F2BF1A4B10B51A4C5B6870
:102FF80023600AF04DFE4FF090400BF0A5FC1748F7
:103008000BF0A2FC16480BF09FFC16480BF0C4FF0F
:1030180015480BF0C1FF0BF08BFE4FF0E0220023A8
:1030280013615361936172B64FF0FF319A0002F158
:10303800604202F561420133082BC2F88010C2F8E1
:103048008011F3D162B6034B1B6883F308882368A9
:103058009847FEE70000FF1F7005002000040048A5
:103068000008004800380140004400400749084A69
:10307800881AEFF30883521A1A44013A013B98421E
:1030880088BF0022AA210DF047BF00BF0000012021
:1030980000040000044B5A69586910F0020018BF78
:1030A800C2F38000704700BF000400584FF0B042E0
:1030B800D2F8943043F40043C2F894304FF47A7352
:1030C80000BF013B9BB2002BFAD14FF0B043D3F8BD
:1030D800942022F40042C3F89420D3F89420520498
:1030E800FBD40C4BD3F8902022F40042C3F8902074
:1030F8004FF47A7200BF013A92B2002AFAD1D3F89B
:10310800902042F40042C3F890204FF400629A6184
:10311800704700BF0004005810B503230522202182
:103128004FF09040FFF7CFFEBDE810400323052283
:1031380010214FF09040FFF7C6BE08B5FFF7AAFF71
:10314800003818BF012008BD08B5FFF7F6FF00B921
:1031580008BD00BFF9E74FF0904310229A62202281
:103168009A6170474FF0904320229A6210229A6128
:1031780070470000024B4FF480225A60704700BF2E
:1031880000E100E00348002303224FF40051FFF759
:103198009ABE00BF00040048034B186980F4005031
:1031A800C0F34030704700BF0004004810B50F4C12
:1031B800002305224FF400414FF09040FFF783FEB3
:1031C8002046002306222021FFF77DFE00231A4611
:1031D80020464FF40041FFF776FEBDE8104000237B
:1031E800052201214FF09040FFF76DBE0004004812
:1031F80005494B691A04DB4302F4001203F020036B
:1032080013438B61704700BF000400480C4BD3F890
:10321800FC2022F08072C3F8FC20D3F8FC2042F096
:103228008072C3F8FC20A3F55D431A6822F00102FE
:103238001A601A6842F001021A6000225A60704748
:1032480000ED00E00649074B074A1B68B3FBF2F3A1
:1032580010B54C6843434A68121B9A42FBD310BD11
:10326800001000E04402002040420F001FB5022376
:10327800CDE9013101A80123694603930AF072FEE2
:1032880000280CBF0420052005B05DF804FB0146AA
:1032980008B501200AF020FE00280CBF04200520F4
:1032A80008BD08B5FFF7E2FF031F5842584108BDA3
:1032B80008B5FFF7ECFF031F5842584108BD00004E
:1032C8002DE9F047294B2A4D01280E461446294975
:1032D800294A0FBF79277827AA461D4606BF884680
:1032E8009A4690460AF0ACFD39462846FFF7D9FFC2
:1032F80028B900240AF0B6FD2046BDE8F087002E64
:1033080008BF4FF4FC64073424F0070405F11007E4
:10331800B1463444AAEB050AA1450BD14FF011324E
:103328004FF0FF332846FFF7C3FF041E18BF0124E0
:10333800A400DFE76EB90AEB0703D3E90023B3F172
:10334800FF3F08BFB2F1FF3F06D1083709F108096E
:10335800E2E7D9E90023F2E7B84505D93846FFF78F
:10336800A7FF0028F1D1C4E70324C3E700C003087E
:1033780000C80308FFCF0308FFC7030810B50AF009
:103388005FFD09487821FFF78CFF044638B10748EC
:103398007921FFF786FF041E18BF0124A4000AF054
:1033A80061FD204610BD00BF00C0030800C8030827
:1033B80030B5084D002340F2EF749AB2914201D81B
:1033C800042030BDA34203D05A5DC2540133F4E750
:1033D8000320F6E710C0030838B504460D4672B658
:1033E8000A4601460020FFF76BFF62B6042806D1A3
:1033F80072B601202A462146FFF762FF62B638BD41
:1034080038B5124B1C68D3F80058B4F1113F09D1F4
:10341800B5F1113F17D0002211460120BDE8384010
:10342800FFF74EBFB5F1113F03D1002211461046F8
:10343800F4E7FFF7A3FF042804D12C4001340CBFA4
:103448000220012038BD0420FCE700BF00C00308AB
:10345800044B9A689107FCD518739A68D207FCD573
:10346800187B70470000015870B50C46451E8E1831
:10347800B44200D170BD15F8010FFFF7E9FF04F859
:10348800010BF5E7084611461A46FFF7EDBF0000A5
:1034980070B5064E04464518A54200D170BD307877
:1034A800FFF7D6FF04F8010BF6E700BF380200204B
:1034B80008461146FFF7ECBF38B504464518AC423C
:1034C80000D138BD14F8010BFFF7C2FFF7E7084633
:1034D8001146FFF7F1BF000010B58CB0282200217B
:1034E80002A80DF019FD4FF0B0431C4C5A6E42F083
:1034F80001025A665B6E03F001030193019BFFF71B
:10350800D5FD082208924FF48272002303924FF4EB
:103518000072CDE90533CDE90933029307920723F9
:103528004FF4E06202A920460B9304920BF0C0FC12
:10353800636823F010036360636823F00803636023
:10354800236843F040032360A3689B07FCD5237BD3
:10355800034BFF221A700CB010BD00BF00000158C9
:10356800380200201B4B10B4DC69A00611D51A687C
:1035780091060ED5184819495A6A038809880133F3
:10358800C3F30A0389B299421FBF1549D2B2CA547C
:10359800038010481F232206036215D503681B0603
:1035A80012D5104B104A1988138889B29BB29942D8
:1035B8000CD013880133C3F30803138013880B4A14
:1035C8009BB2D35CDBB2836210BC704710BCFEF7C1
:1035D80082BE00BF00440040643D0020623D0020E0
:1035E80062350020683F0020663F0020663D0020CD
:1035F8000A490B4A08B50B8812880133C3F308033C
:1036080092B29A4207D0074AD05407480B80FEF777
:1036180047FE012008BD0020FCE700BF683F0020EE
:10362800663F0020663D00200044004038B504464F
:103638004518AC4200D138BD14F8010BFFF7D8FF8C
:10364800F7E708461146FFF7F1BF0000054B064AA9
:103658001B8810880133C3F3080380B2181A18BFF7
:1036680001207047683F0020663F002008B5FFF73B
:10367800EDFFB0FA80F0400908BD0000054B064A8E
:103688001B8812889B1A98B21B0444BF00F500607F
:1036980080B27047643D0020623D0020FFF7EEBF16
:1036A8000848094A0188138889B29BB29942F9D01F
:1036B80013880133C3F30A0313801388034A9BB2A8
:1036C800D05C7047643D0020623D002062350020D8
:1036D800FFF7E6BF70B588B00C46064615460021D0
:1036E800202268460DF018FC231E18BF01231B0377
:1036F800CDE9023569460C230348019604940593E5
:103708000BF06EFC08B070BD0044004010B5064CCC
:10371800236823F001032360FFF7DCFF236843F0ED
:103728000103236010BD00BF00440040002208468A
:103738001146FFF7EBBF000073B5314C236823F047
:1037480001030825236001264FF40030FEF77BFDB6
:103758000421CDE9005603230A224FF09040FFF7D9
:103768002DFB03231A462946CDE900564FF0904019
:10377800FFF724FB002211464FF4E130FFF7AAFFC0
:10378800636823F490436360A36823F02A03A3606B
:103798001C4BB02283F8252320225A602046FEF7CE
:1037A8009AFDFEF78FFD40232362174B00211980F5
:1037B800164B1980FEF77DFD154B1980154B1980A6
:1037C800636823F400636360A36823F00803A360BD
:1037D800636823F480436360A36823F02203A36033
:1037E800A36843F48053A360236833432360E369E9
:1037F8009A02FCD5E3695B02F9D502B070BD00BF3F
:103808000044004000E100E0663F0020683F0020DF
:10381800623D0020643D002008B5FFF78DFF034896
:10382800436ABDE80840FEF732BD00BF00440040CF
:10383800FFF7F2BF1B4B10B4DC69A00611D51A685C
:1038480091060ED5184819495A6A03880988013320
:10385800C3F3080389B299421FBF1549D2B2CA54AB
:10386800038010481F232206036215D503681B0630
:1038780012D5104B104A1988138889B29BB2994205
:103888000CD013880133C3F30A03138013880B4A3F
:103898009BB2D35CDBB2836210BC704710BCFEF7EE
:1038A8001ABD00BF003801406C4100206A41002069
:1038B8006A3F0020704900206E4900206E410020B8
:1038C8000A490B4A08B50B8812880133C3F30A0367
:1038D80092B29A4207D0074AD05407480B80FEF7A5
:1038E800DFFC012008BD0020FCE700BF7049002074
:1038F8006E4900206E4100200038014038B504466A
:103908004518AC4200D138BD14F8010BFFF7D8FFB9
:10391800F7E708461146FFF7F1BF0000054B064AD6
:103928001B8810880133C3F30A0380B2181A18BF22
:1039380001207047704900206E49002008B5FFF744
:10394800EDFFB0FA80F0400908BD00000848094AB8
:103958000188138889B29BB29942F9D01388013340
:10396800C3F3080313801388034A9BB2D05C7047E3
:103978006C4100206A4100206A3F0020FFF7E6BF43
:1039880070B588B00C4606461546002120226846C8
:103998000DF0C2FA231E18BF01231B03CDE902351F
:1039A80069460C2303480196049405930BF018FB11
:1039B80008B070BD0038014073B5304C236823F05F
:1039C80001032360082501264FF48040FEF753FCCD
:1039D8004021CDE900562A4803230A22FFF7EEF9D1
:1039E80003231A46CDE9005625488021FFF7E6F95A
:1039F800002211464FF4E130FFF7C2FF636823F459
:103A080090436360A36823F02A03A3601D4BB02290
:103A180083F8242310225A602046FEF75CFCFEF748
:103A280051FC40232362184B00211980174B198041
:103A3800FEF73FFC164B1980164B1980636823F478
:103A480000636360A36823F00803A360636823F43A
:103A580080436360A36823F02203A360A36843F450
:103A68008053A360236833432360E3699A02FCD53B
:103A7800E3695B02F9D502B070BD00BF00380140B0
:103A88000004004800E100E06E4900207049002071
:103A98006A4100206C41002008B5FFF78DFF0348FC
:103AA800436ABDE80840FEF7F2BB00BF003801409A
:103AB800FFF7F2BF024B1A68024B1A60704700BF4B
:103AC80080490020900A0020054A064B19681368AF
:103AD80099421DBF0133012013600020704700BFC9
:103AE800900A002080490020034A044B11681B7883
:103AF8000B441360704700BF804900204802002033
:103B0800014B1868704700BF804900200148FFF743
:103B180066BA00BF00440140014B586A80B2704742
:103B28000044014008B5FFF7F1FFBDE80840FFF782
:103B3800C1BF0000F8B51A4C1A4F90220021201D71
:103B48000DF0EAF91623062663800F23A380324678
:103B58002C233946A0192680FDF7A6FE124A134BDE
:103B68000025C4E90D2339462C23324604F13E00D2
:103B7800A587FDF799FE0223E3660D4984F8725084
:103B8800012304F17C00A4F87030C4E91D550DF040
:103B980023FA7F2384F89130052384F89230F8BD06
:103BA800DC0400206024010802000F000300050067
:103BB8000412010870B5094E05460C46415C3046B2
:103BC8000DF0C1F9034628B1831B0133DBB2282B62
:103BD80028BF0023F35C2B5570BD00BF582B01088C
:103BE80070B50C46114606460DF0F6F944B10025AD
:103BF800052130460135FFF7DDFFEBB29C42F7D8CF
:103C080070BD0000F7B5054605F11106214C224AA2
:103C1800014636016846FFF7E3FFB01C69462044B9
:103C28000DF0DAF9264404EB051200230227777217
:103C3800A2F81A31142202FB05400421012280F85F
:103C480050104FF4807540F20111A0F84A70C26418
:103C5800A0F8522080F85520A0F85650A0F8581027
:103C680040F2032084F83430E784A562A08584F804
:103C78002E2084F8302084F83330C4F83A30C4F861
:103C88003E30C4F84230A4F84610A4F8481003B0F7
:103C9800F0BD00BF20030020C4110108F7B5054698
:103CA800AF4CB04A05F11106014637016846FFF7E7
:103CB80097FFB81C274469462044FDF7F1FC7B7A3E
:103CC800A94A052B88BF022304EB061088BF7B7224
:103CD8001188437A41FA03F3DF070FD402234372B2
:103CE80061B14807C1F3800308D441FA03F7FF071D
:103CF800D8B240F1D18104EB0613587204EB0511D8
:103D08002B0191F81A01052802D9002081F81A011F
:103D1800E718508897F81A1140FA01F1C90711D429
:103D2800012187F81A1168B18707C0F3400109D447
:103D380040FA01FC1CF0010FCFB200F0B281E1188B
:103D480081F81A71E11891F81B01032802D90020A3
:103D580081F81B0104EB0616717A012903D904299D
:103D680001D000219180E618908896F81B1140FA3E
:103D780001F111F001010ED186F81B1158B110F0B4
:103D8800010108D140FA01F7FF07CEB240F18E8158
:103D9800234483F81B61142303FB054191F84A006F
:103DA800052802D9022081F84A0003FB054393F84D
:103DB8004B10042902D9002183F84B10142303FB6C
:103DC8000543918E93F84B0041FA00F0C00712D4D6
:103DD800012083F84B0071B18807C1F340030AD46E
:103DE80041FA03F6F707D8B240F16581142303FBC3
:103DF800054383F84B00142303FB054393F84C1049
:103E0800032902D9012183F84C10142000FB054036
:103E1800D18E90F84C3041FA03F313F0010310D11E
:103E280080F84C3069B111F001030AD141FA03F668
:103E3800F607D8B240F14481142303FB054383F805
:103E48004C00142303FB054393F84E10012902D9B3
:103E5800002183F84E10142000FB0540118F90F8C4
:103E68004E3041FA03F313F0010310D180F84E30BD
:103E780069B111F001030AD141FA03F6F707D8B284
:103E880040F12381142303FB054383F84E001423D8
:103E980003FB054393F84F10022902D9002183F848
:103EA8004F10142000FB0540518F90F84F3041FA15
:103EB80003F313F0010310D180F84F3069B111F00A
:103EC80001030AD141FA03F6F607D8B240F102819C
:103ED800142303FB054383F84F00142303FB054118
:103EE80091F84D00022802D9002081F84D0003FB0B
:103EF800054393F85010052902D9042183F850107E
:103F0800142303FB054191F85200012802D901202E
:103F180081F8520003FB054393F85510012902D993
:103F2800012183F85510142303FB054393F853101C
:103F3800022902D9002183F85310142000FB054000
:103F4800918F90F8533041FA03F313F0010318D11D
:103F580080F85330A9B111F0010312D106E000BF77
:103F680020030020C4110108DC04002041FA03F6F4
:103F7800F707D8B240F1B380142303FB054383F855
:103F88005300142303FB054191F856000C2802D96D
:103F9800002081F8560003FB054393F84C100129D3
:103FA80006D193F84F10022904BF002183F84F105F
:103FB800142303FB0543012183F8571040F2011134
:103FC800A3F8581094F82630052B02D9022384F858
:103FD800263094F82730042B02D9002384F82730A0
:103FE800B2F86C0094F8273040FA03F313F0010F8D
:103FF800804B0ED1012184F8271050B18607C0F3F9
:10400800400106D440FA01F7FF07CEB26CD583F819
:10401800276094F82810022902D9002184F8281072
:1040280094F82910022902D9012184F82910B2F83C
:104038006E1094F8292041FA02F212F001020CD114
:1040480084F8292049B111F0010206D141FA02F69B
:10405800F607D0B24CD583F8290094F82A200C2A08
:1040680002D9002284F82A2093F832200C2A02D997
:10407800002283F8322093F82B20042A02D9002248
:1040880083F82B2000225C49104611F9014F14F1E6
:10409800780F31DA087031E00133102B7FF425AE48
:1040A8002CE6013110297FF443AE4BE6013110298B
:1040B8007FF468AE6FE60133102B7FF491AE9AE679
:1040C8000133102B7FF4B2AEBBE60133102B7FF423
:1040D800D3AEDCE60133102B7FF4F4AEFDE60133FA
:1040E800102B7FF443AF4CE7013110298AD190E7B8
:1040F8000132102AAAD1B0E7782CCBDC0132D2B237
:104108000C2AC2D13D490022012011F8014F013289
:10411800022CD2B288BF0870042AF6D193F8342052
:10412800012A02D9002283F83420354AB2F87010E7
:1041380093F8342041FA02F212F001020CD183F80C
:10414800342049B111F0010206D141FA02F4E40722
:10415800D0B211D583F8340093F82C20052A02D95F
:10416800032283F82C2093F82D20032A08D80AD19B
:10417800002283F8342006E00132102AE5D1EBE76B
:10418800022283F82D2093F82E20022A02D9012238
:1041980083F82E2093F83020022A02D9012283F8CE
:1041A800302093F833200C2A02D9002283F83320D8
:1041B800142101FB0531FF2203EB05154FF6FF70B3
:1041C80081F8512081F8542083F82F2083F831207A
:1041D8004FF0FF32C5F81C21A5F820011A629A8415
:1041E800A1F85A20A1F85C2083F83500DA861A87EE
:1041F80003B0F0BD20030020590300206503002010
:10420800DC04002030B5052804D8DFE800F01E04DF
:1042180023191E23FEE720251F2400220F21104BFF
:1042280098700338012894BF002001201A7119776B
:104238001A74A3F84850A3F84A409873987630BD8A
:1042480009256F2400220721E9E7142532240022DA
:104258000A21E4E73525132401221921DFE700BFED
:10426800C40200202DE9F74300F11105944F954C45
:104278002D0105F10209B94406464846FDF72CFA16
:104288003D440421804601900DEB0100FEF752F8F1
:104298006B7A637007EB0613E083C4F8088093F821
:1042A8001A01C4F814804FF0010884F85180A4F86A
:1042B8005280A4F85480FFF7A5FF142303FB06736C
:1042C800350193F84A20804B13F922302373237663
:1042D8006378052B09D8DFE803F0030656585A5CC3
:1042E8000023637301E084F80D80784B617B1B88A1
:1042F800617603F00102980748BF42F00202A285E6
:104308005A0748BFA28D84F8281044BF42F004021F
:10431800A285180742BFA28D42F01002A285DA06D4
:1043280042BFA28D42F02002A285980642BFA38D0B
:1043380043F00803A385002384F82A3021B94846AE
:10434800FDF7EAF984F82A003D4495F81B2184F822
:1043580029206AB1E18B02EB021303EB03230B4420
:10436800E383A3684FF0113101FB0233A36063615B
:1043780094F82850E38B6362052D0CD8DFE805F02C
:104388000C51531547490223ABE70423A9E705233A
:10439800A7E70323A5E7FEE7A378032B03D8DFE805
:1043A80003F003464403FEE71825DFF824C184F828
:1043B80020501CE90F008CE80F0040F2E243284629
:1043C800A4F84C30FCF78EFB4FF07F51FCF7DEFB76
:1043D800FCF7DEFDB4F848204FF47A73B3FBF2F330
:1043E800A4F84030142303FB06736D08052D93F8D9
:1043F8005030C0B238BF0525A4F84E0084F850509C
:10440800052B3DD8DFE803F0154236393C3F02253D
:10441800CBE7A378022B08D0052B06D0012B06D0BA
:10442800FEE71925C1E70625BFE70C25BDE71225DC
:10443800BBE74FF416536364002384F8563084F8BE
:104448005830142303FB067696F84C20032A03D031
:1044580096F84F30022B02D1012384F85630511EB2
:104468004B424B4194F8561084F8573089B1012AD1
:104478000FD1FEE74FF41643DDE74FF46143DAE767
:104488004FF4E133D7E74FF46133D4E74FF4964361
:10449800D1E72378142000FB037393F84C30022BE8
:1044A80007D1012384F8583021B194F858301BB152
:1044B800FEE709B9012AF8D003B0BDE8F08300BFD0
:1044C80020030020C402002060240108DC0400202E
:1044D800F402002002484FF4DE72FF210CF01CBDEC
:1044E8002003002002484FF4DE71FEF775BF00BFBD
:1044F8002003002002484FF4DE71FEF759BF00BFC9
:104508002003002008B5FFF7F5FF034B1878BDE836
:104518000840FFF7C3BB00BFC402002038B5FFF74F
:10452800D9FFFEF76DFF04280CD0FFF7D3FFFEF785
:1045380067FF042803D1FFF7DDFF042806D0FFF743
:10454800C9FF03E0FFF7D6FF0428EED12F49304812
:104558002F4C10220CF004FD38B12E4910222046B1
:104568000CF0FEFC08B1FFF7B5FFA38AB3F5215F95
:1045780028D008D30025E8B20135FFF743FB0A2D00
:10458800F9D10023E3774FF42153A382012522694F
:104598001E491F4842F642039A424FF010021CBFC0
:1045A800236101250CF0DCFC70B118491848102271
:1045B800FDF7F8F9184919480822FDF7F3F9FFF74C
:1045C80091FF03E00025E2E7002DF8D1E37F104AD0
:1045D800092B84BF0023E377E17F1420002300FB2D
:1045E8000144013394F84C0082F84C000A2B02F184
:1045F8001402F6D10A4C2170FFF79CFA2078FFF7D5
:104608004DFB2078BDE83840FFF72CBECB110108E0
:1046180020030020DC110108ED110108D20400205C
:10462800C402002030B5C01A1628A8BF16206FF0A3
:104638000805A8429DF80C40B8BF2846A042C8BF4C
:1046480020B2C0B208701844107030BD07B50846D3
:1046580011461A46162300930023FFF7E3FF03B021
:104668005DF804FB0129F7B5054600D9FEE70B4EB6
:1046780006EB01131C460F016278F15D03619B781C
:104688000AF0C0FFE3790193A37900932279637953
:10469800E17828460AF0DDFF03B0F0BD24410108A7
:1046A80038B5836804466BB1024652F8183BDD6999
:1046B80000F11903A847217E20460222BDE83840B0
:1046C8000BF029B838BD000070B58160897A86B0D2
:1046D800044601B101210AF06EFF20460BF0FDF8F7
:1046E80020460BF0D5F8217BFF2903D0FA2220467B
:1046F8000BF0DAF8A3685B7A013B042B04D8DFE8F7
:1047080003F0043E3E414100FEE7E922E121204654
:104718000BF008F9012120460BF097F89621204666
:104728000BF0D4F8382120460BF0E6F820460BF0C1
:10473800EBF8A368204693F90810FFF7B1FFA368C8
:104748009D7A15B319782046FFF78CFF0022114691
:1047580020460AF04AFF0023009340F20322204635
:104768004FF6FF710AF0A4FF20464FF6FF710AF0DA
:10477800C6FF204606B0BDE870400BF076B8DB22D5
:10478800D721C4E76F226B21C1E70F4B0F49DE8B9E
:104798000F4B63614CF250330093204619230B22D0
:1047A8000BF0CEF80123CDE903335B23CDE90153A8
:1047B800102319462046009504220BF0FFF83146D5
:1047C80020460BF01FF9C1E7C4020020A0860100B3
:1047D8000441010810B504460BF047F820464FF68F
:1047E800FF71BDE810400AF08ABF000038B5816843
:1047F800036891F90810DD69044600F1190300F116
:104808001802A847A3689A7A42B11A78012A00D9EF
:10481800FEE7044B03EB0213236138BD024B6361CF
:10482800FBE700BF244101080441010810B50A4C08
:10483800A06858B1236923B9636913B92046FFF703
:10484800D5FFA3689B7A23B123699868A0F57A708D
:1048580010BD63699869F9E75C300020836810B57A
:10486800044683B103691BB943690BB9FFF7BEFF5F
:10487800A3689B7A1BB12369B3F90C0010BD636967
:10488800B3F91C00FAE71846F8E7836810B5044640
:1048980043B103691BB943690BB9FFF7A7FF94F943
:1048A800190010BD1846FCE790F8D8305BB190F8B5
:1048B800D930074A180102EB03139B68197813587B
:1048C80053F821007047837D0E3350F8230070475A
:1048D800002401082DE9F3419DF824701646402F65
:1048E80088464FF05B024FF0000104461D4628BF82
:1048F80040270CF011FB904BDB8B23803278A37898
:1049080062F30203A3707178C90001F00801DBB2F9
:1049180003F0070341EA08111943A1707279E3789B
:1049280062F30003E370B279637962F3861363710B
:1049380096F90200FCF7E1FDE37860F34703E370C2
:10494800F279237962F300032371327A62F3460322
:1049580023713279DBB202F0010203F07F0343EAEC
:10496800C213237132796379C2F3450223F03F03FE
:1049780013436371A37967F34703A3712B78AA786C
:10498800E3716B7802F01F0203F0070343EAC203E6
:1049980023726A88637AC2F3451223F03F031343F4
:1049A80063722A79DBB202F0030203F03F0343EAA1
:1049B80082136372AB88C3F38703A3726A79E37ABD
:1049C800C2F3800223F001031343E372AA79DBB236
:1049D80002F07F0203F0010343EA4203E372EA882C
:1049E800237BC2F3C31223F00F03134323732B7AE1
:1049F800AA7AE3736B7A02F01F0203F0070343EA13
:104A0800C20323746A89637CC2F3451223F03F030F
:104A1800134363742A7BDBB202F0030203F03F0303
:104A280043EA82136374AB89C3F38703A3746A7B75
:104A3800E37CC2F3800223F001031343E374AA7BEF
:104A4800DBB202F07F0203F0010343EA4203E3749E
:104A5800EA89237DC2F3C31223F00F03134323759E
:104A68002B8ADB0863756B8ADB08A375AB8ADB08C6
:104A7800E375EB8ADB0823762B8BB3F5C06F4ED238
:104A8800B3F5007F94BF00230123227B63F3051253
:104A980022736B8BB3F5C06F43D2B3F5007F94BF1D
:104AA80000230123227B63F387122273AB8BB3F5B8
:104AB800C06F38D2B3F5007F94BF00230123227D55
:104AC80063F305122275EB8BB3F5C06F2DD2B3F5E6
:104AD800007F94BF00230123227D63F38712089B84
:104AE80022751F4404F11802BB4220D14FF6FF7310
:104AF80021460DF106000D22ADF80630FDF702FC47
:104B08002146BDF8063021F80D3F4C22FDF7FAFB8F
:104B1800BDF80630A4F8593002B0BDE8F081022390
:104B2800B3E70223BEE70223C9E70223D4E713F859
:104B3800011B02F8011FD7E7C402002013B59DF836
:104B48001040CDE9003413460A460021FFF7C2FEA3
:104B580002B010BD13B5144B0288DB8B9A42044691
:104B68001DD1837803F0F003102B01D0202B18D12E
:104B7800A379A52B15D84FF6FF730DF1060059221E
:104B88002146ADF80630FDF7BDFBB4F85900BDF875
:104B98000630C01A18BF0120800002B010BD0120E5
:104BA800FBE70220F9E700BFC402002030B5374B0D
:104BB800027893F8261061F30302027093F8271025
:104BC80061F30712027093F82810427861F3030228
:104BD800427093F8291061F30712427093F82A1073
:104BE800827861F30302827093F83210827961F35C
:104BF8000302827193F82B10827861F30712827096
:104C080093F83410C27961F30302C27193F82C103F
:104C1800C27861F30302C27093F82D1061F3071292
:104C2800C27093F82E10027961F30302027142797F
:104C380093F8301061F30302427193F833108279CC
:104C480061F30712827103F1390100F10A0200F1E0
:104C5800160411F9015F02F8015FA242F9D193F835
:104C68004610C27D61F30102C27593F8471061F3E3
:104C78008302C27593F8481061F30512C27593F860
:104C8800493063F38712C27530BD00BF200300208E
:104C98000278314BC2F3030230B583F8262002783C
:104CA800C2F3031283F827204278C2F3030283F881
:104CB80028204278C2F3031283F829208278C2F3AD
:104CC800030283F82A208279C2F3030283F8322090
:104CD8008278C2F3031283F82B20C279C2F303024D
:104CE80083F83420C278C2F3030283F82C20C278F8
:104CF800C2F3031283F82D200279C2F3030283F86A
:104D08002E204279C2F3030283F830208279C2F35D
:104D1800031283F8332003F1390100F10A0200F18C
:104D2800160412F9015F01F8015FA242F9D1C27DB0
:104D3800C2F3010283F84620C27DC2F3810283F8E0
:104D48004720C27DC2F3011283F84820C27DC2F316
:104D5800811283F8492030BD200300201FB58DF84B
:104D68000C300123019303AB009313460A4602213A
:104D7800FFF7B0FD05B05DF804FB0000F0B5224D6B
:104D8800012385F87230044685B0B0F80900FCF7B5
:104D9800B0FD6867B4F80B00FCF7ABFD1422A867F8
:104DA80004F10D0105F17C00FCF70EFE94F92130A9
:104DB80085F8913094F8223085F8923004F1230078
:104DC800FFF766FF6E4604F1410304F151071868C6
:104DD8005968324603C20833BB421646F7D10B481E
:104DE8002C2308226946FCF7E1FC94F85130A5F819
:104DF8006C3094F85230A5F86E3094F85330A5F81A
:104E0800703005B0F0BD00BFDC0400201A0500209A
:104E18002DE9F04792B0DFF890A0244C0DF1080876
:104E28004FF0400905460E46174600214A464046BF
:104E38000CF072F89AF8001004EB011122230DF11E
:104E48000A00062201F589718DF80830FCF7AAFDE1
:104E58009AF8001004EB011205A892F81A3192F89A
:104E6800194103F00F0304F00F0444EA031492F805
:104E78001B3103F00F0344EA0324BDF8103023F478
:104E88007F6323F00F031C43ADF81040FFF78EFE3D
:104E9800CDE900893B46324602212846FFF71AFD34
:104EA80012B0BDE8F08700BFC40200202003002034
:104EB800034B04491A68044801FB02001860704754
:104EC800B00500200D6619005FF36E3C38B50A4A3C
:104ED8000A4D13782C78A34203D101332B7028781C
:104EE80038BD1470FFF7E4FF6FF0004398423CBFF1
:104EF80001342C70F3E700BFAD050020AE0500209B
:104F08000A4A126882600A4A002383808371838177
:104F18000384136803615368064A43611368836115
:104F28005368C3614EF660230360704780490020D0
:104F3800F3110108FC11010810B5124C0220FFF70B
:104F480061F92046FFF746FC6FF07F012046FFF726
:104F5800A7FBA36803B9FEE7002120460AF014FB6B
:104F68004FF47A70FEF76EF9204601210AF023FB10
:104F7800A36820461978FFF775FB2046FFF72AFC3F
:104F880010BD00BF5C30002008B590F82030024604
:104F98008BB9FEF701F910B982F8210008BD92F823
:104FA800213001335BB2312B82F82130F6DD012349
:104FB80082F82030F2E7FEF7EFF818B1322382F8D2
:104FC8002130EBE792F82130013B5BB2002B82F8ED
:104FD8002130D8BF82F82000E0E70000134B90F89A
:104FE80020201B68CAB182689B1AB3F57A6F01D971
:104FF800012343710379ABB10D4B427B1B781AB186
:10500800022B1CBF032202739A1E5342534143735F
:10501800837953B10323037370478360EAE701235D
:105028000371F8E74379002BF9D1704780490020D4
:10503800850600200346007B821E012A4FF00002ED
:1050480002D893F8201009B91A73704710467047B0
:1050580070B51B4C1B4E05465B22002120460BF009
:105068005BFF2B6923606B696360174B174D1B78D7
:1050780031789A1E53425341627A05EB011163F36A
:105088000002627201F58971062204F10A00FCF738
:1050980089FC337805EB0315237C95F81A2162F314
:1050A8000713237495F81B21637C592162F30303CA
:1050B80020466374FDF73EF9A4F8590070BD00BF9F
:1050C800A1300020C4020020850600202003002013
:1050D8000A4A38B5138801339BB2502B04460D4653
:1050E80001D8138038BD002305491380FDF718FE49
:1050F80029462046FDF714FEF4E700BF940A002075
:1051080024130108154680B50C490D4E0446FDF7D9
:1051180007FE29462046FDF703FE0A4B00221A80A7
:10512800202746F2A810B762FEF78CF8B761FEF7A1
:1051380089F829462046FFF7CBFFF2E72413010838
:1051480000040048940A002037B50C461D4668B98B
:1051580007480DF106020DF107010AF035FB9DF82D
:10516800061003482B4622460AF0DFF903B030BD8B
:105178005C30002070B50D4616461C460146A0B9A5
:10518800FDF7E9FF0B4833462A460AF0A7F9094814
:105198004FF6FF710AF0B3FA0648A1010AF0C8FAFF
:1051A800BDE870407D20FEF74DB80248FFF712FBBE
:1051B80070BD00BF5C30002037B50C4638B91A48BE
:1051C800836833B9812281F88C2081F88E3003B04E
:1051D80030BD9D7ADDB101F18E020DF106010AF0B4
:1051E800DDFA94F98E30002B04DABDF8062013445A
:1051F800ADF80630BDF90630002B0FDB4FF6FF7314
:10520800ADF80630BDF8063084F88C30DFE70DF1D4
:1052180006010AF008FC84F88E50EBE77F33F1DAD8
:105228004FF68173ECE700BF5C30002070B5114C7D
:105238000D4606465B23224621462846FFF784FF93
:10524800D6E90613206862689A4208BF88420ED1E0
:1052580020465921FDF76EF8B4F85940231A5C42EC
:105268005C4128460449FFF7A7FF601C70BD002475
:10527800F7E700BFA22E0020B42F00200A4608B589
:1052880001460148FFF73EFF040000200023037099
:105298008370437003714371C370704703780022B1
:1052A800022B427104D0032B09D0012B16D0FEE744
:1052B80001230371437183784370C3707047837807
:1052C8004278991AA3EB020218BF012112F0060FC7
:1052D80014BF0122002201714271EDE7027170478B
:1052E80002788170002A0CBF022203220270FFF7A5
:1052F800D5BF000008B5437802789A4213D0052B31
:105308008ABF052303700370027888BF4370064B79
:10531800064813F92210064B19731976836813B1DE
:105328001972FFF7BDF908BD602401085C30002040
:10533800C402002010B50AB9437010BD541E0B2CCE
:10534800FBD80332D2B231F8122040F27E618A4291
:1053580003D95AB222EAE2721AE0B2F5C17F02D248
:105368009A1E52B2F6E740F2A9518A4204D95AB2BB
:10537800052A1CDCDA1EF4E740F256218A4218D9C5
:1053880040F2D4418A4208D95AB2042AF2DD0222F4
:105398009A42C8BF5AB24270CFE7B2F54B7F04D2E7
:1053A8005AB2032AE6DD0122F2E75A1ED9E70322A0
:1053B800EEE70022ECE70000074B282202FB00334F
:1053C8009B681A78542A05D15878A0F17803584276
:1053D800584170470020704778240108074B28225D
:1053E80002FB00339B681A78522A05D15878A0F13D
:1053F80078035842584170470020704778240108C4
:10540800074B282202FB00339B681A78542A04D1E0
:105418005878783818BF012070470120704700BFBE
:105428007824010828230B4A434310B5D158044671
:10543800FFF7D4FF48B92046FFF7BEFF064B1B789D
:1054480028B103EB830301EB8301084610BD01EB90
:105458000311FAE778240108C40200202B2838B584
:1054680005461AD80E4B282202FB00334CB21B7992
:10547800022B0DD0FE2B10D1FFF7D4FF0378E4B236
:10548800A3420AD004702846BDE83840FFF7B8BFE9
:10549800FFF7C8FF90F90030F2E7002038BD00BFE1
:1054A800782401082B2838B504460D4619D80E4B28
:1054B800282202FB00331B79FF2B12D1FFF7B2FF22
:1054C80006222946FCF793FA58B92046FFF7AAFFA7
:1054D80029460622FCF778FA2046BDE83840FFF74F
:1054E8008FBF002038BD00BF782401082DE9F043A4
:1054F800074615462820394A41435018012B046AAB
:1055080087B025D15258364B9A4235D0A3F1CE01F7
:105518008A4233D03349F23B9A4208BF0C46FF23F4
:105528008DF800304FF0000801262046FAF72AFED1
:105538005FFA88F9484529D806F118036B44AE424A
:1055480003F8188C30D80020387007B0BDE8F08315
:10555800022BE4D15258224B9A4211D0591C8A424C
:1055680010D0A3F1CE018A420ED0A3F1F2018A42F3
:105578000AD01D49EC3BCFE71C4CD0E7194CCEE7CD
:105588001B4CCCE71B4CCAE71B4CC8E714F8093086
:105598002C2B06D106F118036B44013603F8188C3E
:1055A800F6B208F10108C0E705F118030DEB030591
:1055B800002315F8182C15F9175C0132D2B2991886
:1055C800C9B2A94207EB030003DB002303700120E3
:1055D800BBE7615C01700133DBB2F0E778240108B6
:1055E8003904002005120108391201085612010871
:1055F800DB120108B91201088F120108054B282295
:1056080002FB00335B6A0BB1188870474FF6FF70D6
:10561800704700BF782401080B4B282202FB003397
:1056280070B51E6A3046FAF7ADFD002201461446F1
:10563800D5B2631CA942D8B200D870BD735D0132DF
:105648002C2B08BF0446F3E7782401080F4B2822C7
:1056580002FB003310B51B79FE2B014614D1FFF76E
:10566800CDFF04460846FFF7D7FF00220146104643
:10567800D3B2994200D810BD44FA02F3DB0744BF05
:10568800431CD8B20132F3E7FF20F4E7782401087D
:105698002DE9F04F4FF0000A1D4E93B004460F4617
:1056A800D146D6F808805FFA8AF54FF0000B0DE076
:1056B80018F8030001920BF00BFCC3B2019A202BDF
:1056C80008BF5F2302F8403C0BF1010B5FFA8BF334
:1056D80040460193FAF756FD019B03F148029842B0
:1056E8006A44E5D802F8409C394602A8FAF740FD1A
:1056F80048B10AF1010ABAF12C0F06F12806D0D1F7
:105708000025284600E00120257013B0BDE8F08F81
:10571800782401082DE9F0411D4E282303FB01667A
:1057280004463379FE2B0D46174618D0FF2B21D09F
:10573800022B28D10846FFF775FE214690F9000094
:1057480009F0CDFD35692B783BB1124920460BF0A5
:10575800EBFB294620460BF0E7FB012015E0084645
:10576800FFF760FE3B46027829462046BDE8F04137
:10577800FFF7BCBE0846FFF755FE06220146204645
:10578800FCF722F9E9E700202070BDE8F08100BFAE
:10579800782401081B140108F8B5194B164628226D
:1057A80002FB063300241A790470022A07460D46C4
:1057B80003D0FE2A13D02046F8BD93F91820914251
:1057C800F9DB93F91C309942F5DC4FF0000165F3E1
:1057D80007013046FFF742FE01243870EBE7002945
:1057E800E9DB3046FFF718FFA842E4DD3046FFF753
:1057F80005FF40FA05F313F00100E6D10446DAE7A5
:10580800782401082DE9F84300230370124B17464A
:10581800282202FB073306461B79FF2B0C4603D0D0
:1058280000252846BDE8F8830846FAF7ABFC0628A9
:10583800F6D104F1FF3804F1050918F8010FFBF758
:1058480015FF05460028EBD0C845F6D12146384655
:10585800FFF728FE3070E4E778240108F8B5104E09
:105868004FF0280C0CFB0266002736790770FE2ED5
:1058780004460B46154603D0FF2E0BD0022E0DD141
:1058880018460BF091FA2A4601462046BDE8F84032
:10589800FFF782BFBDE8F840FFF7B4BF3846F8BD50
:1058A8007824010810B504460846B2B9FBF734FF5E
:1058B800042812D8DFE800F003090B0D0F0008498F
:1058C80020460BF089FB012010BD0649F8E7064980
:1058D800F6E70649F4E70649F2E70020F4E700BFD7
:1058E800081301080D130108121301081713010802
:1058F8001D13010810B504460068FDF711FA0249A6
:105908002068FDF70DFA10BD231301080B1E18BF00
:105918000123122A14D91D2A14D9312A8CBF08222E
:10592800052203710023016080F885304371C0F8B7
:10593800883080F88C3080F88D20A0F88E30704741
:105948000122EEE70322ECE790F88530642B08D8B3
:10595800C2180133DBB2517180F885301844002336
:105968004371704708B50530FAF702FCB0FA80F0C9
:10597800400908BD2DE9F043064691B0084688461F
:105988001546FAF7FFFB06F1050904464846FAF7FB
:10599800F9FBE4B2631CC7B2BB4203DB002011B0C1
:1059A800BDE8F0832246414648460BF0D9FA002864
:1059B800F4D1231D22461E44BA4203461BD300F1EC
:1059C80040036B44002403F8404C0028E6D09DF8BF
:1059D80000303D2BE2D1302368468DF80030FAF7CD
:1059E800D1FB2346DAB2904212D868460BF0DCF9B4
:1059F80028600120D3E716F8011F202905D040337D
:105A08006B440130C0B203F8401C0132D2B2D3E774
:105A180040326A44013312F8402C303A092AE1D95D
:105A2800BCE7000010B50D4B1B78022B04460ED1C5
:105A38000B4B93F8722052B19B6FB3F5215F07D2DD
:105A48000849FFF757FF08492046FFF753FF10BDE5
:105A5800FDD00649FFF74EFF0549F5E7850600200A
:105A6800DC040020261301085C13010892130108C6
:105A7800C813010810B50446FFF7D4FF206807498A
:105A8800FDF75CF9064B206819783031C9B2FDF78B
:105A9800C3F804492046FFF72DFF10BDFE13010887
:105AA800C4020020041201082DE9F0474379702B45
:105AB80090B080460F46164671D18379202B6ED15F
:105AC800C0790BF0FDF900285CD000254FF0020AE0
:105AD8002C4608F105094846FAF754FB824522D3BB
:105AE80005F140030DEB0305002305F8403CC4B362
:105AF800E8461D4618F8010B0BF0EAF97855013510
:105B0800EBB2A342F6D300253D550134E4B2684612
:105B1800FAF738FB6719FFB2874206EB050334D35F
:105B280000221A702DE008EB0A035B793D2B0ED09A
:105B3800202B07D005F140016A1C0DEB010505F883
:105B4800403CD5B20AF101035FFA83FAC3E72C4659
:105B5800F0E705F140036B4413F8400C0BF0B8F97B
:105B680078556846FAF70EFBE5B2A84207EB05033D
:105B780004F10104EDD800220A491A7030460BF0EE
:105B88002BFA012010B0BDE8F08707F140020DEBB9
:105B98000207013517F8402C1A70EDB2B7E700205C
:105BA800F0E700BF081401082DE9FF472C4E282311
:105BB80003FB016604463379FE2B0D4620D0FF2BEC
:105BC8004BD0022B2DD196F9185026490068FDF7C5
:105BD800B5F82846694609F082FB69462046FFF772
:105BE80089FE96F91C5020492068FDF7A7F86946F8
:105BF800284609F074FB69462046FFF77BFE10E053
:105C08000846FFF7FBFCDFF86490DFF864A08046E5
:105C18000027FEB20123324629466846FFF766FC94
:105C280010B904B0BDE8F087BBB248FA03F3DB074C
:105C380011D520684946FDF781F806F13001206842
:105C4800C9B2FCF7E9FF20685146FDF777F86946C5
:105C58002046FFF74FFE0137DBE70649CDE700BFD7
:105C6800782401080A140108121401081A140108FA
:105C78001D14010821140108F0B504468BB008462C
:105C88000D46FFF7E3FC254F254906462068FDF73A
:105C980055F8282303FB05772068B968FDF74EF807
:105CA80020492068FDF74AF82EB91F492046FFF71A
:105CB80021FE0BB0F0BD0122294602A8FFF72AFDFC
:105CC800206802A9FDF73AF83B79FE2B03D0FF2B99
:105CD8001AD01649EAE72846FFF7A4FB05781449C5
:105CE8002068FDF72BF805F130012068C9B2FCF7F0
:105CF80093FF10492068FDF721F8012EE9D10E49DC
:105D08002068FDF71BF8E4E70C4B02A95A786846AF
:105D1800FFF7C8FD0028DCD06946F1E778240108C0
:105D28001A1401081D14010830140108041201088E
:105D3800401401082E14010843140108C40200206D
:105D480070B590F88E3004466BB990F88F30012BFF
:105D580001D9032B07D1214B1B78022B03D02049F3
:105D68002046FFF7C7FD1D4E002594F88E102B29FD
:105D780003D9002384F88C3020E04B1C84F88E3043
:105D880094F88F30012B09D10846FFF715FB00283E
:105D9800EBD10846FFF722FB38B1E6E7022B0ED11C
:105DA8000846FFF709FB0028DFD02046FFF764FF0D
:105DB800013594F88D30EDB2AB42D6D270BD032BCD
:105DC80008D10846FFF70AFB0028CED03378022B0B
:105DD800DFD1EAE7002BF9D0E7E700BF850600200E
:105DE8005214010838B53D4B1A6890F88C30012BD5
:105DF800044671D1D0F88830D31AB3F5FA7F6BD343
:105E0800374DC0F888202846FBF745FB09F076FA9D
:105E180001462068FCF792FF32492068FCF78EFFA4
:105E280005F11400FBF721FF09F068FA0146206824
:105E3800FCF784FF2C492068FCF780FF95F8940054
:105E480009F05CFA01462068FCF778FF27492068CA
:105E5800FCF774FF95F98C0009F05AFA014620689E
:105E6800FCF76CFF22492068FCF768FF95F992005F
:105E780009F04EFA01462068FCF760FF1B492068CC
:105E8800FCF75CFF95F98E0009F042FA014620689C
:105E9800FCF754FF17492068FCF750FF05F1500044
:105EA800FBF7E9FE80B209F03DFA01462068FCF7ED
:105EB80045FF0E492068FCF741FF05F16400FBF738
:105EC800DAFE80B209F02EFA01462068FCF736FFA8
:105ED80009492046FFF70EFD38BD00BF8049002064
:105EE800B42F00206F1401087114010874140108FC
:105EF80072140108771401087A14010830B50446B1
:105F080089B0FFF78FFD13492046FFF7F3FC1249CC
:105F18002068FCF713FF114B1B78022B18D1104D8A
:105F280095F8723093B1206805F17C01FCF706FF03
:105F38000C492068FCF702FF696F6846FBF7E6FC2E
:105F480069462046FFF7D6FC09B030BD0649F8E798
:105F58000649F6E77C1401089D140108850600200F
:105F6800DC04002074140108A41401085814010862
:105F78002DE9F043304EDFF8C480DFF8C49091B0CB
:105F88000446002794F88D20FBB29A4209D994F868
:105F98008E50F37DAB4207F1010705D8002384F842
:105FA8008C3011B0BDE8F083284609F0A7F9014606
:105FB8002068FCF7C3FE41462068FCF7BFFE731952
:105FC8000E35187E09F09AF901462068FCF7B6FEEE
:105FD8001C492068FCF7B2FE56F8250009F0ACF918
:105FE80001462068FCF7AAFE17492068FCF7A6FEC0
:105FF800164908A80AF0F0FF56F82500FAF76EFDD2
:106008004946FAF7C3FD09F043FEFAF7C1FF6946AE
:1060180009F02FF96846FBF7B1FB20686946FCF7E1
:106028008DFE08A92046FFF765FC94F88E300133F1
:1060380084F88E30A6E700BF980A0020B91401083A
:1060480000007A3AC0140108CA140108D0140108E3
:106058002DE9F041254E264FDFF8988004460025AB
:1060680094F88D20EBB29A423ED994F88E30102BDA
:1060780037D8DFE803F00913181A1C1E202224263B
:10608800282A2C2E303234002046FFF7CBFC94F817
:106098008E30013384F88E300135E1E71649204609
:1060A800FFF728FCF3E71549F9E71549F7E715491C
:1060B800F5E71549F3E71549F1E71549EFE71549FC
:1060C800EDE71549EBE71549E9E71549E7E715490C
:1060D800E5E71549E3E74146E1E73946DFE73146B9
:1060E800DDE7002384F88C30BDE8F0814017010813
:1060F80009170108DC160108D5140108F514010870
:106108001F150108441501086C15010890150108B0
:10611800B4150108DD150108061601084A1601081C
:106128006C1601088E160108AD1601082DE9F0431A
:10613800037993B00446C3B190F88C30013B032B2C
:1061480019D8DFE803F00252575C006803685B69FE
:10615800984768B1206803689B6998470023AB4952
:1061680084F88C302046FFF7C5FB13B0BDE8F083F8
:106178002046FFF737FEA64B1E6894F885308BB192
:10618800D4F88830F31AB3F5FA6F0BD9A149204631
:10619800FFF7B0FBA0492046FFF7ACFB002384F8CB
:1061A800853063719B4FDFF87482DFF87492206842
:1061B80003685B6998470028D7D0206803689B6903
:1061C80098470A280546C4F888601DD00D281BD0BA
:1061D8002C2819D03B2817D001462068FCF71CFD55
:1061E80029462046FFF7B0FBE1E713B0BDE8F043CE
:1061F800FFF72EBF13B0BDE8F043FFF7A1BD13B002
:10620800BDE8F043FFF7B4BE39462046FFF772FBFE
:1062180041462046FFF7A6FB50B1022384F88C3094
:10622800002384F88E30002384F885306371BEE73C
:1062380049462046FFF796FB0028EED179492046CB
:10624800FFF790FB0028E8D177492046FFF78AFB43
:10625800054618B12046FFF751FEE4E7734920468A
:10626800FFF780FB40B12046FFF704FC032384F8C6
:106278008C30A4F88E50D6E76D492046FFF772FBA4
:1062880050B12046FFF7F6FB032384F88C304FF417
:106298008073A4F88E30C6E766492046FFF762FB94
:1062A80040B12046FFF7E6FB032384F88C304FF417
:1062B8000073EEE760492046FFF754FB40B12046E3
:1062C800FFF7D8FB032384F88C304FF44073E0E7E2
:1062D8000AAA02A92046FFF7E7FB002846D002A930
:1062E8000DF10200FFF7D4F920B954492046FFF711
:1062F80001FB98E7524B1B78022B06D09DF8020051
:10630800FFF76CF808B14F49F0E79DF828303F2BAC
:106318000DD12046FFF7AEFB9DF8025020462946D6
:10632800FFF7AAFC29462046FFF73EFC7BE70BB99E
:106338004549DBE79DF802500AA92A460DF10300FA
:10634800FFF78CFA08B94149D0E72046FFF792FBDE
:1063580029462046FFF790FC9DF80330002B3FF4B8
:1063680062AF05213A48FBF7B0FC5CE739492046A3
:10637800FFF7F8FA90B136480621FBF7A6FC20464D
:10638800FFF778FB2E4B1B78022B05D02D492046B2
:10639800FFF7B0FA3049A9E73049A7E73049204666
:1063A800FFF7E0FA28B101212948FBF78EFC2D49B7
:1063B8009CE72D492046FFF7D5FA90B124480721DC
:1063C800FBF783FC2046FFF755FB1D4B1B78022B80
:1063D80005D01C492046FFF78DFA244986E7244951
:1063E80084E7244901AA2046FFF7C4FA00285AD0B6
:1063F800019D092D01D9204978E72046FFF73AFB8E
:106408001E4B1B789D423DD11D496FE7821701083D
:10641800804900209C1701089E17010801230108E4
:10642800A81701080814010801220108AD1701087E
:10643800B0170108B5170108BB170108C1170108F3
:106448008506002052140108DD170108F517010818
:1064580080300020081801080F18010826180108C4
:106468003A1801083F180108561801085D18010874
:10647800761801088C18010898180108C402002031
:10648800BC1801082A461D480A21FBF720FC1C49B4
:106498002068FCF753FC05F13001C9B22068FCF70D
:1064A800BBFB184922E718492046FFF75BFA054667
:1064B80040B10123154984F88C302046FFF71AFAB9
:1064C800134913E713492046FFF74CFA28B1042370
:1064D80084F88C3084F88E50A5E60F492046FFF7E3
:1064E80041FA08B103213DE794F885100B4A0C4B9B
:1064F80000290CBF11461946F8E600BF803000207D
:10650800D118010804120108FA180108E71801084F
:10651800001901081D190108271901086817010841
:10652800741701080148FFF701BE00BFEC05002001
:1065380070B5224CE569AB0607D523689E0604D5DD
:10654800606A1F4BC0B21B6898471F232806236246
:1065580015D52368190612D51A4B1B4A19881388B2
:1065680089B29BB2994219D013880133C3F3080347
:1065780013801388154A9BB2D35CDBB2A3626A0608
:106588001AD50E4803685B0616D5FBF79BFE402319
:1065980003620F4BBDE870401B6818470748FBF7BC
:1065A8009AFE4023236250E8003F43F0400340E84E
:1065B8000032002AF7D1E2E770BD00BF008000403A
:1065C8003C020020603500205E3500205E3300204C
:1065D800400200200848094A0188138889B29BB202
:1065E8009942F9D013880133C3F308031380138841
:1065F800034A9BB2D05C70475C3300205A330020BA
:106608005A310020FFF7E6BF70B588B00C46064641
:10661800154600211C2201A80AF07EFC231E18BF83
:1066280001231B03CDE9033501A90C230348029676
:106638000594069308F04AFA08B070BD008000403F
:1066480010B5064C236823F001032360FFF7DCFF35
:10665800236843F00103236010BD00BF00800040A1
:1066680013B5134C2046FBF724FEE9B111484FF44B
:1066780000524FF48061FFF7E3FF23680E4823F0D0
:1066880001032360636823F480336360236843F065
:106698000103236001210923CDE9003103231A46B0
:1066A800FCF78CFBFCF7D2F9012002B010BD00BF4B
:1066B80000800040A08601000008004813B5134C74
:1066C8002046FBF7F6FDE9B111484FF400524FF4AC
:1066D8008061FFF7B5FF23680E4823F001032360AC
:1066E800636843F480336360236843F001032360E5
:1066F80001210923CDE9003102220323FCF75EFBC7
:10670800FCF7A4F9012002B010BD00BF00800040D2
:10671800A08601000008004873B5384C236823F0B0
:106728000103012023600926FBF799FD0546019026
:106738000323334800960A220221FCF73FFB032378
:106748001A462F482946CDE90065FCF737FB002299
:106758002C481146FFF758FF236823F000532360A5
:1067680004F1080353E8003F23F0604304F10801F3
:1067780041E80032002AF3D104F1080353E8003F4E
:1067880023F0606304F1080242E800310029F3D1E4
:106798001D4BA02283F8262340255D601748FBF790
:1067A8009AFDFBF78FFD194B25621980184B19804C
:1067B800FBF77FFD174B1980174B1980636823F48B
:1067C80000636360A36823F00803A360636823F48D
:1067D80080436360A36823F02203A360A36843F4A3
:1067E8008053A360236843F001032360C3699A02BE
:1067F800FCD5C3695B02F9D502B070BD00800040CA
:1068080000080048801A060000E100E05E3500201C
:10681800603500205A3300205C3300200649074ABF
:106828000B8812880133C3F3080392B29A421EBF41
:10683800034AD0540B807047603500205E35002035
:106848005E330020F8B5012380F86C3090F8BD3035
:10685800044603F0FF005BB194F8BD5004F16C07E7
:106868000026B3B29D4204D8002384F8BD3001202D
:10687800F8BD17F8010FFFF7D1FF0136F1E7000067
:106888000148FBF70DBD00BF0080004007B521B1EE
:1068980003B05DF804EBFCF721BB0D4B0D481A68FB
:1068A80022F001021A605A6822F400425A601A68FB
:1068B80042F001021A600923019100930222032386
:1068C8000121FCF77BFA03B05DF804EBFCF7BEB8D6
:1068D800008000400008004837B50446FFF71CFF59
:1068E800134B144D1A6822F001021A605A6842F4D8
:1068F80000325A605A6842F480325A601A6842F08C
:1069080001021A6001210923CDE900312846032339
:106918000222FCF753FA0222114628460323FCF709
:10692800D2FA0021204603B0BDE83040FFF7AEBFE1
:106938000080004000080048002282810271C28065
:10694800028182720261FFF7C7BF036810B504466F
:106958001B689847237A082B03D9092B02D00023F8
:10696800237210BD236820465B6898470028F6D03C
:10697800FCF7B4FA0A232372BDE81040FFF780BF82
:1069880001460148FFF7E1BFC8150020014601484C
:10699800FFF7DBBF8C06002010B500210446FFF787
:1069A80075FF0023237210BD0148FFF7F5BF00BF34
:1069B800C81500200148FFF7EFBF00BF8C06002074
:1069C80008B5017A094A0929126801D8026108BD87
:1069D8000169521A142AFAD900210172FFF756FFE9
:1069E8000348FBF76FFC40230362F0E7804900206F
:1069F800008000400238C0B210289ABF014B185CD2
:106A080000207047CA2301083B4B0246586A137A94
:106A180010B580B233B19389C31A9BB2FA2B84BFE5
:106A280000231372137A9081052B19D8DFE803F03D
:106A380003080E334A564F2912D1012313720FE06F
:106A4800572901D10223F9E70023F7E70023FF299B
:106A5800937206D141F204731381537E002BF3D154
:106A680010BD9F290FD901F01F000124947282F8EC
:106A78003200FFF7BFFF507218B982F84B40092364
:106A8800DCE70523DAE71829DED80029F7D0032345
:106A980051721372E1E7B2F86E02B2F87242431C07
:106AA8002340B2F870429C421EBF801880F87412CE
:106AB800A2F86E32937A517A0133DBB2994293721B
:106AC800DDD9CDE7907A431C1044DBB29372C176CE
:106AD800517A9942C4D801239376D0E7907A431C1F
:106AE8001044DBB2937280F83210517A9942B7D2CF
:106AF800012382F84B30C2E7004401402DE9F043FE
:106B080089B0002301AFB0F868908DF804300446CE
:106B1800B8460125B4F86A2048461146EEB2FCF79B
:106B280001F8A0B1192D11D091451FBFA318B4F8D1
:106B38006C1093F86E30013214BF0A40002308F835
:106B4800013F18BFA4F86A200135E3E72E46B6B224
:106B58000024013417F8010BA4B2FFF75FFEA64228
:106B6800F7D8012009B0BDE8F08370B590F86650F9
:106B780000F14C040026B3B29D4200D870BD14F851
:106B8800010FFFF74BFE0136F5E770B5457E044669
:106B980005B1FEE7012680F84C6090F8663033B105
:106BA800FFF7E3FF84F866503546284670BDB0F815
:106BB8006A10B0F86800FBF7B5FF0028F5D020464A
:106BC800FFF79CFFF0E7027FC37E02F0070243EA6B
:106BD80002230B80838BC3F3CA034B80C369C3F3BF
:106BE8008A338B8090F82030C27F03F00F03DB01DB
:106BF80043EA5203CB80038CC3F30A130B81036A65
:106C0800C3F3CA334B8190F8243090F8232003F063
:106C18001F039B0143EA92038B81838CC3F34A13BE
:106C2800CB81C38CC3F30A030B8290F8283090F809
:106C3800272003F03F035B0143EAD2034B82836AB8
:106C4800C3F38A138B82438DC3F34A03CB8290F834
:106C58002C3090F82B2003F07F031B0143EA12131A
:106C68000B83C36AC3F3CA134B83C38DC3F38A036D
:106C78008B8390F8303090F82F20DB0043EA5213D2
:106C8800CB8390F8312040F2547312F0010F14BFF7
:106C98001A46AC220A8490F8312012F0020F08BF7D
:106CA800AC234B847047437E70B504460D463BB118
:106CB800002303728E18B54203D100232372A376F2
:106CC80070BD236815F8011B1B6820469847F2E73A
:106CD8000346407E30B568B193F8664004F0FF057E
:106CE8004CB103F14D040C6093F86610117000224A
:106CF80083F8662030BD2846FCE7000042765AB388
:106D08000123037640F2FF11A0F86C1040F2FF71E6
:106D18000023A0F872127F2180F84C30A0F86A3066
:106D28008376A0F8683080F84B30A0F8703280F88D
:106D38006630A0F86E32A0F8763AA0F8743AA0F857
:106D4800781A80F8FA3A52B9054B064A1A60064B87
:106D5800064A1A60FFF7F0BD01760029D2D17047C4
:106D68003C0200208969000840020020B16900083F
:106D7800F8B5477E04460D4617B100263046F8BDE3
:106D8800037E002BF9D0FFF71BFEA37E03F0FF065E
:106D9800002BF2D0A77629462046FFF714FFEDE72F
:106DA800427E10B50346E2B9007EB8B193F84C4074
:106DB80004F0FF0094B11C7983F84C200CB11A71CF
:106DC800DA80DC889A790134052ADC8007D0092A20
:106DD80005D0012A4FF0000305D10B7010BD012327
:106DE800FBE70020FAE71846F8E70346007E60B1A3
:106DF80093F84B2002F0FF003AB1002283F84B20B1
:106E080093F8323003F01F030B707047F8B506464D
:106E18000D461746002119224D300AF07DF8284604
:106E2800FFF7E8FD05F01F050446603D0134024602
:106E380086F84D50394606F14E00E4B20AF0D4F80F
:106E480086F86640F8BD70B590F8FA4AC4B9B0F84B
:106E5800745AB0F8762AAE1AB3B2360444BF8033F7
:106E68009BB27BB1954208D08318013293F87A4AD5
:106E7800B0F8783A1A40A0F8762A0C70012070BD54
:106E88000020FCE71846FAE710B53A4C86B01822FD
:106E9800002168460AF040F8237837488DF8063014
:106EA800FDF7DCFCADF800003348FDF7EEFC9DF87B
:106EB800073094F851208DF8030062F303038DF82E
:106EC80007302E4B93F87220002A47D09DF80520F2
:106ED80042F001028DF8052093F8912093F8923042
:106EE8008DF8042003F00F039DF80720244863F36E
:106EF8000712244B8DF807201A78931E5A425A41DC
:106F0800214B1B795B0043F0010343EA820390F8AD
:106F18009320402A8CBF0022012243EAC2039DF835
:106F2800022003F00F0322F00F0213438DF8023002
:106F3800FAF7B1FA9DF8023040288CBF00200120F2
:106F480060F304138DF8023010482C236A460B2195
:106F58008DF80830FFF75AFF06B010BDBDF80430B1
:106F680023F4FF7323F0010343F07F03ADF80430EB
:106F78000523B9E7C40200205C300020DC040020AF
:106F8800B42F002085060020B8050020C815002071
:106F98007FB518220021684609F0BEFF42F642007C
:106FA800FAF796FCADF800004FF42150FAF790FC80
:106FB8000749ADF80200142201A8FAF7F3FC0548C6
:106FC8006A460421FFF722FF07B05DF804FB00BF03
:106FD80032190108C815002010B5124C86B01822C5
:106FE8000021684609F098FF94F87230B3B1606FD9
:106FF800FAF76EFCADF80000A06FFAF769FC1422EE
:10700800ADF8020004F17C0101A8FAF7CBFC0648B0
:107018006A460521FFF7FAFE06B010BD034914229F
:10702800F2E700BFDC040020C815002004120108A4
:107038002DE9F04F0C463549282303FB041189B08C
:1070480007462046FEF7DAFA0B79D1F82080FE2BA6
:10705800814603D14FF6FF73984206D14146384620
:1070680009B0BDE8F04F09F0B7BF2046FEF7DAF9DE
:10707800002590F800B02E46AA462C46EAB24046B3
:107088000192F9F77FF8019A013090424FF02D01F3
:1070980002D809B0BDE8F08F18F802000AF1200CF8
:1070A800EC440AF101032C28DBB20CF8180C00D0D0
:1070B80040BB5E4503D049FA06F0C00718D50DF16C
:1070C800080E0022D0B254FA82FC83425FFA8CFC8C
:1070D80008D85444013404F0FF040136502CF6B2A9
:1070E8000FD9FEE71EF8010B07F80C000132E9E79B
:1070F8003955631CDBB218F80220FA540234E4B2A2
:10710800EBE7002301359A46B8E700BF7824010869
:10711800054B1870054B064800221A70054B0122D2
:1071280007211A70FBF7F2BC0D2E00200E2E00204E
:107138003C2000200C2E0020054A0648002313702E
:10714800054A1370054A07211370FBF7DFBC00BF1F
:107158000D2E00203C2000200E2E00200C2E00209A
:1071680010B50B78033B0C46082B0BD8DFE803F06F
:1071780010050C1A1D0A0A0A0E00042100F67420D4
:10718800FBF7C4FC207810BD0521F7E70B21F5E7D4
:10719800042100F67420FBF7B9FC0521FBF7B6FCC7
:1071A8000B21EDE7FFF7C8FFECE74878FFF7B0FFE2
:1071B800E8E707B58DF807100DF10701FFF7D0FFD5
:1071C80003B05DF804FB0000F0B5704D2C782B2C53
:1071D80087B00ED918220021684609F09DFEFF23CA
:1071E8006B488DF800306A460721FFF70FFE07B09D
:1071F800F0BD684E3178182200294AD1664F68469A
:1072080009F08AFE282303FB04738DF800401B79DC
:10721800FE2B29D0FF2B2FD0022B09D1012320468A
:107228008DF80130FEF7FEF890F900308DF8123035
:107238002B78282202FB03770DF10200B96810228F
:10724800FAF7B0FB524807216A46FFF7DFFD012332
:10725800297852483370FFF7EBFE5148072107B0F1
:10726800BDE8F040FBF752BC042320468DF80130FE
:10727800FEF7D8F80378D9E7052320468DF80130C2
:10728800FEF7D0F8062201460DF11200FAF78AFB44
:10729800CEE7012947D10021684609F03DFE3E4B63
:1072A8008DF80040282202FB04331A79022A0BD0F9
:1072B800FE2A19D0002436486A460821FFF7A6FDA1
:1072C80044B302233370C8E71A7D8DF805201A7E6F
:1072D8008DF801201A7F8DF80320196906220DF117
:1072E8000700FAF75FFBE5E75B6A83B11B882B4968
:1072F800ADF8013015220DF10300FAF753FB2748CA
:10730800F8F740FF142894BF00240124D3E74FF670
:10731800FF73ECE734702B7801332B70214B1B780B
:10732800002B9AD063E7022968464FF0000116D176
:1073380009F0F2FD1C498DF8004017220DF10100FB
:10734800FAF730FB1548F8F71DFF6A46044609218D
:107358000F48FFF75BFD2B2C15D90323B2E709F083
:10736800DBFD12498DF8004017220DF10100FAF7F4
:1073780019FB9DF800300648803B6A4609218DF8C4
:107388000030FFF743FD00233370C4E70D2E0020C3
:10739800C81500200E2E0020782401080F2E00208A
:1073A8003C2000200C2E0020242E00203B2E002004
:1073B80010B500230B70024600782B280C4611D814
:1073C800094B282101FB00331B79FF2B06D0B2F9AA
:1073D8000110FEF743F82070012010BD511CFEF784
:1073E80061F8F8E71846F8E7782401080438072810
:1073F8000DD8DFE800F004060C080C0C0C0AFFF7A7
:10740800C7BDFFF7E9BDFFF7DFBEFFF73DBD70471A
:10741800D20638B505460C4604D5BDE838402049A3
:1074280009F0DABDCB044CBF1E491F4909F0D4FD51
:10743800A1070BD51D49284609F0CEFDE3072ED438
:1074480028461B49BDE8384009F06EBDA20501D5A4
:107458001849F0E7230601D51749ECE7E00501D5FF
:107468001649E8E7164BA34301D11649E3E7E103C0
:1074780001D51549DFE7220501D51449DBE7E30605
:1074880001D51349D7E7600701D51249D3E721078A
:1074980001D51149CFE7E202D0D51049CBE738BD75
:1074A80044190108491901084D1901085219010820
:1074B8007719010857190108DA1D0108CD1F0108BD
:1074C800100001005C190108611901083A1E010841
:1074D80066190108691901086E190108721901086D
:1074E80010B51422044600212A3009F015FD0023A6
:1074F800C4F8D032A4F8D432012384F8D63210BDAF
:107508000B68C0F890304B68C0F894300B7A80F85C
:107518009830012380F82D3080F8333090F8963079
:10752800DB0980F8D5327047993001F1280351F80A
:10753800042B40F8042B9942F9D10B8803808B78EF
:107548008370704710B500F1C40301F1340251F89B
:10755800044B43F8044B9142F9D1012380F82E30B3
:1075680010BDF83001F11C0351F8042B40F8042B2E
:107578009942F9D10B780370704710B500F21513D2
:1075880001F11C0251F8044B43F8044B9142F9D124
:10759800012380F8323010BD10B500F2311301F12B
:1075A8001C0251F8044B43F8044B9142F9D140F2C4
:1075B80001134385012380F8303080F8D23290F8E7
:1075C800D53253B990F8D4323BB9D0F83931C0F834
:1075D8002C32D0F83531C0F8283210BD00F26710CF
:1075E80001F1100351F8042B40F8042B9942F9D10A
:1075F8000B880380704700F24D1001F1180351F811
:10760800042B40F8042B9942F9D10B88038070476A
:1076180010B500F2791301F1140251F8044B43F844
:10762800044B9142F9D1012380F83130D0F89930D8
:1076380013F0100308D0D0F89D3013F010031CBFCE
:10764800D0F8A130C3F3001380F83D3010BD00F22C
:107658008D1001F1140351F8042B40F8042B9942C2
:10766800F9D10B880380704791F8203030B57BB989
:107678000B4600F2A31201F1340453F8045B42F8FC
:10768800045BA342F9D11B881380012380F82F30B3
:1076980091F82030012B0ED100F2D91301F13402F8
:1076A80051F8044B43F8044B9142F9D10A881A80E7
:1076B800012380F8343030BD0B68C0F80F324B68B6
:1076C800C0F813320B7A80F81732012380F8D332CE
:1076D80070470B68C0F818324B68C0F81C32012399
:1076E80080F8323070470B68C0F820324B68C0F819
:1076F8002432012380F83630704710B500F50A733C
:1077080001F13C0251F8044B43F8044B9142F9D182
:10771800012380F8303080F8D43210BD10B500F560
:10772800197301F1340251F8044B43F8044B9142A8
:10773800F9D10A881A80012380F82C3010BDF0B5E1
:1077480000252C460126AB4206D803680C4004FAF3
:1077580002F213430360F0BD06FA05F73C43013516
:10776800F1E770B50446084694F82A6016B9002671
:10777800304670BD94F8E0300022022B84F82A20AD
:10778800F5D90A60D4F83551002DC8BF6D423223AF
:10779800B5FBF3F11E2301EB4101FFF7D0FFD4F84D
:1077A800351102231E22C90FFFF7C9FFE0E770B5A4
:1077B8000446084694F82B6016B90026304670BD7A
:1077C80094F8E0300022022B84F82B20F5D9D4F865
:1077D80039510260002DC8BF6D423223B5FBF3F169
:1077E8001E2301EB4101FFF7AAFFD4F83931002B22
:1077F8004FF002034FF01E02B4BF03211946FFF7F2
:107808009EFFDBE738B50446084694F8D022AAB9AB
:1078180094F82C30DBB384F82C2004F5197304F2A7
:107828009A2204F5267153F8045B42F8045B8B42F4
:10783800F9D11B8813800123A4F8D03200230360F8
:10784800182594F8D132312B06D85A1C234484F8D1
:10785800D12293F89B12E1B994F89A1201231940A6
:107868000722FFF76CFF94F89A1201230F22C1F345
:107878004001FFF764FF94F89A1201231722C1F31D
:107888008001FFF75CFF002384F8D03201231846FB
:1078980038BD2A46083D0723EDB2FFF750FFF82D03
:1078A800CFD194F8D132312BD6D8EFE703462DE962
:1078B800F04793F82D600846002E62D093F81552D1
:1078C800D3F89010B3F88B4193F8D58293F8D3721C
:1078D8000022AD1A83F82D2001F1010118BF0125FE
:1078E8004CB1632CD7BFC4EB84143F2431346422D9
:1078F800D8BFB4FBF2F4B3F91331002B44D064229F
:1079080093FBF2F3522BA8BF5223132BB8BF1323B8
:10791800A3F113094FF0000A05235246C0F800A04E
:10792800FFF70DFF022305225146FFF708FF4146E6
:1079380001230722FFF703FF01230822FFF7FFFEB9
:10794800514601230922FFF7FAFE02230A22FFF714
:10795800F6FE01230C22FFF7F2FE01230D22394621
:10796800FFF7EDFE01230E222946FFF7E8FE072365
:1079780013222146FFF7E3FE06231A224946FFF7A2
:10798800DEFE3046BDE8F0879946C3E72DE9F843A7
:1079980090F82E800D46B8F1000F3AD090F8E130FB
:1079A8000021FF2B80F82E1003D00F2B28BF0F23A8
:1079B800194690F8E090B9F1030F2DD84FF0000662
:1079C8002FD07F273446002228462A600423FFF759
:1079D800B6FE022304224946FFF7B1FE0122022126
:1079E8003846FAF7C9F90823014606222846FFF760
:1079F800A6FE02230E223146FFF7A1FE02221146FF
:107A08002046FAF7B9F90A23014616222846FFF755
:107A180096FE4046BDE8F883A9F10306062E28BF66
:107A280006260A23B0F8D870D0F8D440B7FBF3F78D
:107A38000B4B7F2FA8BF7F279C4208DC094B9C4239
:107A480009DB64234FF0030994FBF3F4BBE7064C0E
:107A58004FF00309B7E7054C4FF00309B3E700BF40
:107A6800C3C9C1003D363EFF18F00100E80FFEFF14
:107A78002DE9F04F90F8303085B005460E462BB909
:107A880000230093009805B0BDE8F08F002380F82C
:107A9800303090F8D2320093002BF1D0D0F8280281
:107AA800F9F720F86A49F9F771F86A49F9F76EF8B1
:107AB8008146D5F83501F9F715F86549F9F766F8FB
:107AC8006449F9F763F88046484607F0F7FF8346AC
:107AD800404607F0F3FF0746D5F83901F9F702F8F1
:107AE8005B49F9F753F85B49F9F750F80446D5F8BC
:107AF8002C02F8F7F7FF5649F9F748F85549F9F70E
:107B080045F801462046F8F737FF824608F012F894
:107B18000190404608F00EF80446484608F00AF876
:107B28000390504607F0CAFF214602905846F9F7DD
:107B38002DF8039B044619463846F9F727F8029AA8
:107B48001146F9F723F801462046F8F715FF019981
:107B580004463846F9F71AF8214607F093FF3E49DC
:107B6800F9F714F800210446F9F7AEF920B12046D8
:107B78003A49F8F703FF04462046F9F7E3F980B2DB
:107B8800A0F1B40424B2002CBCBFB43004B2B4F5E4
:107B9800B47FA8BFA4F5B47449464046A8BF24B230
:107BA800F8F7EAFE4FF07C51F8F7F0FF07F0C2FF54
:107BB8004FF07C5180465046F8F7E8FF07F0BAFFCF
:107BC8000146F8F7E3FF5946F8F7E0FF3946F8F7BA
:107BD800DDFF414607464046F8F7D8FF01463846DC
:107BE800F8F7CCFE07F050FF002707F02BFF1C49E1
:107BF800D5F841513760642395FBF3F5F8F7C6FFD4
:107C0800F9F7A0F9F8F76EFFF9F79CF902220321BA
:107C1800FAF7B2F80C2301463A463046FFF78FFDD3
:107C28002846F8F75FFFF9F78DF902220321FAF7E2
:107C3800A3F80D2301460C223046FFF780FD0723E9
:107C48001922032194FBF1F1FFF779FD1AE700BF30
:107C580095BFD63335FA8E3CE12E65420000B44319
:107C6800706D424B2DE9F84390F8319004460D466B
:107C7800B9F1000F3BD000261E4980F83160D0F8DA
:107C88008501F8F783FF08F003F81A498046D4F80D
:107C98007D01F8F77BFF07F0FBFFB4F989112E602F
:107CA8000746404601EB8104F9F74CF9012202210D
:107CB800FAF762F80923014632462846FFF73FFDE6
:107CC8003846F9F73FF901220221FAF755F8082357
:107CD800014609222846FFF732FD0B2311222146CF
:107CE800FFF72DFD01231C223146FFF728FD4846EA
:107CF800BDE8F883000020412DE9F84390F83D9055
:107D080004460D46B9F1000F3BD000271E4980F804
:107D18003D70D0F88501F8F739FF07F0B9FF1A4927
:107D28008046D4F87901F8F731FF07F0B1FFB4F9CC
:107D380089112F600646404601EB8104F9F702F9E4
:107D480001220221FAF718F8092301463A46284683
:107D5800FFF7F5FC3046F9F7F5F801220221FAF7AA
:107D68000BF80823014609222846FFF7E8FC0B23F5
:107D780011222146FFF7E3FC01231C221946FFF7D5
:107D8800DEFC4846BDE8F883000020412DE9F843B1
:107D980090F8329004460D46B9F1000F46D00027FE
:107DA800244980F83270D0F81901F8F7EFFE22491B
:107DB800F8F7ECFE2149F8F7E1FD07F069FF1D49E6
:107DC8008046D4F81D01F8F7E1FE1B49F8F7DEFEFE
:107DD8001B49F8F7D3FD07F05BFF1A490646D4F8AC
:107DE8001802F8F7D3FE07F053FF2F600446404609
:107DF800F9F7A8F80B2301463A462846FFF79FFCF7
:107E08003046F9F79FF80A2301460B222846FFF768
:107E180096FC2046F9F796F801220321F9F7ACFF02
:107E28000B23014615222846FFF789FC4846BDE882
:107E3800F88300BFE12E65420000A04000006144C5
:107E48000000E1430000C84238B50346084693F8ED
:107E5800334014B90024204638BD93F8D652691C23
:107E6800C9B20022042983F8332083F8D61203D933
:107E7800012183F8D612EDE7012DEBD193F8941088
:107E880002601823FFF75BFC042318222946FFF73A
:107E980056FCE0E71C2945D8DFE801F00F1214165C
:107EA800181A1C1E44204422442426282A2C2E302A
:107EB800323436383A3C3E4042001B4909F08CB80F
:107EC8001A49FBE71A49F9E71A49F7E71A49F5E7A2
:107ED8001A49F3E71A49F1E71A49EFE71A49EDE7B2
:107EE8001A49EBE71A49E9E71A49E7E71A49E5E7C2
:107EF8001A49E3E71A49E1E71A49DFE71A49DDE7D2
:107F08001A49DBE71A49D9E71A49D7E71A49D5E7E1
:107F18001A49D3E71A49D1E71A49CFE71A49CDE7F1
:107F28001A49CBE71A49C9E7D11D01084D190108BB
:107F3800791901087E1901088319010888190108AF
:107F48008D19010892190108971901089C1901084F
:107F5800A1190108A6190108AB190108B0190108EF
:107F6800B5190108BA190108BF190108C41901088F
:107F7800C9190108CE190108D3190108D81901082F
:107F8800DD190108E2190108E7190108EC190108CF
:107F980004120108192941D8DFE801F00D10121464
:107FA80016181A1C1E4020222426282A2C2E30326D
:107FB8003436383A3C3E1A4909F00EB81949FBE7FD
:107FC8001949F9E71949F7E71949F5E71949F3E7AD
:107FD8001949F1E71949EFE71949EDE71949EBE7BD
:107FE8001949E9E71949E7E71949E5E71949E3E7CD
:107FF8001949E1E71949DFE71949DDE71949DBE7DD
:108008001949D9E71949D7E71949D5E71949D3E7EC
:108018001949D1E71949CFE71949CDE71949CBE7FC
:108028005719010892190108D11D0108F119010811
:108038004D190108F6190108FB190108001A010871
:10804800AB1901087E1901088D1901088819010862
:10805800051A0108BF190108831901080A1A01083D
:108068000F1A0108141A0108191A01081E1A010822
:10807800231A0108281A01082D1A0108321A0108C2
:10808800371A010804120108102925D8DFE801F081
:10809800090C240E1012141618241A1C1E2424204D
:1080A80022000E4908F098BF0D49FBE70D49F9E792
:1080B8000D49F7E70D49F5E70D49F3E70D49F1E7F4
:1080C8000D49EFE70D49EDE70D49EBE70D49E9E704
:1080D8000D49E7E70D49E5E70D49E3E757190108B9
:1080E8004D1901083C1A0108CD1F0108881901081B
:1080F800D3190108411A0108461A01087E19010816
:108108008D190108C9190108831901080A1A0108FB
:1081180004120108142921D8DFE801F00B0E10120F
:108128001420201620182020202020201A20201C6F
:108138001E000B4908F050BF0A49FBE70A49F9E756
:108148000A49F7E70A49F5E70A49F3E70A49F1E76F
:108158000A49EFE70A49EDE70A49EBE70A49E9E77F
:10816800D11D01084D1901084B1A01087E19010893
:108178008319010892190108501A0108B019010859
:1081880057190108551A01080412010823289ABF33
:10819800014B185C02207047DB2301080B46013BAA
:1081A8001146032B0BD8DFE803F002040608FFF79B
:1081B80071BEFFF7EFBEFFF767BFFFF7ABBF01491F
:1081C80008F00ABF0412010838B5384B0446821C6F
:1081D80003F1280153F8040B42F8040B8B42F9D140
:1081E80000252946C4E9245584F898502B2204F127
:1081F800990008F091FE2946342204F1C40008F0E1
:108208008BFE29461D2204F1F80008F085FE294658
:108218001C2204F2151008F07FFE29461C2204F2E5
:10822800311008F079FE29461A2204F24D1008F0A0
:1082380073FE2946122204F2671008F06DFE2946E3
:10824800142204F2791008F067FE2946162204F277
:108258008D1008F061FE2946362204F2A31008F0BA
:108268005BFE2946362204F2D91008F055FE29464D
:10827800C4E98655C4E98855C4F80F52C4F81352A6
:1082880084F817523C2204F50A7008F045FE294686
:10829800362204F5197008F03FFE3622294604F20A
:1082A8009A2008F039FE204638BD00BF2410010886
:1082B8002DE9F04FC77E837E457F867F90F820E0CA
:1082C80090F82B8090F819C0BF000C4647EA931726
:1082D80003F03F01037F03F0010247EA822705F01C
:1082E8000F02D20142EA530206F07F031B0143EA60
:1082F8001513C57F89B06D0045EAD6150EF0030643
:10830800059345EA462390F82160009306F01F057F
:10831800AD0145EA9E0390F8225090F824E00193BD
:10832800ED0045EA561390F8235002930EF0070625
:1083380045EA062390F82550039305F03F06760199
:1083480046EADE0390F8266090F827E00493B6002A
:1083580046EA95160EF0010546EA852690F828505B
:10836800069205F00F0B4FEACB1B4BEA5E0B90F819
:1083780029E00EF07F0A4FEA0A1A4AEA151A90F81D
:108388002A506D0045EADE1508F0030E45EA4E2531
:1083980090F82CE00EF01F094FEA891949EA98096C
:1083A800490190F82D80007E41EADC010CF0070CB1
:1083B80040EA0C204FEAC80848EA5E180791F9F726
:1083C800E3F8079920800846F9F7DEF86080384618
:1083D800F9F7DAF8069AA0801046F9F7D5F8059B60
:1083E800E0801846F9F7D0F820810098F9F7CCF822
:1083F80060810198F9F7C8F8A0810298F9F7C4F8E4
:10840800E0810398F9F7C0F820820498F9F7BCF8DE
:1084180060823046F9F7B8F8A0825846F9F7B4F800
:10842800E0825046F9F7B0F820832846F9F7ACF80F
:1084380060834846F9F7A8F8A0834046F9F7A4F8FE
:10844800E08309B0BDE8F08F4A78013A92B2023170
:108458000020F9F7FBB8000038B50446017500297B
:1084680044D04FF6FF730025A0F8F030204B80F879
:10847800BD5080F8CE5080F86C50C0F8D05080F8CD
:10848800655080F8DC5080F86650C0F8E05080F8FD
:10849800675080F8EA5080F86850C0F8EC5080F8CF
:1084A8006A50C0F8F43080F86B5080F80751C0F873
:1084B800085180F80E51C0F8105180F81651C0F8D4
:1084C800185100F58E70FFF70BF80A4B0A4A1A602C
:1084D8000A4B0B4AC4F8F453A4F8F853C4F8FC53F5
:1084E8001A602046BDE83840FEF726BA38BD00BFFE
:1084F8000000C07F3C02002095690008400200206F
:10850800BD690008037D70B504460D4613B9002601
:10851800304670BDFEF754FA94F8653003F0FF0654
:10852800002BF4D0002384F8653004F115012046AF
:10853800FFF78AFFA37D23449B7D8342E7D1294629
:108548002046FFF7B5FEE3E70346007D30B500B3EC
:1085580093F86C4004F0FF00DCB11D79002483F827
:108568006C4065B1132A1C7114D8134C227802B9D7
:10857800DA800132D2B2022A88BF00222270DC8857
:108588009A790134012ADC8002D0022A00D01AB973
:108598000A7030BDDC80F2E793F8672002F0FF0430
:1085A80032B1002283F8672004230B702046F0E7DD
:1085B80003230B70EDE700BFB5050020027D0346DD
:1085C8000AB90020704790F8682002F0FF0022B135
:1085D800002283F868200A70704793F86A2002F036
:1085E800FF002AB1002283F86A2001230B7070472C
:1085F80093F86B2002F0FF0022B1002283F86B2071
:108608000223F3E793F8662002F0FF00002AD8D08F
:10861800002283F866205A7DEE2AD2D1DB7D812B99
:10862800CFD10323E2E738B504461D46EA230846BE
:1086380084F86D30AB1C114684F86E302A4684F8F5
:108648006F0004F1700008F0CFFC04F16D012046C2
:10865800FFF7FAFE6319043583F87000EDB284F869
:10866800BD5038BD13460A468221FFF7DCBF000023
:1086780070B50C4600F1BE060546102200213046B2
:1086880008F04AFC6379032B10D12079FFF77EFDAF
:1086980022680146D2B23046FFF780FD94F90630D1
:1086A800002B03DB0349304608F03EFC012385F824
:1086B800CE3070BD77190108002310B51A464FF661
:1086C800FF74191D00EB410101334988A14218BF0D
:1086D80052180A2BF5D1B0F829301344B0F82B20E2
:1086E8001A44B0F82D30B0F82F001344184410BDC8
:1086F8002DE9F04190F82F7004460D4697B30026F7
:1087080080F82F6000F2A310FFF7D6FFB4F9C1314B
:10871800D4F8A3812E60B342B8BF34464FF0640248
:1087280090FBF2F1A8BF0A222846A8BF93FBF2F4F7
:1087380009230022FFF703F8012202212046F9F756
:108748001BFB0823014609222846FEF7F8FF47F6D7
:10875800FF7141454FF00F034FF01102A8BF41468A
:10876800FEF7EDFF3846BDE8F0812DE9F04190F8BD
:10877800347004460D4697B3002680F8346000F242
:10878800D910FFF799FFB4F9F731D4F8D9812E60E1
:10879800B342B8BF34464FF0640290FBF2F1A8BF71
:1087A8000A222846A8BF93FBF2F409230022FEF709
:1087B800C6FF012202212046F9F7DEFA0823014606
:1087C80009222846FEF7BBFF47F6FF7141454FF0E7
:1087D8000F034FF01102A8BF4146FEF7B0FF38461D
:1087E800BDE8F081F0B591B00D46F22301A9044629
:1087F8001646ADF80830FFF759F838B12389ADF8B7
:108808000A30019B039301238DF8093001A9204602
:10881800FFF728FA70B19DF8093010A9062202FB6B
:108828000312218A22F8361C0133019942F8341CBC
:108838008DF8093001A92046FFF75EFA70B19DF85E
:10884800093010A9062202FB0312218D22F8361CDA
:108858000133019942F8341C8DF8093001A92046EA
:10886800FFF794FA70B19DF8093010A9062202FBAF
:108878000312618A22F8361C0133019942F8341C2C
:108888008DF8093001A92046FFF780F870B19DF8EE
:10889800093010A9062202FB0312618922F8361C4E
:1088A8000133019942F8341C8DF8093001A920469A
:1088B800FEF757FF70B19DF8093010A9062202FB98
:1088C8000312618822F8361C0133019942F8341CDE
:1088D8008DF8093001A92046FEF769FF70B19DF8AF
:1088E800093010A9062202FB0312A18822F8361CBF
:1088F8000133019942F8341C8DF809309DF809704C
:10890800082F11D801A92046FFF7F2FE60B110AA7E
:10891800062303FB0723A28923F8362C0137019A83
:1089280043F8342C8DF809709DF80970082F11D878
:1089380001A92046FFF719FF60B110AA062303FB1F
:108948000723E28A23F8362C0137019A43F8342C9E
:108958008DF809709DF80970082F11D801A92046D3
:10896800FFF786F860B110AA062303FB0723E28904
:1089780023F8362C0137019A43F8342C8DF8097006
:108988009DF80970082F11D801A92046FFF75CFA55
:1089980060B110AA062303FB0723A28A23F8362C0A
:1089A8000137019A43F8342C8DF809709DF8097045
:1089B800082F11D801A92046FEF724FF60B110AA9C
:1089C800062303FB0723E28823F8362C0137019A94
:1089D80043F8342C8DF809709DF8090050B100EB6C
:1089E800400043000233DAB2327002A9284608F088
:1089F800FBFA012011B0F0BD10B5524BD0F8D020D1
:108A08001B6894B004463AB19A1A40F6C4118A42D7
:108A180084BF012280F8CE20D4F8E0203AB19A1A17
:108A280040F6C4118A4284BF012284F8DC20D4F8BD
:108A380008213AB19A1A40F6C4118A4284BF012229
:108A480084F80721D4F810213AB19A1A40F6C411D3
:108A58008A4284BF012284F80E21D4F8EC203AB16E
:108A68009A1A40F6C4118A4284BF012284F8EA2087
:108A7800D4F818213AB19A1A40F6C4118A4284BF30
:108A8800012284F8162194F8CE2072B1002284F8CD
:108A9800CE20C4F8D03004F1BE0210232121204694
:108AA80014B0BDE81040FFF7BEBD94F8DC1041B12A
:108AB800C4F8E030082384F8DC20194604F1D40215
:108AC800EDE794F8072142B184F80711C4F808319A
:108AD80004F1F8020F230221E1E794F80E1141B1E5
:108AE80084F80E21C4F8103104F586720223072198
:108AF800D5E794F8EA2042B184F8EA10C4F8EC30DB
:108B080004F1E40206231E21C9E794F8161141B1C5
:108B180084F81621C4F8183104F58A720223092151
:108B2800BDE70DF1030201A904F58E70FFF75AFEA7
:108B380030B19DF8033001AA80212046FFF773FD6C
:108B480014B010BD8049002070B591F8205004463B
:108B58000E465DBB0846FFF7AFFD642390FBF3F0BC
:108B680040BAA4F8D400B6F91E30581C1CBF0A2518
:108B780093FBF5F56DBAA4F8D6503368591C16D096
:108B88000C4A934228BF13461A0C84F8D8201A0AB4
:108B980084F8D92084F8DA3096F923305A1C08BFB3
:108BA800002384F8DB30012384F8DC3070BD002317
:108BB800EAE700BFFFFF7F0038B50D4604460F49BE
:108BC800A868F7F7E3FFF8F7BDF940BAA4F8E4009E
:108BD80068680A49F7F7DAFFF8F7B4F940BAA4F871
:108BE800E600E8680549F7F7D1FFF8F7ABF9012384
:108BF80040BAA4F8E80084F8EA3038BD00401C46C2
:108C080010B54B681BBAC0F8F8308B681BBA4FF424
:108C18007A72C0F8FC30CB6893FBF2F31344044635
:108C280083F310035BBAA0F804314B8B5BBA11498C
:108C3800A0F80231D0F8F400F7F7A8FF0E49F8F7CA
:108C480059F8F8F7A5F940BA94F8F030A4F80001FB
:108C5800FF2B0CD094F8F120FF2A02D0934238BFA2
:108C6800134684F80631012384F8073110BD002328
:108C7800F7E700BF0000C8426666664010B50B46BD
:108C88004A68C0F8F42004460649D868F7F77EFF1A
:108C9800F8F758F9012340BAA4F80C0184F80E310A
:108CA80010BD00BF0000C84270B58A68C2F3170241
:108CB8004A2A90B004460B4600F0F48040D8212A96
:108CC80022D8172A06D8002A79D0012A00F005816F
:108CD80010B070BD183A092AFAD801A151F822F04B
:108CE800178E0008D98C0008D98C00082F8F00082F
:108CF800D98C0008D98C0008FB8D0008D98C000895
:108D0800D98C0008C78E00082A2A00F032813E2A32
:108D1800DED14D78192D01F10C0100F24E812A4661
:108D280001A808F061F901ABC5F11A020021581930
:108D380008F0F2F801A904F58E70FEF75CFCC7E7AD
:108D4800AD2A00F0588129D8932A45D01BD87C2A0F
:108D580000F08580882ABBD14D78152D01F10C01D2
:108D680000F239812A4601A808F03EF901ABC5F1A5
:108D780016020021581908F0CFF801A904F58E70E1
:108D8800FEF765FCA4E7A22AA2D101A8F9F77EFCA8
:108D980001A904F58E70FEF78FFC99E7F22A00F01E
:108DA8003381FD2A00F05481E22A91D101A8F9F714
:108DB80087FC01A904F58E70FEF795FC88E701A8E9
:108DC800F9F764FC01A92046FFF752FC01A904F554
:108DD8008E70FEF795FB7BE701A8F9F71FFC01A948
:108DE8002046FFF7B1FE01A904F58E70FEF73CFCA2
:108DF8006EE7194601A8F9F72EFC01A92046FFF7EE
:108E0800DBFE01A904F58E70FEF7B7FB60E75D781D
:108E1800332D03F10C0114D82A4601A808F0E4F810
:108E280001ABC5F134020021581908F075F89DF816
:108E3800213084F8F03001A904F58E70FEF782FB2A
:108E480046E70A4601AD3C33106851682E4603C612
:108E580008329A423546F7D110683060E7E74D7816
:108E6800382D01F10C010FD82A4601A808F0BCF8EA
:108E780001ABC5F139020021581908F04DF89DF8E9
:108E8800253084F8F13023E70A4601AD44331068F1
:108E980051682E4603C608329A423546F7D11378F0
:108EA8003370ECE701A8F9F79EFC01A92046FFF70B
:108EB800E5FE01A904F58E70FEF7AAFB08E719463E
:108EC80001A8F9F7C8FB01A92046FFF799FE01A9F7
:108ED80004F58E70FEF760FBFAE64D782A2D01F155
:108EE8000C0110D82A4601A808F07EF801ABC5F19C
:108EF8002B020021581908F00FF801A904F58E700B
:108F0800FEF712FBE4E60A4601AD343310685168F7
:108F18002E4603C608329A423546F7D1118893780F
:108F2800B3703180E9E75D781C2D03F10C0110D88E
:108F38002A4601A808F058F801ABC5F11D02002126
:108F4800581907F0E9FF01A904F58E70FEF709FB2F
:108F5800BEE60A4601AD2433106851682E4603C6A2
:108F680008329A423546F7D1106830601379337168
:108F7800E9E74D78112D01F10C0110D82A4601A816
:108F880008F032F801ABC5F112020021581907F0B8
:108F9800C3FF01A904F58E70FEF720FB98E60A4688
:108FA80001AD1C33106851682E4603C608329A4238
:108FB8003546F7D113883380EBE70A4601AD2433F1
:108FC800106851682E4603C608329A423546F7D1D2
:108FD80013883380AEE60A4601AD1C331068516829
:108FE8002E4603C608329A423546F7D110683060DB
:108FF8009388B380C1E601A8F9F762FB01A904F5DB
:109008008E70FEF766FB63E64D783B2D01F10C018F
:1090180010D82A4601A807F0E7FF01ABC5F13C02CA
:109028000021581907F078FF01A904F58E70FEF7A2
:1090380064FB4DE60A4601AD4433106851682E467C
:1090480003C608329A423546F7D110683060EBE71C
:1090580001A8F9F7E3FA01A904F58E70FEF75EFBA3
:1090680036E600BF4A7922B18B79012B01D1FFF78F
:109078001BBE7047B0F5E16F03DC10F5E16F04DB50
:109088007047A0F5616000B2F4E700F5616000B2D6
:10909800F3E7000038B5B0F8F8330D4613F00801CF
:1090A800AA8808BFC0F8081113F0020308BFC0F867
:1090B8001831B2F5005F044600F0B28007D86C2A78
:1090C80017D06D2A00F08F806A2A60D038BD42F22E
:1090D80002039A423BD042F6FF739A42F6D1D0F887
:1090E800FC23A968BE30FEF793F9012384F8CE303B
:1090F800ECE7B5F90A00FFF7BDFFF7F7F3FC4C49B9
:10910800F7F744FDF7F71EFF40BAA4F8E400B5F9F5
:109118000800FFF7AFFFF7F7E5FC4549F7F736FD1D
:10912800F7F710FF40BAA4F8E600B5F90C00FFF70E
:10913800A1FFF7F7D7FC3F49F7F728FDF7F702FF3C
:10914800012340BAA4F8E80084F8EA30BEE7B5F88D
:1091580009300A22B3FBF2F35BBAA0F8D430B5F8B1
:109168000B30B3FBF2F35BBAA0F8D630D5F8113068
:1091780080F8DA301A0C80F8D8201A0A80F8D9203A
:109188006B7F80F8DB30012380F8DC309EE7002914
:109198009CD0D5F80A301BBAC0F8F830D5F80E3094
:1091A8001BBAC0F8FC30AB8A242253433233642202
:1091B800B3FBF2F35BBAA0F80031EB8A0A214B4308
:1091C8005BBAA0F80231D0F8F43393FBF2F303F55D
:1091D8007A735BBAA0F804316B7A80F80631012300
:1091E80080F8073172E7B5F90C2052BAA0F80C21C3
:1091F800012280F80E21002B3FF468AFD5F80E103D
:109208000A2391FBF3F303F51C53103383F30F0385
:109218005BBAA0F81431C0F8F41380F8072155E7B9
:10922800AB89A0F8F833D5F81130C0F8FC334DE716
:1092380058A08B416E882E4330B5204C85B005462A
:1092480094F99200F8F7D8F900238DF805308DF8D5
:10925800073094F895308DF80830194B94F893201E
:109268008DF8040098788DF80620F8F7B5F98DF890
:1092780009001448FBF709FBF8F788F98DF80A008C
:109288002046F8F7F6F8F8F7B7F98DF80B002046FE
:10929800F8F701F98DF80C002046F8F7F3F88DF887
:1092A8000D002046F8F708F90A238DF8050001AAF1
:1092B80014212846FFF7B7F905B030BDB42F0020B8
:1092C800C40200205C30002073B5184C05462046C7
:1092D800F8F7CFF8F8F790F98DF800002046F8F77E
:1092E800C8F806461248FBF7B9FA01463046F8F7BF
:1092F8008DF98DF801002046F8F7CDF88DF80200B9
:109308002046F8F7BFF8FF238DF80430094B8DF895
:1093180003009878F8F768F906238DF805006A467F
:109328001D212846FFF77FF902B070BDB42F002039
:109338005C300020C4020020F7B5144D144E0446DA
:1093480095F99200F8F758F98DF80000304695F92C
:109358009270FBF783FA01463846F8F757F995F803
:1093680093308DF801008DF80230304600238DF8D7
:109378000330FBF78AFA05238DF804006A461C219E
:109388002046FFF750F903B0F0BD00BFB42F00200E
:109398005C30002030B591B04EF6EA631A49ADF85A
:1093A8000030044614220DF10200F8F70DFB0DF110
:1093B8000200F6F7E7FEC3B2DA1CD0B2694651FAEA
:1093C80082F26D250DF800504C205070522090709C
:1093D8005320D070312010716FF02B005071012094
:1093E8005072032000219072113306209171D171BF
:1093F8001172D07211735173DBB26A46292120466B
:10940800FFF711F911B030BD321901080038024BCD
:1094180018BF012018707047740500202DE9F0412D
:10942800002A4AD1042B00F2A1809EB2002B42D020
:109438004D4C4FF0800EFF250F8894F81EC0C35D79
:1094480023EA0C03C355A37F01325B081FFA82FC91
:10945800A3773BB90B8801330B8084F81EE00B8897
:10946800C554A37FB1F8008010F8087027EA0303F9
:1094780000F80830A37F5B08A3773BB90B8801335A
:109488000B8084F81EE00B88C554A37FB1F80080D8
:1094980010F8087027EA030300F80830A37F5B0878
:1094A800A37733B90B8801330B8084F81EE00B884F
:1094B800C5546645C0D8BDE8F081FF2AFBD1032B0F
:1094C80000F249819FB2002BF5D0274C0025802659
:1094D800B1F800C094F81EE010F80C3023EA0E032F
:1094E80000F80C30A37F01355B081FFA85FCA377D1
:1094F80033B90B8801330B80A6770B88C254A37F3E
:10950800B1F8008010F808E02EEA030300F80830EC
:10951800A37F5B08A37733B90B8801330B80A67749
:109528000B88C254A37F5B08A37733B90B88013338
:109538000B80A6770B88C254A37FB1F8008010F87F
:1095480008E02EEA030300F80830A37F5B08A3773E
:109558002BB90B8801330B80A6770B88C25467455B
:10956800B6D8BDE8F08100BFA40C00200D889A4C45
:10957800425DA67F22EA06024255A27F520803F501
:10958800C063A2773AB90A8801320A808022A2779A
:109598000A88FF2585540D88A67F425D22EA0602C7
:1095A8004255A27F5208A2773AB90A8801320A8046
:1095B8008022A2770A88FF258554A27F5208A277C5
:1095C8003AB90A8801320A808022A2770A88FF25E0
:1095D8008554A27F5208A2773AB90A8801320A80D4
:1095E8008022A2770A88FF2585540D88A67F425DD0
:1095F80022EA06024255A27F5208A2773AB90A889F
:1096080001320A808022A2770A88FF2585541E0627
:1096180005D40D88A67F425D22EA06024255A27F44
:109628005208A2773AB90A8801320A808022A277C2
:109638000A88FF2585545D0605D40D88A67F425DFE
:1096480022EA06024255A27F5208A2773AB90A884E
:1096580001320A808022A2770A88FF2585549A065B
:1096680005D40D88A67F425D22EA06024255A27FF4
:109678005208A2773AB90A8801320A808022A27772
:109688000A88FF258554DF0605D40D88A67F425D2C
:1096980022EA06024255A27F5208A2773AB90A88FE
:1096A80001320A808022A2770A88FF2585541E0786
:1096B80005D40D88A67F425D22EA06024255A27FA4
:1096C8005208A2773AB90A8801320A808022A27722
:1096D8000A88FF2585545D0705D40D88A67F425D5D
:1096E80022EA06024255A27F5208A2773AB90A88AE
:1096F80001320A808022A2770A88FF2585549A07BA
:1097080005D40D88A67F425D22EA06024255A27F53
:109718005208A2773AB90A8801320A808022A277D1
:109728000A88FF258554DB0705D40A88A57F835C52
:1097380023EA05038354A37F5B08A377002B7FF4F8
:10974800BAAE0B88802201330B80A2770B88FF22E8
:10975800C254BDE8F0810E881F4C855DA77F25EABD
:1097680007058555A57F6D0803F5E063A57735B92D
:109778000D8801350D808025A5770D8842550D8807
:10978800A67F425D22EA06024255A27F5208A277CE
:109798003AB90A8801320A808022A2770A88FF250E
:1097A8008554A27F5208A2773AB90A8801320A8002
:1097B8008022A2770A88FF258554A27F5208A277C3
:1097C800002A7FF418AF0A8801320A808022A27723
:1097D8000A88FF2585540EE7A40C00202DE9F047E0
:1097E8009C4C802500270F80A577FF25057098469B
:1097F800002B00F02C8103F1FF3912FA89F9561E6B
:10980800BA463B460BE0554540F0C0800137BFB231
:109818000A88424580F0B3804E4500F0078116F86B
:10982800015F002BEFD16B1EDBB2FD2B00F2AA808B
:109838003F2B40F2E18005F14103DBB23F2B00F200
:10984800AC80A37F01355B08EDB2A377002B00F055
:10985800E4805B08A37743B90B8801330B8080232E
:10986800A3770B88FF22C254A37FAA0608D4B1F8B5
:1098780000C010F80C2022EA030300F80C30A37F84
:109888005B08A37743B90B8801330B808023A37748
:109898000B88FF22C254A37FEA0608D4B1F800C09F
:1098A80010F80C2022EA030300F80C30A37F5B08B1
:1098B800A37743B90B8801330B808023A3770B88E8
:1098C800FF22C254A37F2A0708D4B1F800C010F8B9
:1098D8000C2022EA030300F80C30A37F5B08A3776F
:1098E80043B90B8801330B808023A3770B88FF22B1
:1098F800C254A37F6A0708D4B1F800C010F80C203E
:1099080022EA030300F80C30A37F5B08A37743B96E
:109918000B8801330B808023A3770B88FF22C25466
:10992800A37FAA0708D4B1F800C010F80C2022EAD7
:10993800030300F80C30A37F5B08A37743B90B88B7
:1099480001330B808023A3770B88FF22C254A37FA7
:10995800EA0705D40D88425D22EA03034355A37F35
:109968005B08A377BBB90A8801320A808022A277F4
:109978000A88FF2585540A884245FFF44DAF002028
:10998800BDE8F0870127AA463B4641E7FBB25246AD
:10999800FFF744FD47E700233AE70A8894F81EC01A
:1099A800835C23EA0C038354A37F3F355B08EDB245
:1099B800A37743B90B8801330B808023A3770B88E7
:1099C800FF22C254A37F5B08A37743B90B880133F6
:1099D8000B808023A3770B88FF22C254A37F6A06DB
:1099E8003FF537AFB1F800C010F80C2022EA0303A6
:1099F80000F80C30A37F2CE7A37F7F355B08EDB21E
:109A0800A377002BEED10B8801330B808023A3773B
:109A18000B88FF22C254A37FE4E70B8801330B8035
:109A28008023A3770B88FF22C254E3E75BB9A37FA7
:109A3800802B1EBF013292B20A80904594BF00204D
:109A48000120BDE8F087FBB25246FFF7E7FC0A8821
:109A5800EDE700BFA40C00202DE9F04F47F26F732B
:109A68000022827003800B78A3F1FE03B3FA83F31C
:109A78005B0983708A780D4612F001011CBF43F020
:109A880080038370D5F8202122F07F4222F0FF0264
:109A980085B0044612B143F008038370AA68C2F384
:109AA8001702FF2A1ED9B2F5803F18D363F07F034F
:109AB800A37041F002014FF0020B09234FF00A0C8A
:109AC8000822E1700B20CDF804C01E4617464FF05F
:109AD800070E4FF006094FF0050A042117E043F07E
:109AE8000203A370180600F1D68008234FF0090C72
:109AF80007220A204FF0000BCDF804C01E46174677
:109B08004FF0060E4FF005094FF0040A032195F8AF
:109B1800018004F8018004EB0108297904F80A108F
:109B2800697904F80910A97904F80E10A1780907D1
:109B380009D595F82111A15495F82211A15503468C
:109B4800674662460646A968A154A278900707D5D9
:109B5800BA1C1F46AB68C3F30F23A35596B233460E
:109B6800BBF1000F05D05A1C1F46AB7AA35596B21D
:109B78003346A278D10606D55A1C1F4695F82331DC
:109B8800A35596B23346454A127803F1010914FAEF
:109B980089FA05F10C0B42B16B785A460DF10E01AA
:109BA8005046FFF71BFE00285AD16A78504659469E
:109BB8001FFA82FA07F018FA2278394B6178D243F3
:109BC800D2B2072F9A5C82EA0102995CA27882EAF3
:109BD8000102995CE27882EA0102995C227982EAC0
:109BE8000102995C627982EA0102995CA27982EAAF
:109BF8000102995CE27982EA0102995C1BD0227A1F
:109C08005140082F595C16D0627A5140092F595C8F
:109C180011D0A27A51400A2F595C0CD0E27A5140F7
:109C28000B2F595C07D0227B51400C2F595C1EBF6B
:109C3800627B5140595CA1551AFA89F39BB2B5F879
:109C48000C21E2545A1CB5F80C1192B2090AA1541D
:109C5800AA78981CD20780B20BD405B0BDE8F08F63
:109C6800A378BDF80EA043F04003A37088F800A0C5
:109C7800A2E7D5F81071D5F81811D5F81461275056
:109C880022180F335660916095F81C11117398B221
:109C980005B0BDE8F08F4FF0000B0EE7740500200B
:109CA800842B01082DE9F04F944D0C4683B00146F2
:109CB80007462846164607F097F9914A0023802060
:109CC8002380138482F82200002E00F0CD8095F8BE
:109CD80000C04FF0400B4FEADC1C82F822B09E46D1
:109CE8004FF0FF0892F8229015F803A04FEA4C0CA9
:109CF8001AEA090F4FEA590118BF4CF0010C82F813
:109D08002210002900F0B380BCF1020F00F0448457
:109D1800BCF1030F00F0DF83BCF1010F40F0BA8003
:109D28009E4240F2A18015F8039019EA010F14BF72
:109D38004FF0010C4FF0000C5FEA510A40F0B68377
:109D480001339BB29E42138482F8220040F28C8039
:109D5800E95600294FEA4C0C01DA4CF0010C82F864
:109D680022B0402100919E427ED9009915F80390B7
:109D78004FEA4C0C19EA010F00995FFA8CFC18BFE6
:109D88004CF0010C5FEA510A40F0268401339BB283
:109D98009E42138482F8220066D94FEA4C0115F9D5
:109DA80003C015F80390BCF1000FC9B201DA41F005
:109DB80001014FEA410C19F0400F5FFA8CFC18BF03
:109DC800202100F09F854CF0010C002940F09B8574
:109DD80001339BB29E42138482F8220044D915F9BC
:109DE80003904FEA4C0CB9F1000F5FFA8CF115F8AB
:109DF80003C001DA41F0010149001CF0400FC9B26B
:109E080018BF4FF0200A00F0B98541F0010182F82F
:109E180022A0BAF1000F03D10133138482F8220083
:109E28007D2921D84131238803F1010CA4F800C011
:109E3800F954138C9E4217D992F8221015F803C0D2
:109E480011EA0C0F4FEA510114BF4FF0010C4FF00B
:109E5800000C82F8221021B901339BB2138482F8D6
:109E680022009E423FF63EAF03B0BDE8F08F0133BB
:109E78009BB2BCF1020F138482F8220000F0AD817E
:109E8800BCF1030F00F03482BCF1010F4FF08001E8
:109E98003FF446AF9E42E7D915F803C011EA0C0F0C
:109EA8001ED05FEA51092DD101339BB29E42138423
:109EB80082F82200D8D9E9560029C0F2E8804FF08C
:109EC80080094FEA590182F8221019B90133138425
:109ED80082F822002388591C218007F80380A8E70C
:109EE800490882F8221019B90133138482F8220034
:109EF8002388591C218007F803E09AE7780B002093
:109F0800A40C002019EA0C0FDBD0890840F0C080AF
:109F180001339BB29E42138482F82200A4D9E956E9
:109F28000029C0F2668280215FEA510C40F041822C
:109F380001339BB29E42138482F8220094D9E95CD3
:109F48004FEAD11C49064FEA4C0C40F1BD84202150
:109F58004CF0010C82F8221029B901339BB213840A
:109F680082F8220080219E427FF67EAF15F803908A
:109F78004FEA4C0C11EA090F5FFA8CFC18BF4CF041
:109F8800010C490840F06E8301339BB29E42138452
:109F980082F822007FF668AFE9564FEA4C0C002998
:109FA8005FFA8CFC80F2318480215FEA51094CF021
:109FB800010C40F0658301339BB29E42138482F802
:109FC80022007FF651AF4FEA4C0115F903C0BCF1EE
:109FD800000FC9B280F225844FF080095FEA590961
:109FE80041F0010140F0598301339BB29E42138432
:109FF80082F822007FF638AF15F903C04900BCF19A
:10A00800000FC9B280F226844FF080095FEA59092F
:10A0180041F0010140F04D8301339BB29E4213840D
:10A0280082F822007FF620AF15F903C04900BCF181
:10A03800000FC9B2C0F211844FF0400915F803C0EF
:10A04800490019EA0C0FC9B200F052834FEA5909C6
:10A0580041F0010182F82290B9F1000F40F0048428
:10A0680001339BB2138482F822001FFA81FC002975
:10A078003FF4E0AE00232188013301F10109A4F87F
:10A08800009007F801E099B26145F4D3D1E6402188
:10A0980015F803C011EA0C0F3FF446AF490840F029
:10A0A800A98101339BB29E42138482F822007FF675
:10A0B800DBAE15F803904FEAD91C19F0400F4FEAB0
:10A0C8004C0C00F0F58320214CF0010C002940F0E5
:10A0D800F08301339BB29E42138482F822007FF6FC
:10A0E800C3AE4FEA4C0C5FFA8CF115F903C015F8B2
:10A0F8000390BCF1000F01DA41F00101490019F0A9
:10A10800400FC9B218BF4FF0200C00F02C8441F06A
:10A118000101BCF1000F40F0288401339BB29E423C
:10A12800138482F822007FF69FAE15F903C0490018
:10A13800BCF1000FC9B201DA41F0010182F822B086
:10A148004FF0400A9E427FF68FAE15F803C04900D3
:10A158001AEA0C0FC9B218BF41F001015FEA5A0CA4
:10A1680040F0D58201339BB29E42138482F82200CC
:10A178007FF67AAE15F903C04900BCF1000FC9B2E9
:10A18800C0F275834FF0400C15F8039049001CEAA3
:10A19800090FC9B200F0DA824FEA5C0C41F0010104
:10A1A80082F822C0BCF1000F40F0688301339BB2F3
:10A1B800138482F822001FFA81FC00293FF43AAE8A
:10A1C80000232188013301F10109A4F8009007F860
:10A1D800018099B28C45F4D82BE69E427FF644AEB6
:10A1E800E95C4FF04009C909B2F820C04B0015F8E6
:10A1F8000C1019EA010F4FEA590A01D043F0010384
:10A20800BAF1000F40F0B1820CF1010C1FFA8CFC7E
:10A218006645A2F820C082F822007FF625AE15F91F
:10A228000C905900B9F1000FC9B280F2DC824023CA
:10A2380041F00101002B40F0A5820CF1010C1FFA3E
:10A248008CFC6645A2F820C082F822007FF60CAE8E
:10A2580015F90C304FEA4109002B5FFA89F980F2B1
:10A26800CB82402149F00109002940F09A820CF183
:10A27800010C1FFA8CFC6645A2F820C082F8220067
:10A288007FF6F2AD15F90C104FEA49030029DBB24D
:10A2980080F2BE824FF0400943F00103B9F1000F8C
:10A2A80040F08E820CF1010C1FFA8CFC6645A2F876
:10A2B80020C082F822007FF6D7AD15F90C105B009C
:10A2C8000029DBB280F2C382402143F0010382F807
:10A2D800221029B90CF1010CA2F820C082F8220042
:10A2E8002188013301F1010CA4F800C07B54A0E5DA
:10A2F8009E427FF6B9AD15F803C04FF040094FEA0A
:10A30800DC111CEA090F4FEA41014FEA590A01D052
:10A3180041F00101BAF1000F40F0368301339BB2DE
:10A328009E42138482F822007FF69EAD15F90390B1
:10A3380015F803C04900B9F1000FC9B201DA41F0BC
:10A34800010149001CF0400FC9B218BF4FF0200AA4
:10A3580000F0F18241F00101BAF1000F40F0ED8206
:10A3680001339BB29E42138482F822007FF67CADB3
:10A3780015F9039015F803C04900B9F1000FC9B2E7
:10A3880001DA41F0010149001CF0400FC9B218BFC1
:10A398004FF0200A00F0DA8241F0010182F822A091
:10A3A800BAF1000F03D10133138482F82200413936
:10A3B80039E515F8039019EA0C0F14BF4FF0010C9A
:10A3C8004FF0000C5FEA910A40F0378201339BB2EC
:10A3D8009E42138482F822007FF646ADE956002992
:10A3E8004FEA4C0C01DA4CF0010C82F822B0402103
:10A3F800B9E5402115F8039019EA010F14BF4FF091
:10A40800010C4FF0000C5FEA510A40F00D82013355
:10A418009BB29E42138482F822007FF625ADE9564E
:10A4280015F8039000294FEA4C0C01DA4CF0010CA6
:10A438004FEA4C0C19F0400F5FFA8CFC18BF4FF034
:10A44800200A00F048824CF0010CBAF1000F40F0ED
:10A45800448201339BB29E42138482F822007FF625
:10A4680003AD15F903904FEA4C01B9F1000F15F847
:10A4780003C0C9B201DA41F0010149001CF0400FE4
:10A48800C9B218BF4FF0200A00F0658241F00101FF
:10A4980082F822A0BAF1000F7FF454AE01339BB2C8
:10A4A800138482F822004FF0800A4BE6890819EAE3
:10A4B8000A0F00914FEA4C0C01D04CF0010C82F8C5
:10A4C800221000297FF44FAC01339BB2138482F829
:10A4D8002200802146E415F803C01CEA010F14BFCE
:10A4E800012100215FEA99097FF40BAF01339BB288
:10A4F8009E42138482F822007FF6B6AC15F90390C9
:10A5080015F803C0B9F1000F4FEA410101DA41F033
:10A5180001011CF0400F4FEA410118BF4FF020091C
:10A5280000F0BB8141F00101B9F1000F40F0B781A3
:10A5380001339BB29E42138482F822007FF694ACCA
:10A5480015F9039015F803C04900B9F1000FC9B215
:10A5580001DA41F0010149001CF0400FC9B218BFEF
:10A568004FF0200900F0C38141F00101B9F1000F5B
:10A5780040F0BF8101339BB29E42138482F82200CF
:10A588007FF672ACEB564900002BC9B201DA41F0F4
:10A59800010182F822B00AE792F8229019EA0A0F1C
:10A5A80014BF012100215FEA59097FF41DAE013370
:10A5B8001FFA83FC6645A2F820C082F822007FF6C5
:10A5C80053AC15F90C90B9F1000F4FEA410380F232
:10A5D80002814FF0400A11E64FEA4C0C890819EA4B
:10A5E8000A0F5FFA8CFC019101D04CF0010C002994
:10A5F80040F0D38101339BB29E42138482F822003B
:10A608007FF632AC4FEA4C0115F903C015F80390F8
:10A61800BCF1000FC9B201DA41F00101490019F09B
:10A62800400F5FFA81FA18BF4FF0200C00F07681D6
:10A638004AF0010ABCF1000F40F0728101339BB26D
:10A648009E42138482F822007FF60EACEB564FEA46
:10A658004A01002BC9B201DA41F0010182F822B0A7
:10A66800FFF7DEBB15F803904FEA4C0C11EA090F0F
:10A678005FFA8CFC7FF499AC5FEA51093FF49BAC1C
:10A688004FEA4C0115F803C019EA0C0FC9B27FF460
:10A69800A5AC5FEA59093FF4A7AC15F803C0490017
:10A6A80019EA0C0FC9B27FF4B1AC5FEA59093FF45B
:10A6B800B3AC15F803C0490019EA0C0FC9B201D0B0
:10A6C80041F001015FEA59097FF4B8AC01339BB24C
:10A6D8009E42138482F822007FF6C6AB15F903C0A8
:10A6E8004900BCF1000FC9B2C0F2BA804FF080092E
:10A6F8004FEA590982F82290B9F1000F3FF4B0AC43
:10A708001FFA81FC00297FF4B5ACFFF795BB15F85B
:10A71800039049001CEA090FC9B201D041F00101B8
:10A728005FEA5C0C7FF430AD01339BB29E42138428
:10A7380082F822007FF698AB15F903C04900BCF1F6
:10A74800000FC9B2C0F296804FF0800C4FEA5C0C43
:10A7580082F822C0BCF1000F3FF428AD1FFA81FC3B
:10A7680000297FF42DADFFF767BB15F80C90590051
:10A778001AEA090FC9B24FEA5A037FF459AD002B00
:10A788003FF45BAD15F80CA04FEA410913EA0A0F34
:10A798005FFA89F94FEA53017FF464AD00293FF469
:10A7A80066AD15F80CA04FEA490311EA0A0FDBB2AF
:10A7B8004FEA51097FF470ADB9F1000F3FF472AD63
:10A7C80015F80CA05B0019EA0A0FDBB24FEA590131
:10A7D8003FF47DAD79E515F80C305B064FEA810151
:10A7E8004FD5202324E59B005FFA83F915F80C3038
:10A7F800590648D5202135E58900CBB215F80C104B
:10A80800490642D54FF0200946E54FF0400937E7A1
:10A8180015F80C104FEA89034906DBB238D5202118
:10A8280053E54FF0400938E719EA0A0F4FEA91015A
:10A838004FEA4C0C3FF44AAC46E419EA0A0F4FEAD7
:10A84800D1014FEA4C0C3FF485ABFFF781BB82F88E
:10A8580022B045E54FF040092BE74FF080092FE77C
:10A8680041F0010182F822B01FFA81FC02E44FF0A6
:10A87800800C53E741F0010182F822B01FFA81FCF5
:10A888009EE420237EE720218BE74FF0200997E7FD
:10A898004FF0200182F8221022E54FF020094900EC
:10A8A80019EA0C0FC9B24FEA590A3FF455AD51E500
:10A8B80020214FEA4C0C19EA010F5FFA8CFC4FEA91
:10A8C800510A3FF4C2ADBEE54FF0200182F82210D4
:10A8D8002021FFF748BB4FF0200A4FEA4C0119EA44
:10A8E8000A0FC9B24FEA5A0C3FF413AC0FE44FF009
:10A8F8002009490019EA0C0FC9B24FEA590A3FF476
:10A908004DAD49E520214FEA4C0C11EA090F5FFAD9
:10A918008CFA4FEA510C3FF48DAE89E64FF0200CCB
:10A928004FEA4A0119EA0C0FC9B24FEA5C0A3FF430
:10A938006EAAFFF76ABA4FF0200A49001AEA0C0F0C
:10A94800C9B24FEA5A093FF411AE0DE64FF02003A1
:10A9580082F822302BE54FF0200C82F822C04FF00D
:10A96800200AFFF7EFBB4FF0200C490019EA0C0F43
:10A97800C9B24FEA5C0A3FF48BAD87E54FF020037C
:10A9880082F82230FFF74CBA49001AEA0C0F4FEA56
:10A998009909C9B23FF4C8ADC4E58A4600994FEA9F
:10A9A8004C0C19EA0A0F4FEAD1015FFA8CFC3FF40C
:10A9B8000CAAFFF708BA00BF2DE9F04F5788B7F582
:10A9C8008F7F8BB0144606460BD9002222700022D6
:10A9D8006F2B628000F06581002333700BB0BDE8F7
:10A9E800F08F12780E2A0D4624D80E2A00F2118113
:10A9F80001A151F822F000BFD7A9000827AC000830
:10AA08001BAC00081BAC000827AC000827AC0008EA
:10AA180027AC000827AC000827AC000827AC0008C2
:10AA280075AC00081BAC00081BAC00081BAC000888
:10AA380099AC0008692A40F2EA806A2A40F0E98065
:10AA48009C4FFA8A02F1FF3C1FFA8CFC002A00F0A6
:10AA580078820CF1030CDFF860E2BC44FF22B91CD9
:10AA680011F8010B424061451EF80220F8D19342CB
:10AA780000F0D08100222270C4F80220E280FA8A15
:10AA8800022AA9D939796F2900F02E83032AA3D085
:10AA980079796F2900F03883042A9DD0B9796F2914
:10AAA80000F03583052A97D0F9796F2900F03E83A5
:10AAB800062A91D0397A6F2900F04582072A8BD06F
:10AAC800797A6F2900F03583082A85D0B97A6F29F9
:10AAD80000F03283092A3FF47FAFF97A6F2900F03A
:10AAE8002E830A2A3FF478AF397B6F2900F02A8336
:10AAF8000B2A3FF471AF797B6F2900F026830C2A6B
:10AB08003FF46AAFB97B6F2900F022830D2A3FF426
:10AB180063AFF97B6F2900F01E830E2A3FF45CAF08
:10AB2800397C6F2900F01D830F2A3FF455AF797CDB
:10AB38006F2900F01383102A3FF44EAFB97C6F29B8
:10AB480000F01283112A3FF447AFF97C6F2900F017
:10AB58000E83122A3FF440AF397D6F2908BF4FF0AA
:10AB680012087FF439AF02F101091FFA89F93A4452
:10AB7800A7F816905FFA89F9937050494A4602A8D7
:10AB880006F032FA6F234FF0010CBB704FF0000E45
:10AB98006423A7F800E0A7F816C0237008EB0C039D
:10ABA80099451FFA89F27FF617AF901E02A9A0EB0C
:10ABB80008005A1E0B440A4413FA80F04FF06A0842
:10ABC8004FF007094FF0660A05E0002B40F0BE8100
:10ABD80090423FF401AFFB8A12F8011F07EB030B09
:10ABE80001338BF80210FB822378092BEDD9A3F1EE
:10ABF800640BBBF1050FEBD8653B042B00F2BA825E
:10AC0800DFE813F01F01170112010E011B01632A6F
:10AC180005D800232370C4F80230E380DDE6254F11
:10AC2800FA8AB91801328B70FA822278092A00F25E
:10AC3800A480002A3FF4D0AE013A082A3FF6CCAEF1
:10AC480001A151F822F000BF11AF0008E1A90008E6
:10AC5800E1A9000873AE000873AE0008FBAE000857
:10AC6800C7AE000835AF0008E5AE00087A1C628060
:10AC7800104EEB55A088727F618883189942FFF6C1
:10AC8800ADAE33785F0600F1E4810E232370A5E6AC
:10AC98007A1C6280EB55E2886388934210D20123C4
:10ACA8009BE604490A800122CA8264228B702270C2
:10ACB800002392E6A40C0020842B0108A60C002097
:10ACC8000023638023700223037042802B78FD2BBE
:10ACD80000F08780EB7803722B7943726B794360BD
:10ACE8006A780832728000224FF4BC70DFF8CCC258
:10ACF8007281F6210446013499424FEA54042ED851
:10AD080049D38B4240F08A802B78FD2B7FD04FF0BF
:10AD1800060B2846DFF8A48210F801AF0BEB0A09EE
:10AD280009F1FF3189B2F7F705FB04EB440708EB9B
:10AD38008707ADF808003979019102A8F7F7D6FA24
:10AD480005EB090215F809305278019903EB022343
:10AD5800BDF808209BB29A421FD005233DE6601E2D
:10AD68001418824204F1010780F06C8127F0010178
:10AD780001EB57015CF82110BDE7A2F16401052938
:10AD88003FF62AAE653A042A00F2FD81DFE802F0B8
:10AD9800817D797593002246E2E7BB79DA0706D50B
:10ADA800FA79924582BF521912F80B20B2729B07AA
:10ADB8000BD56300234408EB83036A781B7A9A4215
:10ADC80082BF5B1913F80B30F3724FEA4409A144B0
:10ADD80008EB8908317398F8053073730BB0BDE838
:10ADE800F08F6B790372AB7943726B7A297AEA79BF
:10ADF8001B0403EB0123134443606A7802F10C013E
:10AE08004180A978C9077FF56EAF19326AE74FF01C
:10AE18000A0B7EE70A2201232270DEE50323DCE524
:10AE2800F97684F80090D3E64FF06803B97623707A
:10AE3800CEE6797084F800C0CAE6397784F80080D5
:10AE4800C6E6397001F00103618887F801E0033B29
:10AE580001F1010BA4F802B06B5497F90030002BF4
:10AE6800ACBF634653462370B2E66288511C6180CA
:10AE7800AB54237801332370AEE50722FB762270AA
:10AE880016E76822BB76227012E701227B702270D7
:10AE98000EE762883B70002103F00103033B7970E1
:10AEA800511C6180AB5497F90030002BC0F23281FD
:10AEB8000123237090E56A223B772270F8E66288C6
:10AEC800511C6180AB543B787A78134313F002032A
:10AED80040F0D7806288511C6180AB546288511C55
:10AEE8006180AB543B78D8064CBF69236A23237032
:10AEF80072E56288511C6180AB543B781D074CBFDA
:10AF080067230723237067E562883A83511C6180B1
:10AF1800AB543A787B7712F0010200F0D080062219
:10AF28000833A280E3800423237055E56288511C0E
:10AF38006180AB547B7813F00203CFD009232370D0
:10AF48004AE5FF2293E54FF006080CE6013B082B83
:10AF58003FF63EAE0FF2040B5BF823F09DAF0008FE
:10AF6800D9AB0008D9AB000889AF000889AF000841
:10AF780017B00008E5AF000831B00008C9AF0008F5
:10AF8800638803F1010BA4F802B0E9542378013374
:10AF980023701DE663883B8303F1010BA4F802B01C
:10AFA800E9543B78797713F001036DD00831062313
:10AFB800E180A380042323700AE600BF842C0108E3
:10AFC800638803F1010BA4F802B0E9543B78DB066F
:10AFD8007FF534AF4FF069032370F9E5638803F117
:10AFE800010BA4F802B0E9543B7879780B4313F0CD
:10AFF800020343D1618801F1010BA4F802B06B543C
:10B00800618801F1010BA4F802B06B54DEE7638894
:10B0180003F1010BA4F802B0E9543B7819077FF556
:10B0280000AF67232370D3E5638803F1010BA4F80D
:10B0380002B0E9547B7813F00203E1D04FF0090322
:10B048002370C5E5574902EB4200144651F8201019
:10B0580057E602A92844FEF725FE737FBDF80810BD
:10B068006288CB1A9BB21A446280727F1A44727744
:10B07800E2881344E380338BE95406E608232370FF
:10B08800A6E508232370A7E40C31E18079784FF016
:10B098000A0B11F00101A4F804B028D0618801F16D
:10B0A800010BA4F802B005F801C0618801F1010B99
:10B0B800A4F802B06B54E3880D33E3807AE779781B
:10B0C8000C33E38011F001014FF00A03A38024D070
:10B0D8006388012158186080E95463885918618091
:10B0E800EA54E3880D331DE74FF002083BE5638817
:10B0F80003F1010BA4F802B0E954638803F1010BD2
:10B10800A4F802B0E95455E74FF003082BE54FF0D7
:10B11800040828E5662323705EE463885A1C62806D
:10B12800E95463885A1C6280E954FCE64FF005082C
:10B1380019E54FF0070816E54FF0080813E54FF03A
:10B14800090810E54FF00A080DE54FF00B080AE56D
:10B158004FF00C0807E54FF00D0804E54FF00F0815
:10B1680001E54FF00E08FEE44FF01008FBE44FF045
:10B178001108F8E477290ED084F800E0C4F802E05A
:10B18800A4F806E024E5772B09D000232370C4F83F
:10B198000230E38020E44FF06503237018E565234F
:10B1A800237019E4842C010870B500F5EF66044695
:10B1B80000F5CA613046F7F7E2F90546A06803686A
:10B1C8002A461B6931469847E06830B103682A4629
:10B1D80031461B69BDE87040184770BD08B5034685
:10B1E800806840B1B3F84C14B3F84A04F7F79AFCF6
:10B1F800003818BF012008BD0346806880B1B3F845
:10B208004C24B3F84A14914209D09918013291F8A4
:10B218005004B3F84E140A40A3F84C247047002099
:10B228007047836810B504467BB10023A0F84C34FE
:10B23800A0F84A34C06810B10368DB699847A06871
:10B248000368BDE81040DB69184710BDF8B5224F08
:10B2580004463846F6F70DF9F6F765F9064697F904
:10B268009200F6F760F905463846F6F70BF96423BD
:10B2780084F86236FF2384F86436332384F855361D
:10B28800442384F85636D4F8583684F860666D221C
:10B2980062F31703C4F85836C0F10A000023C4F853
:10B2A8005C3684F8713700B24FF43943A4F872372A
:10B2B80080F30700092384F8630684F8615604F5CF
:10B2C800CA6084F8743704F5A471F7F7B1FC204616
:10B2D800BDE8F840FFF768BFB42F002010B533234E
:10B2E80080F85536442380F85636D0F85836144A34
:10B2F800C0F860266FF31703C0F85836002380F8AB
:10B308005C3680F85D3680F85E3680F85F3680F807
:10B3180071374FF44853A0F87237032209230446C3
:10B3280080F8642680F8743700F5A47100F5CA60C7
:10B33800F7F77EFC2046BDE81040FFF735BF00BF99
:10B348000008800470B586B004460021102202A8C7
:10B35800019105F0E1FD01AB03CB01ABC4F8800618
:10B36800C4F8841603CB01ABC4F88806C4F88C165D
:10B3780003CB04F5D362C4F89006C4F8941601AB65
:10B3880005AE1D4603CDB542106051602B4602F153
:10B398000802F6D12B881380332384F855364423CA
:10B3A80084F85636D4F85836942262F317031021DD
:10B3B8004222C4F8583684F85C16002384F86C26B8
:10B3C8002021282284F85D1684F85E3684F85F36DA
:10B3D80084F8603684F8613684F8623684F8633617
:10B3E80084F8643684F8653684F8663684F86736F7
:10B3F80084F8683684F8693684F86A3684F86B36D7
:10B4080084F86D2684F86E3684F86F3684F87036C2
:10B4180084F8713684F8723684F8733684F8743692
:10B4280084F8753684F8763684F8773684F8783672
:10B4380084F8793684F87A3684F87B3684F871375C
:10B448004FF43243094AA4F872374E2304F5CA6010
:10B45800C4F87C2684F8743704F5A471F7F7E8FB80
:10B46800204606B0BDE87040FFF79EBED016CB0F51
:10B4780010B504469DF8080084F85E26002284F87A
:10B488005F2684F8602684F8612684F8622684F8AA
:10B498006326332284F85526442284F85626D4F8A5
:10B4A8005826A4F85C1684F8643684F871374D2160
:10B4B8008F2361F3170284F873370A2384F865062B
:10B4C80084F87207C4F8582604F5CA6084F87437FB
:10B4D80004F5A471F7F7ACFB2046BDE81040FFF770
:10B4E80063BE0000F0B502298BB004460D461CD19E
:10B4F8003F4B40481B7800EB031000F58970F6F7C6
:10B50800EBF83D4B18603D4A0C236B43D718D358D2
:10B518003A7900210191511E082908D8DFE801F085
:10B5280009095E5E6262070765002D29EBD90BB039
:10B53800F0BD1B788DF8043000218DF8242005A873
:10B548001022019E05F0E8FCBF683846F4F71AFEA1
:10B55800C2B2102A28BF1022394605A805F044FDBA
:10B568002E229DF8243084F860260022C4F85C66F8
:10B57800A4F8625684F8743684F8612605AB04F2A0
:10B58800646509AE1A4603CAB24228606960134668
:10B5980005F10805F6D1332384F85536442384F899
:10B5A8005636D4F85836162262F31703C4F85836BC
:10B5B800002384F871374FF45C43A4F872371923D9
:10B5C80004F5CA6084F8743704F5A471F7F730FB02
:10B5D80020460BB0BDE8F040FFF7E6BD1B88ADF88C
:10B5E8000430A9E71B680193A6E71B680193A3E74A
:10B5F800C402002020030020E005002008000020ED
:10B608002DE9F041884D894F2B78142202FB0373F2
:10B6180088B093F85530012B04460E4613D191F8A3
:10B62800213133B1332B0ED191F822310BB1442B98
:10B6380009D1B368C3F31703172B54D006D8142BBA
:10B648002DD0152B43D008B0BDE8F08103F18073ED
:10B658004B3B23F07F43012BF5D8D6F82031744AB1
:10B6680023F07F4323F0FF039342ECD1358DF0683C
:10B6780040F207239D4200F0D180B5F5027F00F02B
:10B68800BE80B5F5007F08D1F5F782FC942800F05C
:10B69800B680B0F5967F00F0C1800222B6E002A81D
:10B6A8003146F7F7A0F8BDF90800002804DA03A826
:10B6B800F7F7F0F90028C6DB2D28C4DCA4F8BA088F
:10B6C800B4F8B03843F01003A4F8B038BBE701234E
:10B6D80084F8B8380023A4F8BA38564B1B68643B82
:10B6E800C4F8BC38AFE7D6F82031514A23F07F437D
:10B6F80023F0FF039342A6D196F80180B8F1160F04
:10B7080006F10C012ED8424602A805F06DFC02ABEA
:10B71800C8F11702002103EB080005F0FDFB0DF14D
:10B728000E00F7F7B7F9B0F100088CDB424A9DF834
:10B738001E1008EB4803980002EB83031B7999421B
:10B7480081D1B8F12D0F1FFA88F622DC0139029B4E
:10B75800125808291DD8DFE801F01B1B39393B3B7B
:10B768001C1C3D000B4602AA1C36186859689446F2
:10B77800ACE803000833B3426246F6D11868CCF847
:10B78800000099889B798CF80630ACF80410C6E75D
:10B7980013702878F8F782FA2A78142303FB0273C7
:10B7A800012183F8551097F82D300BB987F82D1023
:10B7B800B8F1020F10D1214B07EB0210196800F500
:10B7C8008970F5F7C3FFA4F8BA6879E71380E0E752
:10B7D8001360DEE71360DCE7B8F1000FF3D1184B14
:10B7E8001A78002AEFD083F8008060232380114B59
:10B7F8001B680BB16360E6E74FF0FF33FAE7B4F874
:10B80800B03843F00203A4F8B0380022B3790093AB
:10B81800737929462046FFF72BFE14E7B4F8B038B1
:10B8280043F00403EFE700BFC40200202003002018
:10B83800003344008049002008000020E005002073
:10B84800722E002010B52F4B1A782F4B142101FBB4
:10B858000233044693F85530012B37D12B4BD0F8DF
:10B86800B4281B689A1AB2F57A7F21BFB0F8B028BD
:10B87800C0F8B43842F00102A0F8B02890F8B8280F
:10B8880062B1D0F8BC289A1A312A81BFB0F8B02822
:10B89800C0F8BC3842F01003A0F8B038B4F8B0389B
:10B8A800DA0614D523F01003A4F8B038B4F8BA189F
:10B8B8002046FFF717FEB4F8BA3801339BB22D2B98
:10B8C800A4F8BA3802D9002384F8B83810BD98070C
:10B8D80008D523F00203A4F8B0382046BDE810408C
:10B8E800FFF730BD590702D523F00403F3E7DA0761
:10B8F800ECD523F00103A4F8B0382046BDE8104089
:10B90800FFF7ECBCC402002020030020804900207F
:10B9180038B5134B134A1B68C0F8B438002380F8B5
:10B92800B838A0F8BA38C0F8BC38A0F8B0381370E6
:10B938000D4B0E481B780E4D00EB031000F5897077
:10B94800F5F7CAFE0B4B02241860E0B2F9F76AFD5E
:10B9580001342C2C286305F10C05F6D138BD00BF45
:10B9680080490020722E0020C402002020030020FD
:10B9780008000020E005002000230370FF23437027
:10B988008370C37003717047F8B53A4D04462E783A
:10B998003948142707FB060090F84F60012E0CD099
:10B9A800022E0CD076B9A16090F84C30032B18BF4A
:10B9B8000022A368E26033B9FEE7A360F4E7A2605F
:10B9C8000022F6E7FEE70023C4E90433C4E9523352
:10B9D800C4E95433A3617F23A4F85831F6F788FEED
:10B9E800A878022844D0431F58425841234940F2BE
:10B9F800FF12FDF70BFD0220A4F84E24204A087020
:10BA0800002348708870C8701E4913705370937073
:10BA1800D370C4F8DA31C4F8DE31C4F8E231C4F8BE
:10BA28001233C4F81633C4F81A33A4F84C34A4F803
:10BA38004A341A4601330C2B0A70CA704A708A704D
:10BA480001F10401F6D1104B1B6803F57A7304F673
:10BA5800A800C4F8A438FFF78FFF84F8AD2884F84D
:10BA6800AE28228062602046BDE8F840FFF750BF4C
:10BA78000120BBE7C402002020030020A905002004
:10BA8800750500207905002080490020034640788C
:10BA9800FF2805D0012803D19B78012B08BF02207D
:10BAA8007047007840B14B79834204D18879431EAE
:10BAB8005842584170470020704710B54B790370C1
:10BAC8009379DB0943705379032B044607D1107926
:10BAD800FCF75CFBE0701368DBB2237110BDFF2339
:10BAE800C370FAE77FB58B6833F07F4305460C4691
:10BAF80000F6A8060ED18B79012B0BD101A8F6F719
:10BB0800C5FD9DF80930082B04D001AA214630460E
:10BB1800FFF7D3FF21463046FFF7C3FF78B3A3688A
:10BB2800C3F31703F52B16D16678012E29D83246B0
:10BB380004F10C0101A805F057FA01ABC6F10202A5
:10BB48000021981905F0E8F99DF805309A1E53422E
:10BB5800534185F8AA3895F8AD3853B195F8AE3801
:10BB680021790A480133DBB2CB1A59425941F5F71A
:10BB7800A0FC012385F8AD38237985F8AE3804B0E8
:10BB880070BDA389ADF80430DEE700BFB42F0020F4
:10BB98007FB52E4E044600F11C05B4F85411B4F8D4
:10BBA8005621881A83B2000444BF80339BB20BB974
:10BBB80004B070BD91421FBFB4F85811A3180132E8
:10BBC8000A4096F82D101ABF93F85A31A4F8562156
:10BBD8000023022904F110022946684620D1FEF705
:10BBE800EBFE9DF80030022BD7D1E368DBB9A068E3
:10BBF8000368BDF802201B692946984704F5CA6600
:10BC08002A4669463046F6F781FD31461048FDF769
:10BC180029FA3146204604B0BDE87040FFF762BFFC
:10BC2800F6F7FCFDDDE70B4E69460020F6F7A6FFA8
:10BC3800737833B1A068BDF80220036829461B69F0
:10BC48009847B378002BD9D0E068D1E720030020CB
:10BC58008C060020750500200148FFF717BF00BFBC
:10BC6800B015002070B5594C594E86B000211622E7
:10BC7800684605F051F92046F5F70DFC94F88C302C
:10BC88008DF800008DF80130204694F88D308DF83D
:10BC98000230F5F7F7FB94F8913094F890208DF87E
:10BCA80003005B0002F0010203F00203134394F85F
:10BCB800A52043EA821394F8A62043EAC2139DF80C
:10BCC8000B2002F03C02134320468DF80B30F5F7A9
:10BCD800D0FB05463046F8F7C1FD01462846F5F782
:10BCE80095FC94F893308DF8073094F8943094F8D4
:10BCF80095208DF8083094F8963094F992508DF884
:10BD08000400DB00920002F0040203F0080313436E
:10BD18009DF80B208DF8095022F00C021343304691
:10BD28008DF80B30F8F79AFD01462846F5F76EFCBA
:10BD38008DF80A0004F12800F5F797FF8DF80C003C
:10BD48002046F5F774FB8DF80D0004F11400F5F7A3
:10BD58008CFF8DF80E0004F13C00F5F786FF8DF896
:10BD68000F002046F5F774FB8DF810002046F5F714
:10BD7800A3FB94F8A7308DF81230164B8DF81100FC
:10BD8800DB7D8DF81330FFF767FF134B1A78931E8E
:10BD98005A425A4100F0030343EA02230F4A10486B
:10BDA800127943EA4223BDF8142023F0FC039B05D3
:10BDB80022F4407222F003029B0D134302216A46CB
:10BDC800ADF81430FBF722F806B070BDB42F002090
:10BDD8005C300020980A002085060020B805002065
:10BDE800C815002070B54C88B4F5427F03464FF063
:10BDF80000000AD80D780B2D77D8DFE805F0060F7C
:10BE08001C2C2F32383B54575B6DA2F1240462423C
:10BE1800488062410A7083F809033EE04D2A01D048
:10BE2800582A06D11A7002220A70002083F80903E2
:10BE380070BD0022F8E702F0FD003C2801D0212A5D
:10BE4800F7D15A701A784D2A0CBF082203220A70BB
:10BE580000229A70E9E79A700422DBE79A800522AB
:10BE6800D8E7988800EB02229A800622DCE7DA807D
:10BE78000722CFE7D88800EB022292B2002ADA80A4
:10BE88000CBF0B220A220A7000224A80012283F882
:10BE98000923DB88B3F5407F01D80020C8E70020DC
:10BEA80008704880C4E7DA800922B3E79A800A223A
:10BEB8000A70EBE7B4F5407F3CBFE41822724A8869
:10BEC800013292B24A80D88890429CBF0B220A70F5
:10BED800012283F80923E0E783F808230222087087
:10BEE800488083F809230120A2E708704880D4E736
:10BEF800CB88B3F5407F70B531D8242303700B7815
:10BF080043704B7883700B784D2B14D1CB88C3705A
:10BF18008B88037105230022CD88D4189542A6B2D8
:10BF280010FA84F415D891F808232270CA880132CF
:10BF3800981880B270BD8B78C3708B8803718B881A
:10BF48001B0A4371CB888371CB881B0AC3710823F2
:10BF5800E1E78C180132247A845592B2DCE700209C
:10BF6800E8E700002DE9F74F16464A88B2F5427F08
:10BF780004460D462ED80B780A2B0FD9A3F164027C
:10BF8800032A03D90020287068802DE0653B8F4F75
:10BF9800022B33D8DFE803F063A4A70000210A2BA3
:10BFA800F0D801A050F823F0DDBF0008F7BF000863
:10BFB8008DBF00088DBF00083BC0000849C00008BD
:10BFC80055C000085BC000088DBF00088DBF000881
:10BFD800C9C00008A6F124077E424FF000007E4148
:10BFE80068802E7084F8090303B0BDE8F08F6F2EC7
:10BFF8000CBF642300232B700020F3E716F0040F16
:10C0080014BF4D2358233E7023703A78D1070ED4BD
:10C0180012F0020F14BF21233E236370C2F3C00342
:10C02800D20648BF43F00203A3700423E3E73C238E
:10C03800F3E7A68005232B7084F809130020D3E7C3
:10C04800A38803EB0623A3800623D4E7E68007230F
:10C05800F1E7E38803EB0623E3806523CBE70DF1E3
:10C0680006007E70F6F75EFA3978F6F753FAA78875
:10C078002179F6F74FFA390AF6F74CFAE788A179E9
:10C08800F6F748FA390AF6F745FA9DF80630B3424A
:10C0980006D000232B706B80032384F80933CDE787
:10C0A800002F0CBF66230A232B70012384F8093361
:10C0B80000236B80E288B2F5407FBFD92B70BDE7C3
:10C0C800B2F5407F3CBF121916726B8801339BB2E0
:10C0D8006B80E2889A4201D866232B700123DCE743
:10C0E8007E806723F9E7B7F8028097F8009008EB9D
:10C0F80006284FF6FF730DF106001FFA88F8494627
:10C10800ADF80630A7F80280F6F7F0F82679B4F80B
:10C1180004A03146F6F7EAF84FEA1A21F6F7E6F8EE
:10C1280094F806B0B4F806A05946F6F7DFF84FEAD7
:10C138001A21F6F7DBF8797804F10807F6F7D6F84C
:10C1480052463946F6F7DEF8BDF8063043453AD18F
:10C1580019F0040015D086EA0B01E21D002398B2FD
:10C16800824584F8081307D80223012000222A7088
:10C178006A8084F8093337E712F8010F0133414028
:10C18800EDE7A178F5F75CFA217984F80803F5F76B
:10C1980057FAA18884F80803090AF5F751FAA17932
:10C1A80084F80803F5F74CFAE18884F80803090ACB
:10C1B800F5F746FAE28884F808033946F5F746FAAF
:10C1C80084F80803D0E703230020CFE7082E0020D7
:10C1D800CB88B3F5407F2DE9F04104460D464AD897
:10C1E8004B783C2B40D0A3F12100434243415B00F4
:10C1F8002A784D2AAA7808BF43F00403D10748BF1C
:10C2080043F0080392074FF02402227048BF43F01E
:10C2180010036F226270A370AB88E370AB881B0AAF
:10C228002371EB886371EB88A71C1B0AA37138463E
:10C23800F6F754FC0822E071E988A2F108039BB2E2
:10C24800561C8B42B6B204EB02080FD3063189B2F2
:10C258003846F6F76FF888F80000000AA055E88815
:10C268000A3080B2BDE8F0810123C1E72B441B7A74
:10C27800A3543246E0E70020F4E710B5044681787D
:10C288000020F5F7DDF9217984F80803F5F7D8F9E6
:10C29800A18884F80803090AF5F7D2F9A17984F886
:10C2A8000803F5F7CDF9E18884F80803090AF5F7DA
:10C2B800C7F9E28884F8080304F10801F5F7C6F91C
:10C2C80084F8080310BD00002DE9F74FC788DFF890
:10C2D80090800D4604463A4600F10801002628469B
:10C2E80004F082FE55FA87F7E6804FF03B09BD421D
:10C2F80005D1204603B0BDE8F04FFFF7BEBF15F8E3
:10C30800013BFF2B2AD0FE2B28D0FF2E1ED1362B27
:10C31800EDD858F833204FF0000A10460192F3F791
:10C3280031FF5FFA8AFB5845E388019A0AF1010A4E
:10C3380005D85A1C2344E28083F80890D7E7591C93
:10C34800E180234412F80B101972E6E7FE2ECED1D5
:10C35800E288511C2244E1801372C8E71E46C6E7F2
:10C368004841010830B50F4B1C780F4B142505FBCD
:10C37800043393F84F30012B03D0022B10D00BB1AC
:10C38800FEE7114600234360C0F81233A0F82236B6
:10C39800A0F8203640F2FF330160A0F8243630BD03
:10C3A8000021EFE7C402002020030020F8B5B0F810
:10C3B8002026B0F82236D21A93B2120444BF03F5ED
:10C3C80080639BB2E62B044608D800F2163500F2CB
:10C3D8001236206803685B69984700B9F8BD206881
:10C3E80003689B699847314602462846FFF7FAFCDE
:10C3F8000028EED004F6262729463846FFF7E8FE3F
:10C4080000239AB29042E4D9B4F82016B4F824C6AE
:10C418004A1C02EA0C02B4F822C694451EBF091948
:10C4280017F803C081F826C603F1010318BFA4F862
:10C438002026E6E7F8B500F1080504460A46011D7E
:10C448002846FFF78FFD70B3637A3E2B14D004F6AD
:10C45800262629463046FFF74BFD0246206801682C
:10C468000F693146B847637A3E2B1CD129460E48DE
:10C47800BDE8F840FCF70EBEA389742B0AD042F63B
:10C48800FF729B1A18BF0123A27A9207EBD4002BE4
:10C49800DDD1E8E70023A37204F626212846FFF73A
:10C4A80013FF0123F0E7F8BD8C06002003680BB1E9
:10C4B800FFF7C0BF70470346006868B1B3F820268D
:10C4C800B3F82236D31A98B21B0444BF00F5806033
:10C4D80080B2003818BF012070470346006880B159
:10C4E800B3F82226B3F82016914209D099180132E0
:10C4F80091F82606B3F824160A40A3F822267047B6
:10C50800002070470346006838B10022A3F82226AD
:10C51800A3F820260368DB691847704710B504465E
:10C528000548FEF77EFE0548FFF7ECFF60680368E4
:10C53800BDE81040DB691847080D0020C82000201E
:10C5480070B50A4C25780A4C142606FB054494F865
:10C558004F40012C03D0022C05D00CB1FEE7194640
:10C56800416011B9FEE71146FAE770BDC402002028
:10C5780020030020024B1A790AB901225A71704728
:10C58800B8050020024B1A790AB101229A71704746
:10C59800B805002038B572B6234C0025F6F736FEEC
:10C5A800F7F7C0FAF6F702FEF6F7ECFDF7F734F9FD
:10C5B800F7F772FAF7F7B2FF02232373C4E90455B9
:10C5C800A560F6F789FF194B1D70F6F7A5FD184B06
:10C5D8001848D02283F83223F6F734FE294620463D
:10C5E800154C02F0D1FF4FF47A70F6F72BFE94F851
:10C5F800572094F856101148FAF780FB94F8571012
:10C608000F48FBF729FF94F858400E482146F5F7E4
:10C61800C7FC3CB10C4B0D4A1A600D4B0D4A1A6011
:10C62800FAF77AF862B638BD5C300020380200208C
:10C6380000E100E0E0930400C4020020C8150020D7
:10C648008C060020C80C00203C020020C9230008EA
:10C6580040020020F12C000873B51648164C4FF61E
:10C66800FF7103F0E1F8208023889B0712D5134E51
:10C6780035798DB10F4808236A46002102F055FF2D
:10C68800D6E90602DDE900139A4208BF884201D0C4
:10C698000023238002B070BD02236A46054829465C
:10C6A80002F043FF064BDA8BBDF800309A4218BF00
:10C6B8002580EFE75C300020F60C0020B80500204C
:10C6C800C4020020044A00231370044A1380044A59
:10C6D8001370044A13707047020D0020040D0020E7
:10C6E800A03000208C0A0020024B1878B0FA80F0A5
:10C6F80040097047020D00200D4A11780346A9B978
:10C7080010700C4A012010700B4A032B118009D0BD
:10C71800042B01D083420AD1084B002283F87220EF
:10C72800012070474FF4FA73138070470020704758
:10C73800020D0020A0300020040D0020DC040020A1
:10C74800034A00231370034A1380034A1370704787
:10C75800020D0020040D0020A03000200A4A08B570
:10C76800138883B1013B9BB2138063B9074B1B78D5
:10C77800032B02BF064B01221A70FFF7E1FF054B9E
:10C78800002283F8FA2A08BD040D0020020D0020BB
:10C798008C0A0020C815002010B5C379212B0ED1B2
:10C7A800074CF8F7EBFAFFF7CBFF94F8FA1A0329CE
:10C7B80002D12046FAF7FDFC002384F8FA3A10BDAE
:10C7C800C815002010B50D4B1B78013B032B14D85E
:10C7D800DFE803F002090D072023BDE81040F8F751
:10C7E800BDBA2423F9E7BDE81040F8F711BB2323AD
:10C7F800F8F7B4FA024B00221A7010BD020D00209F
:10C80800A0300020034B01221A7000225A711A71BD
:10C81800704700BF732E0020054A064B12791B7F14
:10C828001AB105495B22F8F7A5BC04495B22FAE76F
:10C83800B8050020C4020020A1300020FC300020F0
:10C8480038B5114B1A79054632B10146002218460F
:10C85800BDE83840F8F7EABC0C4A0D495B23F8F705
:10C8680073FC7DB90A48F8F775F90128044607D022
:10C8780000280849284614BF01240224F8F79CFC24
:10C88800204638BD0148EEE7B8050020582F0020A3
:10C89800FD2E0020B42F0020024B1878831E58422A
:10C8A8005841704785060020044B1B78022B06BFB1
:10C8B800034B93F872000020704700BF85060020E4
:10C8C800DC04002010B5184B1A78184B04461420C5
:10C8D80000FB023393F85500012822D122889306E1
:10C8E80005D522F02002228005230B7010BD12F01E
:10C8F800400317D0FFF7D8FF28B1FFF7F5FE10B9AE
:10C9080000230120F1E7606830B1094B1B681B1A4E
:10C91800312BF5D90023636022F0400222800623E0
:10C92800EFE700231846E0E7C402002020030020B8
:10C938008049002013B50DF107010446FFF7C2FF37
:10C9480018B19DF8070002B010BD2080FBE7000079
:10C958002DE9F04106460C461546FFF7A5FF70B1D4
:10C96800184B93F82D30581E012819D8164BB3F8D8
:10C978005861B3F85671002291B28D4201D8BDE8D2
:10C98800F081B3F85401411C3140B9421FBFC018AF
:10C9980014F802C080F85AC1A3F854110132EBE729
:10C9A800032B09D1094E0D44AC42E8D014F8011B01
:10C9B8003046FFF77BFDF7E770680368BDE8F04194
:10C9C8001B69184720030020080D0020C8200020FC
:10C9D800F8B5214B214D1F79CB78C3F3000385F8B7
:10C9E80095304B79C3F3801385F896300646C8789E
:10C9F80040080C46F4F791FD85F892002379C3F3BB
:10CA0800060385F893306379227903F03F035B00CE
:10CA180043EAD21385F89430E6B1DFB1A37803F086
:10CA2800F003202B04D12046BDE8F840FFF7B4BE40
:10CA3800A2790B48E11D5208FFF78AFFA17905F199
:10CA480064004908F5F713F905F13C00BDE8F84022
:10CA5800F5F707B9F8BD00BF732E0020B42F0020EA
:10CA68007830002070B50546B8B9184B184E1B78B9
:10CA7800184A14794CBB022B174812D1B17801F02F
:10CA88000701F8F72DFC4379C3B931460120FFF7B8
:10CA98009FFF1248F4F7C8FC09E0114B114E1B78B0
:10CAA800E6E701229342027044710471EDD80B4805
:10CAB80080F89050BDE87040F4F7B4BC0A4B1C7481
:10CAC8005C825C61094B1C71DFE770BDFE0C0020C5
:10CAD800FD2E0020B8050020732E0020B42F002062
:10CAE800FF0C0020582F0020080D0020C82000202F
:10CAF80010B50246FFF7D8FEB8B10C4B93F82D30AD
:10CB0800591E012904D8BDE810400948FEF766BB44
:10CB1800032B04D1BDE810400648FFF7CCBC506891
:10CB28000368BDE810405B69184710BD200300206A
:10CB3800080D0020C820002010B50246FFF7B4FEFB
:10CB4800B8B10C4B93F82D30591E012904D8BDE813
:10CB580010400948FEF750BB032B04D1BDE8104034
:10CB68000648FFF7BABC50680368BDE810409B69E7
:10CB7800184710BD20030020080D0020C820002001
:10CB88002DE9F04FDFF8C88098F8004097B081464B
:10CB98000E461746002C53D12E4B1B78022B4BD137
:10CBA800DFF8B4B00DF1180A25465846ECB2FFF785
:10CBB8009FFF40B15846FFF7BFFF0135402D0AF8E7
:10CBC800010BF2D12C4625482146F5F750F82448A8
:10CBD800F5F747F8234D8DF8129095F8A4308DF8A5
:10CBE8000C30214B85F89190DB788DF80D30284674
:10CBF80095F890308DF81130F4F73BFC8DF80E0065
:10CC0800F8F764F910F0010F8DF8130018BF3E46CD
:10CC180028468DF81460F4F73EFC98F800308DF83B
:10CC280010007BB9114A1248009406AB03A9F7F724
:10CC380085FF17B0BDE8F08F0748FFF76FFCC9E71D
:10CC48000024C7E7094A0A4803A9FFF7BBFDF0E734
:10CC5800A030002085060020783000200430002015
:10CC6800DC2F0020B42F0020732E00207A2E002005
:10CC7800FC30002030B4084C257925B10146204607
:10CC880030BCF8F7E5B9054C94F8A430013384F8C2
:10CC9800A43030BCFFF774BFB8050020B42F0020C3
:10CCA80008B50246FFF700FE18B9A2F82206A2F856
:10CCB8002006054B93F82D30032B04D1BDE808401E
:10CCC8001046FFF773BB08BD2003002070B5002392
:10CCD8009CB2A24200D870BD058886886C1C34407E
:10CCE8004688A6421EBF2D18CE5CAE7103F1010323
:10CCF80018BF0480ECE708B56830FFF7E7FF08BD08
:10CD0800A0F11400F7E7000038B50A4B93F82D306E
:10CD180000F5EF65022B0446284608D1FCF79CFE77
:10CD28000246294604F24A40FFF7D0FF38BDF5F71E
:10CD380026FCF5E7200300202DE9FF410446B0F862
:10CD48004C14B0F84A04F5F7EDFEE3684BBBDD2858
:10CD580008D804F5F37604F5ED75A06803685B69F7
:10CD6800984710B904B0BDE8F081A06803689B69D2
:10CD780098472A46034631466846F5F74FFD00288E
:10CD8800EBD09DF80030022BECD104F5CA65324691
:10CD980069462846F5F7BAFC29462046FFF7B4FF4E
:10CDA80094E0DD28DED84D4D2B780133DBB2012B22
:10CDB8002B700FD900232B70A06803685B69984714
:10CDC80050B901232B70E06803685B69984730B954
:10CDD800287004E0002BEFD02B78012BF3D004F55A
:10CDE800F37604F5ED772B78002B36D1A06803682D
:10CDF8005B69984788B3A06803689B6998473A4677
:10CE0800034631466846F5F709FD0028EBD0DFF800
:10CE1800D08069460120F5F7B1FE98F8023033B1A9
:10CE2800E068BDF80220036831461B6998479DF801
:10CE38000030022B11D104F5CA67324669463846DC
:10CE4800F5F764FC98F800301BB139462046FFF727
:10CE58005BFF39462046FEF7D3FB04F21E3604F288
:10CE680012372B78012B7FF47DAFE06803685B698C
:10CE7800984700283FF476AFE06803689B699847B5
:10CE88003A46034631466846F5F7C8FC0028E8D01C
:10CE9800134F69460220F5F771FE7B7833B1A0681D
:10CEA800BDF80220036831461B6998479DF8003099
:10CEB800022B7FF457AF04F5CA6532466946284607
:10CEC800F5F724FC3B78002B7FF466AF2946204613
:10CED80004B0BDE8F041FEF793BB00BFB4050020E5
:10CEE800750500201D4B70B51D680446FFF7DCFC76
:10CEF80058B9C4F8A458A4F85601A4F85401A4F8E1
:10CF08004C04A4F84A0484F8AD08154E96F82D3060
:10CF1800013B012B21D82046FEF73AFE2046FFF7B9
:10CF28000BFF104B1B78142202FB036696F8523055
:10CF380063B1D4F8A438EB1AB3F57A7F08D3C4F8F0
:10CF4800A4582046BDE87040FEF780B9C4F8A4583C
:10CF58002046BDE87040FEF775BC70BD80490020D2
:10CF680020030020C40200202DE9F04FDFF878816B
:10CF780098F80030012B85B000F249810BB9F6F71B
:10CF880075F85A4DFFF706FB696C5948F6F7CEFB62
:10CF9800584B00221A809A70574B20229A61072416
:10CFA8004CF25030013CF6F723F9F6F74BF914F040
:10CFB800FF04F5D1514802F066FC013880B24FF603
:10CFC800FD73984203D94E490120F8F757F94D4BA4
:10CFD8004D491C804D4B49481C80F7F775FB7D2057
:10CFE800F6F730F94A48F6F7C5F8F7F789FF95F8E4
:10CFF80020B0BBF1200F00D9FEE795F82800454E78
:10D00800AB8D01930528696A95F8297095F82A303F
:10D01800B07100D9FEE7404A4FEA001E02EB001C3F
:10D0280052F80E2002B9FEE7DCF808E09CF80C90F4
:10D03800B2609CF80420C6F810E00092F27186F8FD
:10D048000C9086F8D900B482A446A246A646019A56
:10D0580042FA0CF2D20707D5012202FA0CFA4EEA7C
:10D068000A0A1FFA8AFE92460CF1010CBCF1060F5F
:10D07800EDD1DFF8A0C0BAF1000F01D0ACF814E090
:10D08800BCF814E0BEF1000F00D1FEE7009AA2EB55
:10D098000902D2B25A4528BF5A4605288CF81720EB
:10D0A80000F00482012800F2088207F1FF30C0B2C4
:10D0B80000F0F281022831D8581EC0B203280CD8DB
:10D0C8000C2A02D90C208CF817009CF81700904203
:10D0D80001D98CF817203C4623E0122A84BF12237A
:10D0E8008CF817300023F0E79F2E0020C4020020A0
:10D0F80030020020FA0C0020000400485C300020B8
:10D108005A1A0108F40C0020C8020020F60C00206E
:10D11800B8050020980A002000240108052B28BF24
:10D128000023A3482246F4F7F9FC0024A14B86F813
:10D13800D840B4759E48FF261E705E70F7F7B4FBA2
:10D1480001469D4802F045FA9C4B1C809C4B1C7084
:10D158009C4B1C709C4B1C809C4B1C809C4B1C70DB
:10D168009C4B1C809C4B1C709C4B1C709C4B1C70DB
:10D178009C4B01201C70FFF7A5FAFFF7BDFAB5F824
:10D188004830B5F84A2095F840109748F4F710F958
:10D19800B5F848109548F4F741FC9548F8F776F843
:10D1A8002A78944B9448142101FB023393F84E10CB
:10D1B800F4F7FEFE914B924A92499348FEF7E4FB3E
:10D1C8008E4A90499148FFF7CDF813468D498C4A0D
:10D1D8008F48FFF7B5F9B5F848208E498E48F8F71B
:10D1E80095FB7548F7F751FB8C48F4F775FD8C48AB
:10D1F800F4F74DFD8B48F4F79DFE8B4B1C708B4B61
:10D208001C808B4B1C80F6F755FC88F80060F6F7FD
:10D218005BFC6C4D00283ED06E4A13880BB1013B75
:10D228001380664A138813B9824BB3F84830013B20
:10D238009BB2012B138040F04481614A1370FFF7C1
:10D248008DFA2B783BBB7C4A614B90781978138810
:10D25800002840F04081002B00F0EF83013B9BB297
:10D268000229138040F03D81744B20229A626F4C52
:10D278002388002B00F03C81013B9BB2704823803F
:10D28800F7F782FE4C48F7F700FB23881BB96D4976
:10D298006D48F5F745FD4D4E6C4C3388022B00F078
:10D2A8002A81042B00F04F81012B0FD1404B9A7D2E
:10D2B800D97D0132D2B2914298BF00229A754B4B68
:10D2C8001146187AFFF7D6FC0223338023889BB2D5
:10D2D800EBB13388032B40F04F812388D80703D55F
:10D2E800002323800423338023889BB27BB12388C7
:10D2F80023889A0748BF23882388394ADB0748BF11
:10D30800238800231370374A2380338013702B78C7
:10D31800002B00F09081334F274800242C70F7F73A
:10D3280059FA97F80090B9F1000F00F033812046C0
:10D33800FFF798FB2D4B1E4D1C722B4BAA7D83F8D3
:10D34800A7203A782649224C012A94BF00220122BC
:10D3580083F8A5200A78012A94BF00220122B9F196
:10D36800010F83F8A62023780AD93248002B00F051
:10D378001481012B00F01681164BB0F84C201A804E
:10D388002378022B03D1134B1B8803B9237022780F
:10D3980000230120022A30803B700B7058D01449BA
:10D3A8000B70002A54D1FFF7CBF9FFF7A5F94FE02E
:10D3B800980A0020A02E00205C3000205831002060
:10D3C800F80C00208D0A0020702E0020000D00208F
:10D3D8008506002088060020860600208406002096
:10D3E800FF0C0020FE0C0020B42F00208C30002001
:10D3F800732E002020030020C80C002034020020D7
:10D40800DC15002030020020080D0020C820002074
:10D418007830002000000020EC050020744900202E
:10D42800803000207C0600209E2E00209C300020AA
:10D438009E300020C4020020FA0C0020000400489E
:10D44800B80500206610010804000020F60C002032
:10D45800A04A138813B9A04BB3F84A30013B9BB2DA
:10D46800138013B99D48F4F72AF89C48F3F7D9FFBD
:10D478002378022B02D09948F3F782FF984B1F7844
:10D48800002F00F0B880974B20229A62F7F72AF80D
:10D49800012388F80030B9E0022805D80C2A02D9FF
:10D4A8000C238CF817303C4600233AE67B1E022BEF
:10D4B800FAD8082AF7D90823F3E78B48F4F7C8FA0B
:10D4C80033E6002B7FF4BBAE01232B70874B5A6ADF
:10D4D800874B1A80B3E6002B00F0AD82013B9BB26C
:10D4E80013801388002B7FF4C2AEF5F781FEBEE6E9
:10D4F80040F2E733C2E67D4B7D4A5B6A12889B1A8D
:10D508009BB240F2ED2293427FF6E0AE794B7A4827
:10D5180000271F70F7F7EEFE7348F7F7C5F90146C5
:10D52800764802F056F8764B187AFFF775F9032318
:10D538003380744B74481F80744B278001221A7102
:10D54800F4F7CEFBC2E66D484FF6FF71F5F70AFE19
:10D5580002F0D5F86948002102F005F97D20F5F7B9
:10D5680071FE6B4A0523338000231370694A1370D8
:10D57800644A13802380A9E6052B7FF4B5AE23887F
:10D5880099077FF5B1AE00202080FFF759F9614B6C
:10D598001870A9E6FFF736F9CCE6012222705E4A38
:10D5A8001370E9E65C4ADFF8749113780133DBB253
:10D5B800137099F80020C2B990F850C09C453FF606
:10D5C800DBAEDFF85CA19AF8723043B9554B1B7992
:10D5D8002BB96AB1FFF7B4F801238AF87230022335
:10D5E8002370012389F80030C6E64FF0050CE5E703
:10D5F8004D490C20E9E44B48F7F7F0FCF7F71AFD22
:10D608000128064605D003283FF442AF05B0BDE81F
:10D61800F08F4448F7F790FC41F28833A5F8DA30E8
:10D62800304B85F8D8602022A5F8DC709A613F4B12
:10D6380027709E70EAE7284C3D4D94F85630EBB1C0
:10D648003C493D48F9F794FB68B122783B4B1421DB
:10D6580001FB0233012293F84C30032B04BF012352
:10D668002B70354B1A7134480DF10B01F9F798FB03
:10D6780020B19DF80B30FBB1012B20D094F8563027
:10D6880023B994F85730002B00F01F812A480DF178
:10D698000B01F9F7AAFB002864D09DF80B30033B77
:10D6A8000F2B5FD8DFE803F04C5E5E7B5E5E5E7D2D
:10D6B8005E8399A7ACB2AEB0FEF7D4FADEE71E4897
:10D6C80003A9F9F7C0FB0028D8D09DF80C00F9F79A
:10D6D8008DFED3E79E300020C4020020B42F002026
:10D6E8008C0A002000040048980A002000440140E9
:10D6F800702E0020F80C0020A02E00205C300020A6
:10D708008C300020F40C0020744900208C06002086
:10D71800FF0C0020FE0C0020860600208406002056
:10D72800DC040020B8050020641A0108FA0C002067
:10D738009E2E00207A2E0020C815002020030020ED
:10D74800F6F7E0FEA04B1B78022B07D10420FEF76A
:10D75800D3FF9E4B032283F8FA2A03E003219B4858
:10D76800F9F727FD94F85730002B00F0AE80984960
:10D778009848FAF7C7FE08B101232B70B4F848207F
:10D78800944802A9FAF7E0FE00284CD09DF808302A
:10D79800042B48D8DFE803F0415B5F639300062160
:10D7A800DDE78D49A1F13300F9F7DAFCDAE7874FB5
:10D7B80003A907F13300F9F7FBFD0028D2D09DF843
:10D7C8000C30002BCED0804B18780228CAD1FEF737
:10D7D80093FF0C2387F8FA3AC4E77B4B1B78022B9C
:10D7E80005D10320FEF788FF784B0D22B3E77B4B6A
:10D7F80001221A70B6E701217948F4F762FAB1E715
:10D808000221F9E70321F7E70821F5E76F4B75488F
:10D8180093F83310F4F792FBA4E76E48FBF70CFD7E
:10D82800714B00221A706B4F0DF109013846FAF757
:10D83800C5FE002849D09DF80930022B43D8002B9B
:10D8480000F0898066480121F4F73DFA3DE061481F
:10D85800FBF73AFDE7E75F48FBF76EFDE3E7624F4A
:10D868003B784BB959480DF10A01F9F7ECFA18B1B0
:10D878009DF80A00F9F7BAFD54480DF10B0203A907
:10D88800F9F726FA68B19DF80B2003995148FAF781
:10D89800E9FE3B780133DBB2022B88BF00233B70E3
:10D8A800C1E7FFF701F80028F3D0504B93F82D306B
:10D8B800013B022BEDD84748FBF79EF8E9E74548BE
:10D8C800FBF768FDAFE7032B4BD094F8583023B132
:10D8D8003F494748F4F793FC08B92B78BBB10023BC
:10D8E8002B70424D23783A494248142707FB0353CB
:10D8F80093F84D20F3F73AFD237835493E4807FB66
:10D90800035595F84A3095F85620F7F713FD3B4B29
:10D918001B78002B7FF47AAE3388022B3FF476AE67
:10D928003748FFF7DFFA3748FFF7BAF93648F4F710
:10D93800E4F92B48F4F7B0F910B93148FEF7FAFFCB
:10D94800431E0B2B73D8DFE803F03B616472152983
:10D9580033727266726E97F869102248F4F7EEFA1D
:10D96800B3E7BA7D1948023AD2B207F11801F9F7BC
:10D978009AF9AAE7144B1878022805D1FEF7BCFEDD
:10D98800124BFF2283F8FA2A1648F4F7EBFA00281C
:10D998003FF43CAE114B01221A7037E60A4B1B7854
:10D9A800022B01D10320E9E70C4B01221A70EBE7A7
:10D9B800F6F7A8FD044B1B78022BE5D10420DDE720
:10D9C800FEF7D8FDE0E700BF85060020C815002057
:10D9D8007A2E00208C060020FB1500208C0A0020DF
:10D9E800803000207C060020AF05002020030020A6
:10D9F800C80C0020E4050020A02E0020F80C002010
:10DA0800080D0020C820002074490020FEF7BAFD48
:10DA1800BAE7F5F7E9FA0A48F4F75CF9C1B2094838
:10DA2800F4F78CFAB0E70648F4F754F9ACE70428A1
:10DA38003FF42EADA8E7632352E540F2F3130FE459
:10DA4800803000207C06002008B5FFF78DFAFCE73F
:10DA580038B5244B244A1A60244B254A1A605A6167
:10DA68009A62DA63234A1A655A66234A9A67234AEE
:10DA7800234B244802F10801283200245A6140F25D
:10DA8800FF12C3E91A427F251F4A1960C3F87022A2
:10DA9800C3F86C42C3F8744AC3F8785A1B4B036046
:10DAA80000F58E70FAF790FB194B1A4A1A601A485B
:10DAB8002146F3F70BFC194B194AC3F84C24C3E968
:10DAC8005545A3F84A44174B40F2FF32C3F82426C1
:10DAD800C3F82046144B154A1A60154B154A1A60AC
:10DAE80038BD00BF5C300020841A0108B42F002024
:10DAF800C0110108A8110108B41101085443010814
:10DB0800C81500208C0600200000FF074C430108C0
:10DB1800C80C00206C1B0108E4050020080D00203B
:10DB28000000FF01C82000207830002008430108C9
:10DB3800744900203843010830B59BB020220021E9
:10DB48000BA803F0E9F91822002102A803F0E4F970
:10DB58001C4A136823F4C06343F40073136013680A
:10DB680003F4C0630193019B01224FF40413CDE930
:10DB7800082300230A9310210623CDE915134FF437
:10DB880000330224032517934FF0005C4FF0007315
:10DB980008A8CDE91345CDE9183C00F045FB08B1CC
:10DBA80072B6FEE7CDE90400CDE906004F23214611
:10DBB80002A8CDE9023500F0D1FD08B172B6FEE742
:10DBC8001BB030BD00040058154B07B51A6842F465
:10DBD80080721A601A6842F400721A601A6822F495
:10DBE80080621A6000F0A0F8FFF7A6FF4FF0B0437C
:10DBF800DA6C42F00102DA64DA6C02F00102019296
:10DC0800019ADA6C42F00202DA64DB6C03F0020378
:10DC18000093009B03B05DF804EBFFF715BF00BF4E
:10DC2800004000587047FEE7FEE7FEE7FEE7FEE724
:10DC3800704770477047F5F757BF70470D488546DE
:10DC4800FFF7FBFF0C480D490D4A002302E0D458AA
:10DC5800C4500433C4188C42F9D30A4A0A4C00232E
:10DC680001E013600432A242FBD303F091F9FFF7FD
:10DC7800ABFFFEE70000012000000020A802002002
:10DC8800AC490108A8020020F44A0020FEE77047CA
:10DC98004FF0B04310B59A6B4FF0FF329A63D96BCF
:10DCA800DA630024996B9C63D96BDC63196C1A6482
:10DCB800196C1C64596C5A64596C5C64996A9A6250
:10DCC800996A9C62D96ADA62D96ADC62196B1A634A
:10DCD8001A6B1C63FFF7DBFF204610BD38B5104CEC
:10DCE800237805460BB9012038BD00F08DFA22785B
:10DCF8004FF47A73B3FBF2F3B0FBF3F000F074F86F
:10DD080004460028EFD10F2DEDD8024629464FF0E2
:10DD1800FF3000F037F8034B20461D60E4E700BFF2
:10DD2800480200204C02002010B5032000F018F82B
:10DD380000F06AFA064B18600F20FFF7CFFF044681
:10DD480018B9FFF76FFF204610BD0124FBE700BF9D
:10DD580044020020014B1868704700BF804900202A
:10DD68000749CA6822F4E0620302120403F4E0637C
:10DD7800120C134343F0BF6343F40033CB60704786
:10DD880000ED00E0164B30B5DC68C4F30224C4F1A2
:10DD98000703251D042B28BF0423062D4FF0FF354C
:10DDA8008CBF033C002405FA03F321EA0303A540D2
:10DDB80022EA0502A340002843EA0203ACBF00F1AF
:10DDC8006040084A4FEA0313B8BF00F00F00DBB207
:10DDD800AABF00F56140135480F8003330BD00BF7E
:10DDE80000ED00E014ED00E00138B0F1807F0BD2C7
:10DDF8004FF0E023054A5861F02182F823100020F3
:10DE0800072298611A6170470120704700ED00E011
:10DE18000A4A536943F4802330B55361EFF3108401
:10DE280072B60023CD58C5500433B3F5807FF9D1BD
:10DE38001369DB03FCD484F3108830BD004000581C
:10DE4800064B5A69002ABFBF054A9A6002F1883218
:10DE58009A60BABF5869C00F002070470040005848
:10DE680023016745044B5A6942F000425A615869D8
:10DE7800C043C00F704700BF0040005870B505464A
:10DE8800FFF768FF124E04463369D90313D4336988
:10DE9800DA0744BF012232614CF2FA32134011D141
:10DEA8000B4E306910F480200BD0FFF753FF001B96
:10DEB800A842F6D304E0FFF74DFF001BA842E3D3C6
:10DEC800032070BD024A1361024A01205360F8E73B
:10DED80000400058844900202DE9F041184D98462B
:10DEE8002B78012B06460C46174626D001232B70AB
:10DEF8004FF47A7000236B60FFF7C0FFA0B9012EC2
:10DF080016D1104A536943F0010353612760BFF3E8
:10DF18006F8FC4F804804FF47A70FFF7AFFF094A97
:10DF2800536923EA0603536100232B70BDE8F0818F
:10DF380039462046FFF76CFFEDE70220F6E700BF01
:10DF48008449002000400058054A536923F47E7331
:10DF580043EAC00040F4803040F00200506170474E
:10DF6800004000582DE9F041234F3B78012B05462E
:10DF780088463FD001233B704FF47A7000237B60C2
:10DF8800FFF77CFF044688B92B68042B13D11B4A82
:10DF9800536943F4803343F0040353614FF47A70B8
:10DFA800FFF76CFF0446154B1A681B6800233B708B
:10DFB8002046BDE8F0814FF0FF33C8F800306E68A6
:10DFC800D5E901321344B3420AD93046FFF7BCFF02
:10DFD8004FF47A70FFF752FF50B1C8F8006004465A
:10DFE800064A536923F47E7323F002035361DAE788
:10DFF8000136E5E70224DBE78449002000400058A9
:10E00800024A136843F48073136070470004005891
:10E01800024B186800F4C060704700BF0004005845
:10E028004FF0B0431868C0F3404070474FF0B0431A
:10E038001868C0F3400070474FF0B042536823F4AB
:10E048007F4343EA0023536070474FF0B04318689A
:10E05800C0F34060704700007FB54FF0B0432C4AD2
:10E06800D3F80831C0F3031003F00F0352F820402F
:10E07800284A52F82330B4FBF3F4FFF7C9FF264BC4
:10E08800054693E80700B5F5007F04AB03E90700F0
:10E0980010D0224B9C4218D303F5B70303F67F53E5
:10E0A8009C4229D903F5741303F510639C4225D8C3
:10E0B80002230BE01A4B9C4207D91A4B9C421BD9EE
:10E0C80003F5370303F5D853F0E7002304AA02EB5E
:10E0D800830353F80C4C144D2B6823F00703234398
:10E0E8002B60FFF737FE06462B6803F007039C42B8
:10E0F80006D1002004B070BD0123E7E70024EAE759
:10E10800FFF728FE801B0228EED90320F2E700BFA4
:10E1180004440108A44301084C100108C0CF6A0058
:10E12800BFEA21013F933402004000584FF0B0434A
:10E1380010B59A68D96812F00C0205D00C2A4AD199
:10E1480001F00303012B50D14FF0B0412B480B686D
:10E1580013F0080306D00B6813F0080337D1D1F881
:10E16800941007E00C68240756BFD1F8943009686A
:10E17800C3F3032350F82330002A0CBF18460020AD
:10E188004FF0B0418A6802F00C020C2A1ED1CA680E
:10E1980002F00302022A2ED0032A06D10B68184A7D
:10E1A80013F4801F174B18BF13464FF0B042D068C6
:10E1B800D168D268C0F306205843C1F30213013373
:10E1C800B0FBF3F0530F0133B0FBF3F010BD0B6855
:10E1D800C3F30313CEE7042A0AD0082A05D11B6823
:10E1E80013F4801304D10748CAE700231846C7E789
:10E1F80003480023C4E7024BD7E700BF04440108E3
:10E208000024F4000048E80108B5FFF78FFF4FF03D
:10E21800B043044A9B68C3F3031352F82330B0FB9E
:10E22800F3F008BDA44301082DE9F0410446002895
:10E2380053D04FF0B0439D68DE6803689B0605F035
:10E248000C0506F0030668D5026A1DB10C2D46D1EF
:10E25800012E44D1002A40D04FF0B043A16A1A6879
:10E26800170756BFD3F894301B681B0903F0F00357
:10E2780099421FD90846FFF7EFFE00282DD14FF02D
:10E28800B042136843F0080313601368A16A23F0CF
:10E29800F0030B431360606AFFF7CEFEFFF7B4FF8D
:10E2A800AB4B1860AB4B1868FFF718FD002834D04B
:10E2B800BDE8F0814FF0B042136843F008031360E3
:10E2C800136823F0F0030B431360606AFFF7B4FE92
:10E2D8000846FFF7C1FE0028E0D00120E8E74FF02C
:10E2E800B043002A54D01A6842F001021A60FFF7BE
:10E2F80031FD0746FFF79AFE002842D04FF0B042A2
:10E30800136843F0080313601368A16A23F0F0034D
:10E318000B431360606AFFF78FFE2368D80748D461
:10E328002368990700F18C8023681E0740F1FA8062
:10E33800A3694FF0B046002B00F0E180D6F8943086
:10E34800E16903F01002914200F0C48003F0030277
:10E35800022AC2D0D80740F1B380D6F8943023F00F
:10E368000103C6F89430FFF7F5FC0746D6F8943059
:10E37800990740F1A580FFF7EDFCC31B112BF5D9D8
:10E3880004E0FFF7E7FCC01B0228B3D903208FE79E
:10E398001A6822F001021A60FFF7DCFC0746FFF753
:10E3A80045FE0028B9D0FFF7D5FCC01B0228F6D9D6
:10E3B800ECE7082D03D00C2D05D1032E03D163689B
:10E3C800002BADD189E74FF0B043A1681A6822F459
:10E3D80080120A431A606268B2F5803F10D11A6849
:10E3E80042F480321A60FFF7B5FC0746FFF718FEC3
:10E3F800002895D1FFF7AEFCC01B6428F6D9C5E705
:10E40800B2F5041F04D11A6842F400121A60E6E754
:10E41800196821F480311960196821F40011196014
:10E42800002AE0D1FFF796FC0746FFF7F9FD002820
:10E438003FF476AFFFF78EFCC01B6428F5D9A5E73B
:10E44800042D236903D00C2D0ED1022E0CD1002BE4
:10E458003FF443AF4FF0B0426169536823F0FE4385
:10E4680043EA016353605FE74FF0B046BBB13368DE
:10E4780043F480733360FFF76DFC074633685A0531
:10E4880007D57368626923F0FE4343EA0263736049
:10E498004AE7FFF75FFCC31B022BEFD976E7336827
:10E4A80023F480733360FFF755FC074633685B0538
:10E4B8007FF53AAFFFF74EFCC31B022BF6D965E791
:10E4C8004FF0B042E169D2F8943023F010030B43C7
:10E4D800C2F894304FF0B047D7F8943043F00103B6
:10E4E800C7F89430FFF736FC0646D7F894309A07F9
:10E4F80018D4FFF72FFC831B112BF6D946E7D6F863
:10E50800943023F00103C6F89430FFF723FC074644
:10E51800D6F894309B0705D5FFF71CFCC31B112BBD
:10E52800F6D933E72368580754D50B4F3B68D9050C
:10E5380014D4FFF765FDFFF70DFC06463B68DA05C6
:10E548000CD4FFF707FC831B022BF7D91EE700BF8B
:10E55800440200204C02002000040058E3684FF0F9
:10E56800B046002B58D023F08003052B02BFD6F805
:10E57800903043F00403C6F890304FF0B046FFF7F0
:10E58800E9FBD6F8903043F001030746C6F890300F
:10E5980041F28838D6F890309B0705D4FFF7DAFBAC
:10E5A800C31B4345F6D9F1E6E36823F00403812B46
:10E5B8001BD1FFF7CFFBD6F8903043F08003C6F8A5
:10E5C800903007464FF0B04641F28838D6F8903080
:10E5D800180504D5E06A00284AD1002068E6FFF74C
:10E5E800B9FBC01B4045F1D9D0E6FFF7B3FBD6F81D
:10E5F800903023F08003C6F8903007464FF0B046BD
:10E6080041F28838D6F890301905E3D5FFF7A2FB18
:10E61800C01B4045F6D9B9E6FFF79CFBD6F8903009
:10E6280023F080030746C6F8903041F28838D6F8C0
:10E6380090301A0516D4FFF78DFBD6F8903023F0EA
:10E648000103C6F8903007464FF0B04841F28836CB
:10E65800D8F890309B07BDD5FFF77CFBC31BB342AE
:10E66800F6D993E6FFF776FBC01B4045DFD98DE668
:10E678000C2D4ED04FF0B04302281A6822F0807259
:10E688001A6033D1FFF766FB0546FFF7DEFC38BB9F
:10E69800D4E90C314FF0B0420B43D0682D4901400A
:10E6A8000B43E16B0B43216C0B43616C0B43A16B78
:10E6B80043EA0123D360136843F080731360D3687F
:10E6C80043F08053D360FFF745FB0446FFF7BDFCDA
:10E6D800002882D1FFF73EFB001B0A28F6D955E631
:10E6E800FFF738FB401B0A28CFD94FE6FFF732FB6C
:10E6F8000446FFF7AAFC30B94FF0B042164BD16878
:10E708000B40D360D4E5FFF725FB001B0A28F0D99E
:10E718003CE601283FF4CCAD4FF0B043226BDB68F8
:10E7280003F0030191427FF4D8AD616B03F07002EE
:10E738008A427FF4D2ADA16B03F4FE42B2EB012F03
:10E748007FF4CBAD626C03F0604393423FF445AF76
:10E75800C3E500BF8C80C111FCFFFEEE2DE9F0413E
:10E768000D46044610B90120BDE8F081684E3368B3
:10E7780003F007038B4216D323689A0727D54FF077
:10E78800B047A268BB6823F0F0031343BB60FFF7F0
:10E79800E1FA0646BB68DB0319D4FFF7DBFA831BF3
:10E7A800022BF7D911E0336823F007030B433360DA
:10E7B800FFF7D0FA0746336803F00703AB42DBD014
:10E7C800FFF7C8FAC01B0228F5D90320CCE7236855
:10E7D800580617D54FF0B0476269D7F8083123F0CB
:10E7E8000F0343EA1213C7F80831FFF7B3FA0646D6
:10E7F800D7F80831D90305D4FFF7ACFA831B022BED
:10E80800F6D9E2E723685A0713D54FF0B047E26814
:10E81800BB6823F4E0631343BB60FFF79BFA06462B
:10E82800BB689B0305D4FFF795FA831B022BF7D926
:10E83800CBE72368180714D54FF0B0472269BB68A7
:10E8480023F4605343EAC203BB60FFF783FA06462A
:10E85800BB68590305D4FFF77DFA831B022BF7D950
:10E86800B3E72368DA070FD4294C236803F00703BA
:10E87800AB4239D8FFF7C8FC264B1860264BBDE8D9
:10E88800F0411868FFF72ABA6268022A1DD1FFF71B
:10E89800C7FB00283FF467AF4FF0B04641F2883815
:10E8A800B36823F003031343B360FFF753FA074633
:10E8B800B368626803F00C03B3EB820FD4D0FFF7A0
:10E8C80049FAC01B4045F3D97FE7032A02D1FFF775
:10E8D800BCFBDEE712B9FFF7A9FBDAE74FF0B0435C
:10E8E8001B685B05D8D43EE7236823F007032B4356
:10E8F8002360FFF72FFA0646236803F00703AB42AD
:10E90800B8D0FFF727FA801B0228F5D95DE700BFCA
:10E9180000400058440200204C02002030B5046832
:10E9280091FAA1F3B3FA83F303255B0005FA03F325
:10E9380024EA030391FAA1F1B1FA81F149008A406E
:10E948001A43026030BD0000B0F1904F0BD14FF078
:10E95800B043DA6A42F00102DA62DA6A22F00102AE
:10E96800DA6201207047144B984209D14FF0B04346
:10E97800DA6A42F00202DA62DA6A22F00202EFE7A9
:10E988000E4B984209D14FF0B043DA6A42F00402C4
:10E99800DA62DA6A22F00402E2E7094B984209D106
:10E9A8004FF0B043DA6A42F08002DA62DA6A22F0A3
:10E9B8008002D5E70020704700040048000800489E
:10E9C800001C00482DE9F84F0E460F6897FAA7F586
:10E9D8004FF0010BB5FA85F54FF0030A4FF00F0819
:10E9E80037FA05F302D10120BDE8F88F0BFA05F4D8
:10E9F8003C4053D0D6F8049021464A46FFF78EFF94
:10EA080009F1FF33012B19D8B368816894FAA4F28D
:10EA1800B2FA82F252000AFA02F221EA020294FAE7
:10EA2800A4F1B1FA81F149008B4013438360426835
:10EA3800F36822EA04026343134343603369C168FD
:10EA480094FAA4F2B2FA82F252000AFA02F221EA25
:10EA5800020294FAA4F1B1FA81F149008B40134300
:10EA6800B9F1020FC36015D1FF2C716918D8026A79
:10EA780094FAA4F3B3FA83F39B0008FA03F322EAA7
:10EA8800030294FAA4F3B3FA83F39B0001FA03F3A5
:10EA9800134303624A462146FFF740FF01359FE7CB
:10EAA800426A230A93FAA3FCBCFA8CFC4FEA8C0C4A
:10EAB80008FA0CFC22EA0C0293FAA3F3B3FA83F3E4
:10EAC8009B00994011434162E4E700002DE9F041C1
:10EAD800076817F001070546884647D1D8F810207F
:10EAE800D8F8083001681343D8F814201343204A93
:10EAF8000A40134303604368D8F80C2023F44053BA
:10EB0800134343608368D8F8182023F440731343F1
:10EB180083604FF4406000F09FF9D8F80060044625
:10EB280010B3D8F80440FCB1B3B2124A394632F8EF
:10EB380013203B46F2F74CFA090241EA10616308D8
:10EB48000002C01822463B4641F10001F2F740FAA4
:10EB5800C0F31300E8600120EB6AB6B223F00F039C
:10EB68001E43EE62BDE8F0812046F5E70020F9E794
:10EB7800F3E9FFEF444401084FF0B0431868C0F3CD
:10EB8800005070474FF0B0431868C0F380207047BA
:10EB98004FF0B043D3F89000C0F3400070474FF0F7
:10EBA800B0431868C0F3C00070474FF0B04318680E
:10EBB800C0F34060704700004FF0B043044A9B68C0
:10EBC800C3F3031352F82330B0FBF3F0704700BFD0
:10EBD800A44301084FF0B043034A9B68C3F30223E0
:10EBE80052F82330D8407047E44301084FF0B04250
:10EBF80038B5916801F00C01082950D017D889B3AD
:10EC0800042900F08C80FFF7CAFF46490246002815
:10EC180076D1FFF7C4FF4FF0B043012816BFD3F8F1
:10EC280094201B68C2F3032251F822002AE00C2921
:10EC3800E9D1D36803F00303022B5FD0032B37D04D
:10EC4800FFF7ADFF374C014600284AD1FFF7A7FF71
:10EC5800012816BFD2F894101368C1F3032154F8A1
:10EC680021302CE0FFF79BFF2E4D044658B9FFF7E3
:10EC780096FF012816BFD2F894401368C4F3032402
:10EC880055F8240038BDFFF78AFF01280ABF11682C
:10EC9800D2F89430C1F3031155F82100F2E7FFF7D9
:10ECA8006BFF214B01462148012908BF1846E9E7B7
:10ECB800FFF762FF1D4A1C4B012818BF13464FF08F
:10ECC800B042D068D168D268C0F306205843C1F377
:10ECD80002130133B0FBF3F0530F0133B0FBF3F031
:10ECE800D0E7FFF75CFF01280BBF1368D2F8943018
:10ECF800C3F30313002354F82330E0E70A4BDEE79D
:10ED0800FFF74DFF4FF0B04301280BBF1B68D3F846
:10ED18009430C3F30313002351F82300B2E70248E9
:10ED2800B0E700BF044401080024F4000048E801EB
:10ED38004FF0B04307B51A6842F001021A601A682A
:10ED48009207FCD51A6822F0F00242F060021A60BD
:10ED58005A6822F47F425A605A6822F0FE4242F012
:10ED680080425A604FF4E0229A601A680192019931
:10ED7800104A0A400192019A1A60FFF716FF00280C
:10ED8800FBD14FF0B0430C4ADA6040F23F32986151
:10ED98000192019A1A62D3F8942042F40002C3F84F
:10EDA800942001204FF44032C3F8082103B05DF8E5
:10EDB80004FB00BFFFF4CEFE0010042210B54FF094
:10EDC800B0440328D4F888302AD11F4A03F003033B
:10EDD80043F44033934209D0B3F1031F0DD0013AF5
:10EDE800934211D1BDE81040FFF700BFFFF7CAFEFC
:10EDF8000128164818BF002010BDFFF7C9FE431EA2
:10EE080058425841C003F7E7FFF7F0FEFFF7D4FE7A
:10EE1800A3680F4AC3F3C22352F82330D840EBE764
:10EE2800034043EA00400B4B9842DFD0B0F10C1F7F
:10EE3800E3D0043B9842D5D0FFF7D8FEFFF7BCFEDD
:10EE4800BDE81040FFF7C6BE020003000024F4002E
:10EE5800E443010808000C0008B54FF0B043D3F8AC
:10EE680088301840B0F5006F09D0B0F5406F0DD06C
:10EE7800B0F5806F11D1BDE80840FFF7B7BEFFF7C6
:10EE880081FE0128094818BF002008BDFFF780FE51
:10EE9800431E58425841C003F7E7FFF7A7FEFFF7A4
:10EEA8008BFEBDE80840FFF795BE00BF0024F400C4
:10EEB80003685B0670B502462DD4D1E900363343AA
:10EEC800CE68056848690C6A33430E6933438E6916
:10EED80003433343CE6925F47F45334325F0BF050B
:10EEE80023432B43136053688D6823F4706323F026
:10EEF800040345EA10401843B5F5006F50603EBF63
:10EF0800536843F480535360B4F5005F01D18B8C90
:10EF18001361012000E00020D36923F40063D3616A
:10EF280070BD00001A4A0368904210B502D0B0F1D3
:10EF3800804F09D14C6823F07003904243EA0403E0
:10EF480009D0B0F1804F06D0124A904203D002F5A2
:10EF58008062904203D1CA6823F44073134303606C
:10EF68008B68C3620B888362094B984207D003F50C
:10EF7800C053984203D003F58063984201D10B69CE
:10EF88000363436943F001034361012010BD00BFDF
:10EF9800002C0140004401400F4B98420BD14FF028
:10EFA800B0431A6C42F480421A641A6C22F480420C
:10EFB8001A6401207047094B98420AD14FF0B043B8
:10EFC8009A6B42F400329A639A6B22F400329A6385
:10EFD800EFE70020704700BF0038014000440040C0
:10EFE80038B50368DB0704460D464DD42A69AB687B
:10EFF800016813436A691343EA691343234A0A40C1
:10F00800134303604368EA6823F44053134343609F
:10F018008368AA6923F44073134383601C4B9842A6
:10F0280020D10320FFF7CAFE2B68F0B16A68E2B16D
:10F038000B2B15D8174951F82330E969B0FBF3F0C9
:10F04800B1F5004F4FEA520319D103EB4003B3FB6C
:10F05800F2F34FF6F0721A40C3F342031343E3602E
:10F06800012003E00C4B984207D00020E26A2B886D
:10F0780022F00F021343E36238BD0C20D2E70344A9
:10F08800B3FBF2F39BB2EAE70020F5E7F369FFEF81
:10F09800003801405C4401080044004010B53024A9
:10F0A800632807D80C703021092808D8303011702F
:10F0B800187010BD01346438E4B2C0B2F0E7013111
:10F0C8000A38C9B2C0B2EFE730B5302442F20F7542
:10F0D800A84212D80C703021B0F57A7F14D2117082
:10F0E8003022632816D81A703023092817D8039AB3
:10F0F8001370049B3030187030BDA0F51C500134DB
:10F108001038E4B280B2E3E70131A0F57A70C9B2F1
:10F1180080B2E1E701326438D2B280B2E1E701336C
:10F128000A38DBB280B2E0E770B5324D324E302497
:10F13800A84232D80C70314D314C3021A04230D821
:10F1480011703049302288422FD21A702E4A30234B
:10F1580090422ED8049A13702C4A302390422FD80C
:10F16800059A1370302342F20F7290422ED8069AF5
:10F1780013703023B0F57A7F2ED2079A137030239C
:10F1880063282ED8089A1370302309282DD8099A95
:10F1980013700A9B3030187070BD0134E4B23044EB
:10F1A800C6E70131C9B22844C8E70132D2B2401AD1
:10F1B800C9E70133A0F57420DBB2A0F51070C7E7EA
:10F1C8000133A0F5C330DBB2A038C7E70133A0F59F
:10F1D8001C50DBB21038C8E70133DBB2A0F57A70F7
:10F1E800C8E70133DBB26438CAE70133DBB20A3857
:10F1F800CBE700BFFFC99A3B003665C4001F0AFA77
:10F20800FFE0F505809698003F420F009F860100B9
:10F2180010B58B1C0C464A1CFFF740FF0023E37017
:10F2280010BD002810B50C460FDA10F1800F0FD072
:10F238004042C0B22D222346611C03F8032BA21CB6
:10F24800FFF72CFF0023237110BDC0B22022F2E784
:10F258002D228020EFE713B50B1D0193CB1C0093E3
:10F268004A1C8B1C0C46FFF72FFF0023637102B06A
:10F2780010BD10B588B001F10903069301F1080328
:10F288000593CB1D04938B1D03934B1D02930B1DFC
:10F298000193CB1C00934A1C8B1C0C46FFF744FFC0
:10F2A8000023A37208B010BD0A2230B5012314460A
:10F2B800824207D95A1E12B20A24150406D5002222
:10F2C800CA5430BD01339BB26243F1E7B0FBF4F599
:10F2D80004FB1500303088542846013AEDE7031E38
:10F2E80010B50C4603DBBDE81040FFF7DDBF584200
:10F2F8000131FFF7D9FF2D23237010BD10B5034C42
:10F308002146FFF785FF204610BD00BF9C4900201D
:10F3180010B5034C2146FFF784FF204610BD00BFFF
:10F328009C49002010B5034C2146FFF794FF204666
:10F3380010BD00BF9C49002010B5034C2146FFF7C3
:10F3480098FF204610BD00BF9C49002013B50368F4
:10F358008DF807109C680DF107010123A04702B042
:10F3680010BD07B503688DF807101B6901220DF160
:10F378000701984703B05DF804FB2DE9F0411D46ED
:10F38800036804465B690F4616469847236820467B
:10F398001B689847221D39462046FFF7D7FF2DB135
:10F3A80023682A461B693146204698472368204629
:10F3B8005B689847236820469B69BDE8F0410C21AB
:10F3C80018472DE9F0411E46036804465B69154657
:10F3D8000F469847236820461B689847221D3946E0
:10F3E8002046FFF7B3FF20460021FFF7BAFF236846
:10F3F8002046DB68324629469847236820465B68E2
:10F40800BDE8F04118472DE9F0411F46036804465E
:10F418005B690D4616469847236820461B6898473F
:10F42800221D20460D21FFF791FF290A2046FFF7EC
:10F4380098FFE9B22046FFF794FF236831463A4621
:10F4480020461B699847236820465B6898472368CD
:10F4580020469B69BDE8F0410C21184707B50123F8
:10F468008DF807200DF10702FFF7CDFF03B05DF817
:10F4780004FB2DE9F0411F46036804465B690D460D
:10F4880016469847236820461B689847221D204641
:10F498001D21FFF75BFF290A2046FFF762FFE9B24B
:10F4A8002046FFF75EFF20460021FFF75AFF23683A
:10F4B8002046DB683A4631469847236820465B6811
:10F4C800BDE8F041184707B501230DF10702FFF722
:10F4D800D0FF9DF8070003B05DF804FB2DE9F0416B
:10F4E8001E46036804465B690F461546984723681D
:10F4F80020461B689847221D20460E21FFF726FF4D
:10F5080039462046FFF72DFF236829463246204614
:10F518001B699847236820465B68984723682046FC
:10F528009B69BDE8F0410C2118472DE9F0411E46C2
:10F53800036804465B690F461546984723682046CA
:10F548001B689847221D20461E21FFF7FFFE3946FB
:10F558002046FFF706FF20460021FFF702FF236839
:10F568002046DB68324629469847236820465B6870
:10F57800BDE8F041184710B5002304461A46C021DB
:10F58800FFF7FBFE207910BD37B504460D468DF810
:10F598000710012380210DF10702FFF7EEFE236813
:10F5A800012D9B690CBF322140F2DC51204603B08B
:10F5B800BDE83040184737B501230C468DF80710D1
:10F5C8000DF107028A210546FFF7D7FEAC7103B09B
:10F5D80030BD07B5042309BA01910DEB030286215A
:10F5E800FFF7CBFE03B05DF804FB07B502238DF8E7
:10F5F80004108DF805208F2101AAFFF7BEFE03B085
:10F608005DF804FB37B58DF8063000238DF8073018
:10F618000423044615468DF804108DF805208B2127
:10F628000DEB0302FFF7A9FE40F689012046FFF71C
:10F638004AFF062D16BF40F0040200F0FB02D2B2CA
:10F6480040F6890120468DF80420FFF707FF03B034
:10F6580030BD73B515468DF8033000229DF818307B
:10F668009DF81C608DF8002004468DF801108DF877
:10F6780004308C2106236A468DF802508DF8056007
:10F68800FFF77BFE40F236712046FFF71CFF5EB1A4
:10F6980000F0FB0240F2367120468DF80020FFF79B
:10F6A800DDFE657102B070BD40F00402D2B2F1E730
:10F6B80007B55BBAADF80430BDF810305BBAADF8E9
:10F6C800063049BA082352BAADF80010ADF8022046
:10F6D80019466A46FFF751FE03B05DF804FB07B50B
:10F6E800022301AA1221FFF76CFE9DF804309DF851
:10F6F800050000EB032080B203B05DF804FB07B5FA
:10F70800022349BAADF8041001AA1946FFF735FEDD
:10F7180003B05DF804FB07B502238DF804108DF8DB
:10F7280005208E2101AAFFF728FE03B05DF804FB2F
:10F7380013B56FF07F43994228BF19460B0C044656
:10F748008DF804300B0A8DF805308DF8061001AAE3
:10F7580003238321FFF711FE236864219B69204658
:10F76800984702B010BD13B56FF07F43994228BF88
:10F7780019460B0C04468DF804300B0A8DF8053039
:10F788008DF8061001AA03238221FFF7F6FD2368EE
:10F7980064219B692046984702B010BD37B5032302
:10F7A8000D461446142101AAFFF70BFE9DF80430FC
:10F7B8005B085B422B809DF90530002BB8BF0333F3
:10F7C8009B10237003B030BD37B502230D46144695
:10F7D800132101AAFFF7F5FD9DF804302B709DF861
:10F7E8000530237003B030BD10B543680D4A23F0CF
:10F7F8007F4323F0FF039342044611D1002240F6D1
:10F808000211FFF72BFE40F644112046FFF75BFE7E
:10F8180040F00202D2B240F644112046FFF71EFE25
:10F8280010BD00BF0001010070B505460E46FFF788
:10F8380056FF314604462846FFF761FFA30702D565
:10F848002846FFF7D1FF204670BD07B5002914BF31
:10F85800402320238DF807300DF10702012393215F
:10F86800FFF78BFD03B05DF804FB10B500230446D9
:10F878001A46C121FFF781FD236820469B69BDE830
:10F8880010404621184708B5FFF775FE80B208BD3D
:10F8980007B50023ADF8043001AA02230721FFF7BA
:10F8A8006CFD03B05DF804FB07B5130C8DF805304B
:10F8B80052BA04238DF80410ADF8062097210DEBF9
:10F8C8000302FFF75AFD03B05DF804FB08B50A46CA
:10F8D80040F6AC01FFF7C2FD08BD10B540F6D801EF
:10F8E8000446FFF7F0FD40F01E02D2B240F6D80100
:10F8F8002046FFF7B3FD10BD08B50A4640F6E701FC
:10F90800FFF7ACFD08BD000007B5054B01930423C4
:10F918000DEB03029521FFF730FD03B05DF804FB02
:10F928000407000107B502238DF804108DF805209F
:10F93800982101AAFFF721FD03B05DF804FB000040
:10F9480013B504461C48B0FBF1F1080C8DF8000013
:10F95800080A8DF8010004988DF803208DF804300A
:10F968008DF80210F0F758FD11A3D3E90023F0F742
:10F97800F7FEF0F7DDFF030C8DF8053043BA6A4651
:10F98800ADF80630204608238B21FFF7F6FC40F639
:10F9980089012046FFF797FD40F00402D2B240F6F5
:10F9A800890120468DF80020FFF758FD02B010BDF0
:10F9B800000000008084EE3F0000093D1FB58DF86F
:10F9C80007309DF818308DF808309DF81C308DF8F8
:10F9D80009309DF820308DF80A309DF824308DF8D4
:10F9E8000B3049BA9DF82830ADF804108DF8062080
:10F9F8008DF80C3001AA09238C21FFF7BEFC05B055
:10FA08005DF804FB07B5002349BAADF80010ADF85E
:10FA1800023001936A4608234FF4D861FFF7F3FCDC
:10FA280003B05DF804FB13B503230C4601AA1421A7
:10FA3800FFF7C7FC9DF806305B085B42238002B0E5
:10FA480010BD000038B5044600F03CFA21460546D2
:10FA58002046F1F761FA80B9204600F067F84FF0C8
:10FA68007E51F1F74FFA40B101F08CFA212303607F
:10FA7800BDE83840024800F097B8284638BD00BFB6
:10FA88000412010800F060BB38B5054600F090F894
:10FA9800294604462846F1F73FFA68B90021284666
:10FAA800F1F712FA40B101F06DFA21230021036049
:10FAB8000846F1F71FF90446204638BD07B51A4A2B
:10FAC80020F000439342014605DC002103B05DF8B5
:10FAD80004EB00F001B9B3F1FF4F04DBF0F74CFF82
:10FAE80003B05DF804FB694600F0B4FB00F00302C4
:10FAF800012A07D0022A0CD082B90199009800F097
:10FB0800EBF8EDE70199009800F066F900F1004084
:10FB1800E6E70199009800F0DFF8F7E70199009807
:10FB2800012200F059F9DBE7D80F493F20F00040E7
:10FB38007047000007B51B4A20F000439342014676
:10FB480006DC0022002103B05DF804EB00F044B9A4
:10FB5800B3F1FF4F04DBF0F70FFF03B05DF804FBD0
:10FB6800694600F077FB00F00300012808D002285E
:10FB78000BD090B901990098012200F02DF9ECE71B
:10FB88000199009800F0A8F8E7E701990098012288
:10FB980000F022F900F10040DFE70199009800F039
:10FBA8009BF8F7E7D80F493F004870470000C07F2F
:10FBB80020F00042B2F1FF4F2DE9F0410346044620
:10FBC8000AD30146F0F7E2FF01462046F0F7D6FED9
:10FBD80004462046BDE8F081002AFAD0002806DA5B
:10FBE8000146F0F7C9FE0146F1F784F8F0E710F096
:10FBF800FF424FEAE0513DD0C3F3160343F400033C
:10FC0800CA07A1F17F0558BF5B0000246D105B0097
:10FC1800192026464FF0807172189A42DDBF561897
:10FC280064189A1A1A4601384FEA42034FEA5101FA
:10FC3800F2D1BAB1144E154F30683968D6F8008041
:10FC4800F0F79AFE01464046F1F748F950B130689E
:10FC580039683668F0F792FE01463046F1F734F914
:10FC680068B10234641004F17C5404EBC554B0E765
:10FC78005B0001321802FBD5013A891ABCE701344E
:10FC880024F00104EEE700BF5002002054020020D7
:10FC9800C0F3C7537F3B162B10B5014614DC002B6D
:10FCA80007DA013300F0004101D141F07E510846E6
:10FCB80010BD084A1A411042F9D04FF48001194189
:10FCC800014421EA0201F2E7802BF0D1F0F756FE59
:10FCD8000146ECE7FFFF7F002DE9F04120F00044EA
:10FCE800B4F1485F0646884603DAF1F72BF9002895
:10FCF8005CD031463046F0F749FF4FF07C5105465D
:10FD0800F0F744FF2B4907462846F0F73FFF2A49FA
:10FD1800F0F734FE2946F0F739FF2849F0F72CFEB2
:10FD28002946F0F733FF2649F0F728FE2946F0F771
:10FD38002DFF2449F0F720FE2946F0F727FF224936
:10FD4800F0F71CFE2946F0F721FF2946F0F71EFFC1
:10FD5800414605463046F0F719FF01462846F0F7B8
:10FD68000BFE1A4B9C4205460ADC01463846F0F762
:10FD780003FE01464FF07E50F0F7FEFDBDE8F0812E
:10FD8800134B9C42CCBF134C04F17F4421464FF0E7
:10FD98007E50F0F7F1FD214606463846F0F7ECFDB7
:10FDA8002946F0F7E9FD01463046E5E74FF07E5079
:10FDB800E4E700BF4ED747ADF6740F317CF29334B9
:10FDC800010DD037610BB63AABAA2A3D9999993EF5
:10FDD8000000483F0000903E2DE9F84320F0004322
:10FDE800B3F1485F04460F46914603DAF1F7AAF8E3
:10FDF800002835D021462046F0F7C8FE05460146C2
:10FE08002046F0F7C3FE294906462846F0F7BEFE0D
:10FE18002749F0F7B1FD2946F0F7B8FE2549F0F774
:10FE2800ADFD2946F0F7B2FE2349F0F7A5FD2946B6
:10FE3800F0F7ACFE2149F0F7A1FD8046B9F1000FBB
:10FE480011D101462846F0F7A1FE1D49F0F794FDAF
:10FE58003146F0F79BFE01462046F0F78FFD044639
:10FE68002046BDE8F8834FF07C513846F0F78EFE07
:10FE7800414681463046F0F789FE01464846F0F78C
:10FE88007BFD2946F0F782FE3946F0F775FD0C49EF
:10FE980005463046F0F77AFE01462846F0F76EFD33
:10FEA80001462046F0F768FDD9E700BFD3C92E2FD9
:10FEB800342FD7321BEF3836010D50398988083C6A
:10FEC800ABAA2A3E2DE9F04720F00048B8F17E5F42
:10FED800044605460CD18C49F0F758FE8B49054677
:10FEE8002046F0F753FE01462846F0F747FD06E0A6
:10FEF80009DD0146F0F740FD0146F0F7FBFE044638
:10FF08002046BDE8F087B8F17C5F0BDAB8F1485FAE
:10FF180073DA7F49F0F732FD4FF07E51F0F7F2FFC8
:10FF28000028EDD12046FFF701FE01464FF07E5034
:10FF3800F0F722FD4FF07C51F0F728FE7549064690
:10FF4800F0F724FE7449F0F719FD3146F0F71EFE6C
:10FF58007249F0F711FD3146F0F718FE7049F0F7D5
:10FF68000DFD3146F0F712FE6E49F0F705FD3146FA
:10FF7800F0F70CFE6C49F0F701FD3146F0F706FE8C
:10FF88006A4981463046F0F701FE6949F0F7F4FC0A
:10FF98003146F0F7FBFD6749F0F7F0FC3146F0F722
:10FFA800F5FD6549F0F7E8FC3146F0F7EFFD4FF055
:10FFB8007E51F0F7E3FC82463046FFF7F9FD5F4BD0
:10FFC8009845074663DD51464846F0F793FE3946A3
:10FFD800F0F7DCFD3946F0F7D1FC0146F0F7CEFC2E
:10FFE8005749F0F7CBFC01464748F0F7C5FC002D10
:08FFF8000446D8BF00F10044EB
:020000040801F1
:1000000082E70146F0F7C6FD44490546F0F7C2FD18
:100010004349F0F7B7FC2946F0F7BCFD4149F0F73A
:10002000AFFC2946F0F7B6FD3F49F0F7ABFC294697
:10003000F0F7B0FD3D49F0F7A3FC2946F0F7AAFD23
:100040003B49F0F79FFC2946F0F7A4FD39490646E5
:100050002846F0F79FFD3849F0F792FC2946F0F763
:1000600099FD3649F0F78EFC2946F0F793FD3449A7
:10007000F0F786FC2946F0F78DFD4FF07E51F0F742
:1000800081FC01463046F0F739FE2146F0F782FD4B
:10009000014620462DE7014620F47F68F0F772FC08
:1000A000514604464846F0F729FE01462046F0F73F
:1000B00071FD28F00F08814641464046F0F76AFD81
:1000C00001463046F0F75CFC414604463846F0F7FE
:1000D00059FC01462046F0F711FE0146F0F752FCAC
:1000E00001460C48F0F74CFC01464846F0F748FC46
:1000F000414604464046F0F745FC01461348F0F7F8
:100100003FFC01462046F0F73BFC01460F4870E7F4
:10011000DB0FC93F2EBD3BB3CAF2497108EF11385E
:10012000047F4F3A4611243DA80A4E3E90B0A63EA9
:10013000ABAA2A3E2EC69D3D6133303F2D5701406C
:1001400039D119409999793F2EBD3B33DB0F493F97
:10015000F8B521F00046B6F1FF4F034605DC20F06C
:100160000042B2F1FF4F074604DD1846F0F70AFCE3
:10017000034611E0B1F17E5F03D1BDE8F84000F025
:10018000CBB98C1704F0020444EAD07432B9022CC3
:100190004CD0032C00D1294B1846F8BD1EB9002FB6
:1001A0004ADA274BF8E7B6F1FF4F0ED1B2F1FF4F15
:1001B00004F1FF3405D1022C3AD8224B53F82430F5
:1001C000EAE7022C36D8204BF8E7B2F1FF4FE6D031
:1001D000921BB2F1F45F4FEAE25017DA002901DA1C
:1001E0003C3015DB1846F0F789FDFFF7A3FC00F063
:1001F00093F90346012C0DD0022C0ED0002CCBD04D
:1002000012491846F0F7BEFB11490CE0114BF1E71B
:100210000023EFE703F10043BEE70C491846F0F76F
:10022000B1FB01460A48F0F7ABFBA1E7084BB3E787
:10023000094BB1E70023AFE7064BADE7DB0F49C041
:10024000DB0FC9BF8C440108984401082EBDBB33A5
:10025000DB0F4940DB0FC93FDB0F493F2DE9F04F72
:10026000A04A20F00046964287B00C46824604DC45
:10027000002308604B6000251AE09B4A96424BDC45
:1002800000289A499A4F26F00F0623DDF0F778FBF5
:10029000BE42054610D09749F0F772FB0146206038
:1002A0002846F0F76DFB9349F0F76AFB0125606083
:1002B000284607B0BDE8F08F8F49F0F761FB8F4902
:1002C0000546F0F75DFB014620602846F0F758FB35
:1002D0008A49E9E7F0F756FBBE4205460ED085494C
:1002E000F0F750FB014620602846F0F749FB8149B2
:1002F000F0F748FB4FF0FF356060D9E77E49F0F733
:1003000041FB7E490546F0F73DFB0146206028464B
:10031000F0F736FB7949EBE7794A964200F3918092
:10032000FFF708FC77490746F0F734FC4FF07C51A3
:10033000F0F728FBF0F70AFE0546F0F7D7FB6B490C
:100340008146F0F727FC01463846F0F719FB69496A
:1003500080464846F0F71EFC1F2D07460CDC6A4A13
:10036000691E26F0FF0352F82120934204D039463B
:100370004046F0F705FB0BE039464046F0F700FB3E
:10038000C0F3C753C3EBD653082B4FEAE65B01DC3F
:10039000206026E058494846F0F7FCFB0746014636
:1003A0004046F0F7EDFA014606464046F0F7E8FA17
:1003B0003946F0F7E5FA514907464846F0F7EAFBB7
:1003C0003946F0F7DDFA014607463046F0F7D8FA2D
:1003D000C0F3C753ABEB030BBBF1190F16DC206066
:1003E000B046266840463146F0F7CAFA3946F0F77B
:1003F000C7FABAF1000F6060BFF65AAF06F10046C7
:1004000000F10040266060606D4251E73F49484678
:10041000F0F7C0FB074601463046F0F7B1FA014657
:1004200080463046F0F7ACFA3946F0F7A9FA384979
:1004300006464846F0F7AEFB3146F0F7A1FA07460C
:1004400095E7B6F1FF4F05DB0146F0F799FA6060DA
:10045000206010E7F715863FA6EBC7563046F0F749
:1004600075FDF0F743FB014603903046F0F788FA3C
:100470004FF08741F0F78EFB0646F0F767FDF0F787
:1004800035FB0146049005463046F0F779FA4FF007
:100490008741F0F77FFB00210590F0F70FFDF0B1E9
:1004A00000212846F0F70AFD002814BF012302238B
:1004B000184A01920222009221463A4603A800F00F
:1004C00037F9BAF1000F0546BFF6F2AE236803F123
:1004D00000432360636803F10043636094E70323F0
:1004E000E6E700BFD80F493FE3CB1640800FC93F76
:1004F000D00FC93F434435370044353708A3852E14
:10050000800F494384F9223FA444010800A3852EAB
:1005100032318D24244501082DE9F04120F00045B9
:10052000B5F1A14F044680460EDBB5F1FF4F04DD67
:100530000146F0F727FA044603E0002800F3CE80D6
:10054000674C2046BDE8F081664B9D420EDCB5F15C
:10055000445F08DA6449F0F715FA4FF07E51F0F77E
:10056000D5FC0028EDD14FF0FF361CE0FFF7E2FA92
:100570005E4B9D4204467CDCA3F5D0039D4267DCC4
:100580000146F0F7FFF94FF07E51F0F7F9F94FF01F
:10059000804105462046F0F7F5F901462846F0F778
:1005A000ADFB0026044621462046F0F7F3FA01464B
:1005B0000746F0F7EFFA4E490546F0F7EBFA4D49DA
:1005C000F0F7E0F92946F0F7E5FA4B49F0F7DAF9E8
:1005D0002946F0F7DFFA4949F0F7D4F92946F0F750
:1005E000D9FA4749F0F7CEF92946F0F7D3FA454949
:1005F000F0F7C8F93946F0F7CDFA434907462846DF
:10060000F0F7C8FA4149F0F7BBF92946F0F7C2FA0A
:100610003F49F0F7B5F92946F0F7BCFA3D49F0F744
:10062000AFF92946F0F7B6FA3B49F0F7A9F92946A0
:10063000F0F7B0FA01463846F0F7A4F92146F0F792
:10064000A9FA731C014633D12046F0F799F972E7F5
:100650004FF07E51F0F794F94FF07E510546204659
:10066000F0F790F901462846F0F748FB01260446CA
:1006700099E72A4B9D4214DC4FF07F51F0F780F947
:100680004FF07F5105462046F0F784FA4FF07E5137
:10069000F0F778F901462846F0F730FB02260446C9
:1006A00081E701461E48F0F729FB032604467AE756
:1006B0001C4B53F82610F0F763F92146F0F760F968
:1006C000194B014653F82600F0F75AF9B8F1000F1C
:1006D0000446BFF636AF00F1004432E7134C30E772
:1006E000DB0FC9BFFFFFDF3ECAF24971FFFF973F33
:1006F000D769853C59DA4B3D356B883D6E2EBA3D46
:100700002549123EABAAAA3E21A215BD6BF16E3D52
:1007100095879D3D388EE33DCDCC4C3EFFFF1B4081
:10072000000080BF4C4801083C480108DB0FC93F6E
:100730002DE9F04FDBB002920493649ABB4B059015
:1007400053F822300193049B0091013B0393029BD9
:100750001A1DC0F29B80DC1E48BF1C1DE410671CE4
:10076000FB000693029B039AA3EBC707019B03EBD5
:100770000209659BA4EB02081EAE03EB880A002564
:100780004FF0000B4D4540F38380049A1EAB03EB02
:1007900082050DF58C7B4FF000090023019A9145ED
:1007A00040F39E8013460AAA02EB83030893659BDD
:1007B000DDF8048003EB840307935AAB03EB880353
:1007C0000AAC53F8505C2646C3464FF087490DF5F6
:1007D0008C7ABBF1000F00F388803946284600F080
:1007E0005BFA4FF078510546F0F7D4F900F0A0FA23
:1007F0004FF08241F0F7CEF901462846F0F7C0F8F5
:100800000546F0F7A3FB0646F0F770F901462846C7
:10081000F0F7B6F8002F814640F3868008F1FF32EA
:100820000AABC7F1080153F8225045FA01F31E4400
:100830008B40ED1A0AAB43F82250C7F107031D4164
:10084000002D7FDD002201369246904500F3B080F6
:10085000002F05DD012F00F0BD80022F00F0C580C4
:10086000022D6FD149464FF07E50F0F789F881464E
:10087000BAF1000F66D039464FF07E5000F00CFA06
:1008800001464846F0F77CF881465BE0002466E7C5
:1008900018EB050F07D45AF82500F0F727F946F8AA
:1008A000040B01356EE75846F9E70793059BDAF824
:1008B000001053F82800F0F76DF901463046F0F7C4
:1008C00061F8079B064608F10108039A9045AAF1D2
:1008D000040AEADD4BF8046B09F1010904355DE710
:1008E000AA461E464FF00008EFE74FF06E5128462B
:1008F000F0F750F9F0F72AFBF0F7F8F849460990BD
:10090000F0F748F901462846F0F73AF8F0F71EFBF1
:100910000BF1FF3B099B46F8040B5AF82B101846C5
:10092000F0F730F8054654E706D108F1FF330AAA7C
:1009300052F82350ED1183E74FF07C51F0F7DCFAC9
:10094000054698BB00214846F0F7B8FA002800F0A9
:10095000988008F1FF342346002201998B424CDA3B
:10096000002A67D00AAB083F53F82430002B00F070
:10097000868039464FF07E5000F08EF9A2468146BF
:1009800046AF4FF06E58BAF1000F80F2AF802746A5
:100990000022002FC0F2D98046A9254B01EB870B1E
:1009A00090464FF0000AA4EB0709C2E0022549E790
:1009B0002368BAF1000F08D11BB1C3F5807323601F
:1009C0000123013204349A463FE7C3F1FF03236059
:1009D0005346F6E708F1FF320AAB53F8223003F032
:1009E0007F030AA941F822303AE708F1FF320AAB47
:1009F00053F8223003F03F03F3E70AA951F823101C
:100A0000013B0A43A9E7013453F8042D002AFAD028
:100A1000049B1EAA434408F1010602EB83054444EB
:100A20000DF58C79B44208DAA046C6E6884801087C
:100A30005C480108089B0124E6E7079B53F8260061
:100A4000F0F754F8AB4628604FF0000A4FF000086A
:100A5000039B9A4504DD49F8268004350136E1E719
:100A6000059B5BF8040953F82A10F0F793F8014648
:100A70004046EFF787FF0AF1010A8046E8E7013CAC
:100A800070E7069B029A4846991A00F005F94FF064
:100A900087410446F0F730FA00B34FF06E5120461C
:100AA000F0F778F8F0F752FAF0F720F84FF08741B6
:100AB0008146F0F76FF801462046EFF761FFF0F747
:100AC00045FA0AAB08F1010443F828004846F0F75C
:100AD0003DFA0AAB083743F824004AE72046F0F70E
:100AE00035FA0AAB444643F8280042E70AAB53F80C
:100AF0002A00EFF7FBFF4946F0F74CF8414647F86C
:100B00002A004846F0F746F80AF1FF3A81463AE7EC
:100B100053F8040B5BF8041B03920293F0F73AF8C6
:100B200001464046EFF72EFFDDE9023280460AF12A
:100B3000010A01998A4501DCCA45E9DD5AAB03EB9C
:100B40008909013F49F8A08C23E7649B022B07DC4D
:100B5000002B4EDC2ED006F007005BB0BDE8F08F16
:100B6000649B032BF7D10DF1C80B0BEB8407B84640
:100B7000A246BAF1000F49DCA146B9F1010F60DCD1
:100B80000020012C76DC329A339B002D78D100991D
:100B90000A604B600A469060DDE757F82410EFF7D3
:100BA000F1FE013C002CF8DA0DB100F10040009B91
:100BB0001860D0E7002032AFF4E757F82810EFF7BD
:100BC000E1FE08F1FF38B8F1000FF6DAADB100F13F
:100BD0000043009A014613603298EFF7D1FE4FF0C0
:100BE000010844450BDA0DB100F10040009B58604C
:100BF000B1E7A046002032AFE5E70346E9E757F842
:100C0000041FEFF7BFFE08F10108EAE7D8F800304B
:100C100058F8042C0293194610460192EFF7B2FEE1
:100C2000019A014681461046EFF7AAFE029B19463B
:100C3000EFF7A8FE48F804090AF1FF3AC8F8009057
:100C400097E757F8043CD7F800A00193514618469F
:100C5000EFF798FE019B014680461846EFF790FE9D
:100C60005146EFF78FFE47F8040909F1FF39C7F83D
:100C7000008082E75BF82410EFF784FE013C80E7F8
:100C8000009902F1004203F100430A604B600A46FA
:100C900000F100407FE700BF30F0004238B5034666
:100CA0000D4604462ED0B2F1FF4F04D30146EFF7B4
:100CB00069FE034626E010F0FF4F18D14FF098412F
:100CC000EFF768FF174A954203460CDBC0F3C752A3
:100CD0000446193A4CF250318D420ADD1249184649
:100CE00061F31E0000E01149EFF754FFE1E7D20D78
:100CF000F0E75119FE29F1DC002905DD24F0FF445D
:100D000044EAC153184638BD11F1160F01DA0749FC
:100D1000E5E701F1190024F0FF444FF04C5144EA9B
:100D2000C050E1E7B03CFFFFCAF249716042A20D3A
:100D300070B5C0F3C7557F3D162D0146044620F01F
:100D4000004625DC002D0EDA1649EFF71BFE0021C8
:100D5000F0F7DCF828B1002C22DA134B002E18BF74
:100D60001C4621461AE0114E2E41304216D00D4944
:100D7000EFF708FE0021F0F7C9F80028F1D0002CA9
:100D8000BEBF4FF400032B41E41824EA0604E8E751
:100D9000B6F1FF4F02D3EFF7F5FD0146084670BDEF
:100DA0000024DEE7CAF24971000080BFFFFF7F0028
:100DB0000A22002100F07EB8012B2DE9F04786467B
:100DC000904601D0242B06D900F0E0F816230360EA
:100DD0000020BDE8F08736480D462A4615F8014B3D
:100DE000065D16F00806F8D12D2C2ED12C780126A0
:100DF000951C002B57D0102B09D1302C07D12A7805
:100E000002F0DF02582A49D16C781023023506F12E
:100E1000004C0CF1FF3C0022BCFBF3F9104603FB35
:100E200019CAA4F13007092F14D83C46A34220DD8B
:100E3000571C07D0814519D301D1A24516DB00FB11
:100E40000340012215F8014BEBE72B2C04BF2C7853
:100E5000951CCEE7A4F14107192F01D8373CE5E7EF
:100E6000A4F16107192F04D8573CDFE74FF0FF3298
:100E7000E8E7531C08D12223CEF800306046B8F1D1
:100E8000000FA6D0691E06E006B14042B8F1000F7F
:100E90009FD0002AF6D1C8F800109AE73024002B22
:100EA000B5D10823B3E7302CA9D00A23AFE700BFA0
:100EB0009548010813460A46014602480068FFF7B4
:100EC0007BBF00BFA4020020024B0344587800F00F
:100ED0000300704794480108034B1B5C03F00303B5
:100EE000022B08BF2038704795480108884210B58A
:100EF00001EB020402D98442234607D8431EA142D3
:100F000008D011F8012B03F8012FF8E7024401463D
:100F10008A4200D110BD13F8014D02F8014DF7E7E8
:100F200002440346934200D1704703F8011BF9E7DE
:100F300010B50246147813460132002CFAD1013B59
:100F400011F8012B03F8012F002AF9D110BDC9B205
:100F50000346184613F8012B12B18A42F9D17047A3
:100F6000002918BF0020704710B56AB101398418F4
:100F700010F8012B11F8013F9A4203D1A04201D091
:100F8000002AF5D1D01A10BD1046FCE7014B1868B5
:100F9000704700BFA402002070B50D4D0D4C641BBE
:100FA000A4100026A64209D10B4D0C4C00F02EF8DF
:100FB000641BA4100026A64205D170BD55F8043B61
:100FC00098470136EEE755F8043B98470136F2E7BB
:100FD000A0490108A0490108A0490108A849010841
:100FE000034611F8012B03F8012B002AF9D17047B1
:100FF0000A44914200F1FF3300D1704710B511F857
:10100000014B03F8014F9142F9D110BDF8B500BF73
:10101000F8BC08BC9E467047F8B500BFF8BC08BCD9
:041020009E46704731
:1010240000080008005001500250035004500550BD
:1010340006500750085009500A500B500C500D50E0
:10104400F150F25001F105500000000001000000D1
:10105400020000006D696E2C00206D572C00205793
:101064002C002E00011F136F01130503020B050250
:1010740000D57FAAFE2B815429FC5683D702A87D74
:1010840052872DF8AC79D3067BAE04D18550FA2F64
:10109400A471DB0E5A8F25F08D58F22773A60CD954
:1010A400F623895C08DD77A2DF0AA07521F45E8B44
:1010B4009D48E23763B61CC9B461CB1E4A9F35E034
:1010C400CF1AB06531E44E9BE633994C18CD67B224
:1010D40039EC4693C712B86D10C56FBAEE3B914414
:1010E4006BBE14C19540EA3F42973DE8BC69C31604
:1010F400EF3A904511C46EBBC613B96C38ED4792F4
:10110400BD68C21743963CE99441EB3E6ABF15C0E3
:101114004B9E34E1B560CA1F62B71DC89C49E336D3
:1011240019CC66B3E732984D30E54F9ACE1BB164C3
:1011340072A70DD88C59F3265B8E24F1A570DA0FB3
:1011440020F55F8ADE0BA17409DC76A3F722885DA3
:10115400D603A97C28FD5782FF2A805501D47EAB93
:101164008451FB2E7AAF05D0AD78D20753862CF983
:101174006162636465666768696A6B6C6D6E6F70E3
:101184007172737475767778797A30313233343595
:10119400363738395F232D2E000000000000000090
:1011A40000000000371C00080000000000000000E0
:1011B400431C000800000000000000001F1C000881
:1011C4006D6C72732E300053657475705374617254
:1011D400745374783454780053657475705374611F
:1011E40072744D61726B65720021656E6421006DCD
:1011F4004C525301020304006D4C52530403020188
:1012040000656E61626C65642C616E74656E6E61FE
:10121400312C616E74656E6E61322C723A656E2E7D
:1012240020743A616E74312C723A656E2E20743AD1
:10123400616E7432007472616E73702E2C6D6176FF
:101244006C696E6B2C6D61766C6E6B582C6D737063
:101254005800322E342047487A2C393135204D48F5
:101264007A204643432C383638204D487A2C343380
:1012740033204D487A2C373020636D2048414D2C63
:10128400383636204D487A20494E00656E61626CCE
:1012940065642C616E74656E6E61312C616E74656B
:1012A4006E6E61322C72656E207461312C72656EC3
:1012B4002074613200353020487A2C333120487A4A
:1012C4002C313920487A2C464C52432C46534B2C13
:1012D4003139487A377800322E342047487A2C390D
:1012E4003135204643432C383638204D487A2C3447
:1012F4003333204D487A2C373020636D2C38363602
:1013040020494E00202F2D2D00202F653100202F45
:10131400653600202F65313100202F653133000DF3
:101324000A00212120527820706172616D20766557
:101334007273696F6E20736D616C6C657220746872
:10134400616E20547820706172616D2076657273CD
:10135400696F6E2E20212100212120506C6561735C
:10136400652075706772616465207265636569766E
:1013740065722E20202020202020202020202020C4
:101384002020202020202020202020212100212175
:1013940020547820706172616D2076657273696F74
:1013A4006E20736D616C6C6572207468616E20527E
:1013B4007820706172616D2076657273696F6E2E2C
:1013C40020212100212120506C65617365207570F6
:1013D4006772616465205478206D6F64756C652E46
:1013E40020202020202020202020202020202020F9
:1013F40020202020202020212100436F6E66696771
:1014040049643A003F0020206D696E3A2000202094
:101414006D61783A2000202000203D200020205BD0
:10142400612D7A302D39232D2E5F5D002D202875F6
:101434006E617661696C61626C652900205B0028CD
:10144400756E6368616E676561626C6529007761BA
:10145400726E3A207265636569766572206E6F7488
:1014640020636F6E6E6563746564002800292C0028
:101474002C20003B20003B00202054783A20576960
:101484006F4535204D696E6920574C45354A432CCC
:101494002076312E332E303600202052783A200028
:1014A4002D2028756E657870656374656420657297
:1014B400726F722900202063683A20002020665F42
:1014C4007265673A20002020663A2000206B487A33
:1014D40000202068656C702C20682C203F20202D73
:1014E4003E20746869732068656C7020706167655C
:1014F4000020207620202020202020202020202DA5
:101504003E207072696E742064657669636520613B
:101514006E642076657273696F6E002020706C2093
:101524002020202020202020202D3E206C69737450
:1015340020616C6C20706172616D657465727300FA
:101544002020706C206320202020202020202D3E8D
:10155400206C69737420636F6D6D6F6E207061729F
:10156400616D6574657273002020706C207478203E
:101574002020202020202D3E206C69737420547874
:1015840020706172616D6574657273002020706CE7
:10159400207278202020202020202D3E206C69738A
:1015A4007420527820706172616D65746572730085
:1015B400202070206E616D652020202020202020B6
:1015C40020202D3E2067657420706172616D657402
:1015D40065722076616C756500202070206E616DE7
:1015E40065203D2076616C756520202D3E20736555
:1015F4007420706172616D657465722076616C75BA
:101604006500202070206E616D65203D203F202004
:10161400202020202D3E2067657420706172616D4A
:10162400657465722076616C756520616E64206CEA
:10163400697374206F6620616C6C6F7765642076C3
:10164400616C7565730020207073746F726520205F
:10165400202020202D3E2073746F726520706172EB
:10166400616D6574657273002020736574636F6EB9
:101674006669676964202D3E2073656C6563742018
:10168400636F6E66696720696400202062696E6416
:1016940020202020202020202D3E2073746172748D
:1016A4002062696E64696E6700202072656C6F61E8
:1016B400642020202020202D3E2072656C6F616400
:1016C40020616C6C20706172616D65746572207349
:1016D400657474696E677300202073746174732079
:1016E4002020202020202D3E2073746172747320EA
:1016F40073747265616D696E672073746174697364
:10170400746963730020206C697374667265717305
:101714002020202D3E206C697374732066726571DD
:1017240075656E63696573207573656420696E20E1
:101734006668737320736368656D65002020737930
:101744007374656D626F6F7420202D3E2063616C2D
:101754006C2073797374656D20626F6F746C6F6144
:10176400646572002020656D70747920636D640077
:101774002020696E76616C696420636D64002020AA
:1017840073747265616D696E67207374617473201C
:1017940073746F70706564003E00202074696D6519
:1017A4006F75740068656C7000706C00706C2063F9
:1017B40000706C20747800706C207278006572720E
:1017C4003A20696E76616C696420706172616D653E
:1017D400746572206E616D65006572723A206E6F79
:1017E4002076616C756520737065636966696564EC
:1017F400006572723A20696E76616C696420766164
:101804006C7565007073746F7265002020547820C5
:10181400706172616D65746572732073746F726543
:1018240064002020706172616D6574657273207349
:10183400746F7265640062696E64002020547820BD
:10184400656E74657265642062696E64206D6F6490
:10185400650072656C6F61640020205478207061AB
:1018640072616D65746572732072656C6F61646515
:1018740064002020706172616D65746572732072FA
:10188400656C6F6164656400736574636F6E66692B
:10189400676964006572723A20696E76616C696486
:1018A40020636F6E666967206964206E756D62657A
:1018B400722028302D39290020206E6F2063686142
:1018C4006E676520726571756972656400202063B6
:1018D40068616E676520436F6E666967496420744A
:1018E4006F200020207374617274732073747265A6
:1018F400616D696E67207374617473002020736571
:101904006E6420616E7920636861726163746572CC
:1019140020746F2073746F70006C697374667265E1
:1019240071730073797374656D626F6F74005769B6
:101934006F4535204D696E6920574C45354A430043
:101944002145525200414952004143524F00214621
:101954005321004D414E55004352555A00435253B2
:101964004800414800414E474C00484F5200414E08
:101974004748002A00414C5448004155544F004701
:10198400554944004C4F49540052544C200043499B
:101994005243004C414E4400445249460053505275
:1019A4005400464C4950004154554E0050484C4454
:1019B400004252414B00544852570041564F49008F
:1019C400474E4750005352544C0046484C4400463E
:1019D4004F4C4C005A49475A0053595349004152FD
:1019E4004F54004152544C005452544C00545241F0
:1019F4004E00464257410046425742004352555317
:101A040000544B4F4600494E495400515354420030
:101A140051484F5600514C4F5400514C4E440051C4
:101A240052544C005141544E005141434F005448CC
:101A34004D4C004C32514C005354455200534D50C0
:101A44004C00444F434B0041484C440053555246CC
:101A5400004D444554005378206E6F74206F6B0022
:101A640072785F617661696C61626C65206E6F7417
:101A74002074727565000000000000000000000082
:101A8400112D0008F52C00088D340008B934000825
:101A9400D734000851310008F122000855460008E7
:101AA4000000000000000000192200083938000876
:101AB40035370008753600084B36000865230008E2
:101AC400D936000881230008A5360008A52300089C
:101AD4000000000000000000192200081B2200087A
:101AE4001D2200081F2200082322000825220008C6
:101AF400292200082D2200082F2200083322000882
:101B0400000000000000000019220008B93A000893
:101B14001D220008453900081B390008A9230008C4
:101B2400853900082D2200082F22000833220008DE
:101B34000000000000000000192200081B22000819
:101B44001D2200081F220008232200082522000865
:101B5400292200082D2200082F2200083322000821
:101B64000000000000000000012500080D660008C8
:101B7400C5660008696600085053544F5245004337
:101B84004F4E4649472049440042494E445F50481D
:101B9400524153455F5533320052465F42414E44F1
:101BA4000052465F4F5254484F0054585F504F57AD
:101BB40045520054585F44495645525349545900BC
:101BC40054585F43485F534F555243450054585F40
:101BD40043485F4F524445520054585F494E5F4D4D
:101BE4004F44450054585F5345525F444553540095
:101BF40054585F5345525F424155440054585F5313
